:020000040800F2
:10000000002000104924030831AE0208B1C90008DD
:100010002FAE02082DAE02082BAE02080000000031
:1000200000000000000000000000000029AE0208EF
:1000300027AE02080000000025AE0208F9DF000824
:10004000B1240308B1240308B1240308B124030830
:10005000B1240308B1240308395F0208656002086F
:1000600029600208ED5F0208B15F0208193100083B
:1000700009310008F9300008E9300008D9300008DB
:10008000C5300008B1300008B1240308B1240308CA
:100090004DAF0208B1240308B1240308755F0208BC
:1000A000B124030889D7000849D70008B1D7000850
:1000B00079D70008B1240308B1240308B124030848
:1000C000B1240308B1240308B1240308B1240308B0
:1000D000B1240308C950020801E1000885E00008C6
:1000E000FD5E0208B124030815AE0208B12403081E
:1000F00059D70008B124030869D70008B1240308C0
:10010000000000000000000000000000B12403080F
:10011000B1240308B1240308F91E0108DD1E0108FB
:100120009D300008893000087530000861300008F3
:100130004D300008B124030800000000000000005A
:10014000B1240308B1240308B1240308000000000F
:10015000000000000000000000000000000000009F
:100160000000000000000000B1240308B1240308CF
:10017000B12403080000000000000000000000009F
:0801800000000000B124030897
:10018800002870B51EDB0928044620DD012303EB97
:1001980083035B00B0FBF3F2092AF8D87BB10E4E5B
:1001A800B4FBF3F00928CCBF57223022A6FB03E5A5
:1001B800024403FB1044EB0801F8012BF0D10023A3
:1001C8000B7070BD2D230B7040420131DBE73030DE
:1001D80001F8010BF3E700BFCDCCCCCC884230B49A
:1001E8004FF001042ED301FB04F4B0FBF4F58D426B
:1001F800F9D284B1AAB901E0B0FBF4F5092DCCBF5E
:10020800572230222A4404FB150003F8012BB4FBC3
:10021800F1F4002CF0D100221A7030BC7047B0FB0A
:10022800F4F5092DCCBF372230222A4404FB1500EF
:1002380003F8012BB4FBF1F4002CF0D100221A7062
:1002480030BC70470546002AEBD1D7E72DE9F047C7
:1002580014461D46064600234FF47A722046294666
:1002680031F01AFFDFF840814B4A4C4F88FB0031D0
:100278000144C31782FB002EC3EB611188FB0128E0
:1002880087FB00278644464AC3EBEE2EC1EB011CD0
:1002980082FB0E29A0EB8C0C0744424A86F806C064
:1002A800C3EB27474FEAEE7C08EB010ACCEBA90C1D
:1002B80082FB07824FEAE1780CEB4C0CC8EB6A181A
:1002C800AEEBCC0EC8EB0818DFF8E0C086F804E007
:1002D800A1EB880171718CFB0010F917C1EBE212D8
:1002E80040F2B55101FB1272C3EBE050B2F5896FD1
:1002F8004FEA80073CDA40F2DA239A4242DCB2F550
:10030800B77FB4BF4FF0000C4FF0010C4FEA4C0917
:10031800DFF89C8009EB0C0308EBC3031FFA8CFE83
:10032800D88A09EB0C0108EBC10116310B2301E057
:1003380031F8020D824218DA013BF9D1CC4401238D
:1003480038F83C00B37007F2B2770132121ABE4493
:10035800F270A6F800E0204629464FF47A7200238E
:1003680031F09AFE3281BDE8F0870133DBB2E9E76C
:100378004FF0030EF44640F29650DFF834804FF009
:100388000609CEE74FF0020EDFF82480F44640F26B
:1003980029404FF00409C4E7C5B3A29107452EC20E
:1003A800ABAAAA2A73B06D1689888888792D03119B
:1003B800203A030803685A1C02601970704700BF8E
:1003C8002DE9F047089C2578002B804689460CBF0C
:1003D8004FF0200A4FF0300A661C35B3002A29DD99
:1003E800334601E0024698B113F8011B501E00295C
:1003F800F8D1971E60B13D46013D51464046C84779
:100408006B1C002BF8DC257827EAE770013055B122
:10041800041B29464046C847301916F8015B002DD1
:10042800F7D1BDE8F087BDE8F087002A04DC28464C
:10043800BDE8F0870020EBE7571EDCE783684268D9
:10044800D0ED037A00EB83010133934281ED040A76
:10045800836004BF0023836000EB830393ED047A79
:10046800036870EE277A9A42C0ED037A77EEC77A6E
:10047800C0ED037A0CDA013307EE103AF8EEC76ADA
:10048800B7EE007A87EEA60A036030EE070A7047D7
:1004980007EE102AB8EEC77A87EE870A704700BFC2
:1004A80090ED057A90ED004AD0ED066AD0ED014A4C
:1004B800D0ED047A90ED035AD0ED025AA4EE007AFA
:1004C800B0EE406AB0EE470AB0EE667AA6EE247A3D
:1004D80067EEC07AA0EE457AE6EE257A80ED057AD9
:1004E800C0ED067A704700BFD0ED057A90ED013A6D
:1004F800D0ED003AD0ED064A90ED024A90ED077A29
:1005080090ED035A90ED086AD0ED045AC0ED067AD2
:10051800F0EE406A27EE830AC0ED056AA3EEA60A4C
:1005280080ED087AA4EE240AA5EE470AA5EEC60ACD
:1005380080ED070A704700BFD0ED007A90ED017A90
:1005480030EE670AE7EE007AB0EE670AC0ED007A8F
:10055800704700BF704700BF0A44914214D030B4BE
:100568000139551E41F2210211F8014F082380EA92
:10057800042004044CBF82EA40004000013B80B2E2
:10058800F7D18D42F0D130BC704700BF4FF4805393
:1005980083827047012380F84530704770B404683F
:1005A800037B2268022101FA03F31A4213D042693D
:1005B8000A495C2000FB02124FF6FE765068528909
:1005C800C5680068296831402960C168D24392B281
:1005D8000A40C260636070BC704700BFD8670020E3
:1005E80030B40A4B1D7875B1094B002003EBC505E3
:1005F8001A6899885062D4682143D160083323F877
:10060800040CAB42F4D130BC704700BFB86A00207C
:10061800BC6A002010B40268047B11680223A3405E
:10062800194209D00649406800240C7001684FF649
:10063800FE742140016053605DF8044B704700BFB1
:10064800F3520020014B186824F0E8BD84260020EE
:10065800F0B5836983B0054613B11A689B88138582
:100668006869264F8389C3244FF47A734FF0060EC6
:100678006E464FF6FF71013703E0013B9BB28B4298
:100688001DD002899207F8D504734FF47A7302E0FB
:10069800A3B28B4213D00289D20703F1FF34F7D5F6
:1006A800027BD2B20EB132700136BEF1000F08D013
:1006B8000EF1FF3EFF24002FE3D03C78DBE725F066
:1006C8005FFDAB6913B11A689B8893619DF80500BB
:1006D8009DF801609DF802109DF803409DF80420E4
:1006E8009DF8063041EA062143EA002342EA042243
:1006F800012029876A87AB8703B0F0BD803A0308D9
:10070800037A022B01D000207047F0B5036983B04B
:1007180013B11A689B881385044640F2E933C06810
:1007280001E0002B59D00289013B12F0020F9BB265
:10073800F7D0BB23037340F2E93301E0002B4CD020
:100748000289013B12F0010F9BB2F7D0037BE068EE
:100758004FF0060E83896E464FF47A734FF6FF7199
:10076800FF2703E0013B9BB28B4233D002899507F8
:10077800F8D507734FF47A7302E0ABB28B4229D0F5
:100788000289D20703F1FF35F7D5027BD2B20EB149
:1007980032700136BEF1010EE8D1236913B11A682F
:1007A8009B8893619DF804009DF800609DF80110F6
:1007B8009DF802509DF803209DF8053041EA062176
:1007C80043EA002342EA05220120E182228363836F
:1007D80003B0F0BD25F0D4FCDFE725F0D1FCB6E787
:1007E8002DE9F04F90F8553087B00646002B7FD1A1
:1007F800B34B1B78002B00F01D817069038823F030
:1008080040031B041B0C038003889BB223F03803AE
:1008180043F03803038003889BB243F0400303800E
:10082800B36996F84E4013B11A689B88138540F255
:10083800E93302E0002B00F0CF850289013B12F07A
:10084800020F9BB2F6D01A23037340F2E93302E099
:10085800002B00F0C1850289013B12F0010F9BB209
:10086800F6D0037B706940F2E93302E0002B00F018
:10087800AF850289013B12F0020F9BB2F6D00473D8
:1008880040F2E93302E0002B00F0A2850289013B27
:1008980012F0010F9BB2F6D0037BB36913B11A684B
:1008A8009B8893610DF060FA04460DF05DFA84426E
:1008B800FBD07069038823F040031B041B0C0380E2
:1008C800038823F038031B041B0C038003889BB2A6
:1008D80043F040030380337C022B00F09C84B6F97C
:1008E8003A305BB2013300F0658407B0BDE8F08FA1
:1008F8001C09013C052C03F00F0300F2BA85714A6C
:1009080032F8140040FA03F2D50740F1B285012508
:1009180005FA03F3013B184031F00EFC6A4BDFF88F
:10092800C0811F5D074418EBC70400F0A28558F882
:100938003700B4F804E0038A1EEA03037FF458AFD3
:1009480000F13842920A6149E3718B5C03F01F029F
:100958005B092021022B05FA02F2A17100F08E85B5
:10096800032B00F08085012B00F08E8504A900255B
:10097800CDF810E0059523F049FDA388544AF260AC
:10098800B3FA83F2C2F11F02511C40D0D1B201F078
:10099800FC0303F1804303F5803301F00301D3F82E
:1009A80008E088004FF00F0C58F83710DFF8348152
:1009B8000CFA00F72EEA070706F10C0E48F822E0B9
:1009C8009F60D3F808C0434FDFF81CE1C1F38721CB
:1009D800814041EA0C014FF00109996009FA02FCD3
:1009E800B918CEF800C0082304A8049291F86880CA
:1009F8008DF815308DF816908DF814502EF052FCA5
:100A0800354A12F80830F02B00F35285A388B3FA60
:100A180083F3C3F11F035F1C3FF4EAAE012202FA1D
:100A280003F32E490A6813430B60254B1B78002BF0
:100A38007FF4E3AE7069038823F040031B041B0CAA
:100A4800038003889BB223F0380343F03803038004
:100A580003889BB243F040030380B36913B11A685B
:100A68009B88138540F2E93302E0002B00F0B8843C
:100A78000289013B12F0020F9BB2F6D06B2303737D
:100A880040F2E93302E0002B00F0AA840289013B1E
:100A980012F0010F9BB2F6D0037B706940F2E93384
:100AA80002E0002B00F0A7840289013B12F0020F3C
:100AB8009BB2F6D08023037340F2E93319E000BFFC
:100AC80000230020E8610308F4610308FC610308BF
:100AD8009D050008203A0308505B002000040140EF
:100AE800E4610020105B002014040140002B00F09A
:100AF80082840289013B12F0010F9BB2F6D0037B7E
:100B0800B36913B11A689B8893619623AB4CAC4DBB
:100B1800DFF8B4A2AB48DFF8B4C201964FF0100872
:100B28004FF47A779946DAF80430C3F30803002BB8
:100B380040F03084EFF31183002B40F02B842368BE
:100B4800816800BF22689342F9D12A6807FB02FE38
:100B5800AEEB010EBEFBF2FE07FB03EE0126DAF850
:100B68000430C3F30803002B40F0BB83EFF3118379
:100B7800002B40F0B6832368816800BF2268934247
:100B8800F9D1D5F800B007FB0BF2521AB2FBFBF211
:100B980007FB0323A3EB0E03B3F57A7FDFD3B9F189
:100BA8000109C0D1019EB36913B11A689B881385E6
:100BB800706940F2E93302E0002B00F018840289E2
:100BC800013B12F0020F9BB2F6D06823037340F288
:100BD800E93302E0002B00F00A840289013B12F09D
:100BE800010F9BB2F6D0037B706940F2E93302E053
:100BF800002B00F022840289013B12F0020F9BB205
:100C0800F6D00323037340F2E93302E0002B00F02F
:100C180014840289013B12F0010F9BB2F6D0037BCA
:100C2800B36913B11A689B8893619623DFF898A17A
:100C38006448DFF898C101964FF010084FF47A77AE
:100C48009946DAF80430C3F30803002B40F0858393
:100C5800EFF31183002B40F080832368816800BF85
:100C680022689342F9D12A6807FB02FEAEEB010E17
:100C7800BEFBF2FE07FB03EE0126DAF80430C3F3ED
:100C88000803002B40F04B83EFF31183002B40F057
:100C980046832368816800BF22689342F9D1D5F85A
:100CA80000B007FB0BF2521AB2FBFBF207FB03235F
:100CB800A3EB0E03B3F57A7FDFD3B9F10109C0D1F5
:100CC800019EB36913B11A689B881385706940F255
:100CD800E93302E0002B00F0AD830289013B12F0FA
:100CE800020F9BB2F6D06B23037340F2E93302E0A4
:100CF800002B00F09F830289013B12F0010F9BB289
:100D0800F6D0037B706940F2E93302E0002B00F073
:100D18009E830289013B12F0020F9BB2F6D0032397
:100D2800037340F2E93302E0002B00F0908302895C
:100D3800013B12F0010F9BB2F6D0037BB36913B1EC
:100D48001A689B8893610DF00FF804460DF00CF8B3
:100D5800001B0E28FAD9B36913B11A689B8813854A
:100D6800706940F2E93302E0002B00F073830289D6
:100D7800013B12F0020F9BB2F6D06A23037340F2D4
:100D8800E93302E0002B00F065830289013B12F091
:100D9800010F9BB2F6D0037B706940F2E93302E0A1
:100DA800002B00F05A830289013B12F0020F9BB21C
:100DB800F6D01023037340F2E9330CE024730020CB
:100DC8002873002010E000E000ED00E02073002010
:100DD800002B00F042830289013B12F0010F9BB205
:100DE800F6D0037BB36913B11A689B8893610CF042
:100DF800BBFF04460CF0B8FF001B0E28FAD9B369F4
:100E080013B11A689B881385706940F2E93302E0D0
:100E1800002B00F025830289013B12F0020F9BB2E0
:100E2800F6D06C23037340F2E93302E0002B00F0A4
:100E380017830289013B12F0010F9BB2F6D0037BA6
:100E4800706940F2E93302E0002B00F0DB8202898E
:100E5800013B12F0020F9BB2F6D00023037340F25D
:100E6800E93302E0002B00F0CD820289013B12F049
:100E7800010F9BB2F6D0037BB36913B11A689B8844
:100E880093610CF071FF04460CF06EFF001B0E28F6
:100E9800FAD9B36996F8504013B11A689B8813853C
:100EA800706940F2E93302E0002B00F0AE8202895B
:100EB800013B12F0020F9BB2F6D01923037340F2E4
:100EC800E93302E0002B00F0A0820289013B12F016
:100ED800010F9BB2F6D0037B706940F2E93302E060
:100EE800002B00F095820289013B12F0020F9BB2A1
:100EF800F6D0047340F2E93302E0002B00F0888258
:100F08000289013B12F0010F9BB2F6D0037BB36953
:100F180013B11A689B8893610CF026FF04460CF005
:100F280023FF001B0E28FAD9B36913B11A689B88EE
:100F38001385706940F2E93302E0002B00F06B8200
:100F48000289013B12F0020F9BB2F6D01B230373F8
:100F580040F2E93302E0002B00F05D820289013B98
:100F680012F0010F9BB2F6D0037B706940F2E933AF
:100F780002E0002B00F052820289013B12F0020FBE
:100F88009BB2F6D01823037340F2E93302E0002B3A
:100F980000F044820289013B12F0010F9BB2F6D0A7
:100FA800037BB36913B11A689B8893610CF0DCFE6C
:100FB80004460CF0D9FE001B0E28FAD9B36913B108
:100FC8001A689B881385706940F2E93302E0002BA8
:100FD80000F027820289013B12F0020F9BB2F6D083
:100FE8001C23037340F2E93302E0002B00F019825E
:100FF8000289013B12F0010F9BB2F6D0037B7069A6
:1010080040F2E93302E0002B00F00E820289013B36
:1010180012F0020F9BB2F6D01023037340F2E933AB
:1010280002E0002B00F000820289013B12F0010F60
:101038009BB2F6D0037BB36913B11A689B8893619E
:101048000CF092FE04460CF08FFE001B0E28FAD915
:10105800B36913B11A689B881385706940F2E93344
:1010680002E0002B00F0E3810289013B12F0020F3D
:101078009BB2F6D03723037340F2E93302E0002B2A
:1010880000F0D5810289013B12F0010F9BB2F6D026
:10109800037B706940F2E93302E0002B00F0D18154
:1010A8000289013B12F0020F9BB2F6D010230373A2
:1010B80040F2E93302E0002B00F0C3810289013BD2
:1010C80012F0010F9BB2F6D0037BB36913B11A6813
:1010D8009B8893610CF048FE04460CF045FE001B0B
:1010E8000E28FAD9B36913B11A689B8813857069F9
:1010F80040F2E93302E0002B00F0A6810289013BAF
:1011080012F0020F9BB2F6D03823037340F2E93392
:1011180002E0002B00F098810289013B12F0010FD8
:101128009BB2F6D0037B706940F2E93302E0002BF2
:1011380000F05A810289013B12F0020F9BB2F6D0EF
:101148000123037340F2E93302E0002B00F04C81E5
:101158000289013B12F0010F9BB2F6D0037BB36901
:1011680013B11A689B8893610CF0FEFD04460CF0DD
:10117800FBFD001B0E28FAD97269138823F040037F
:101188001B041B0C1380138823F038031B041B0C4F
:10119800138013889BB243F0400313800CF0E4FDE6
:1011A80004460CF0E1FD8442FBD0BA4A01231370D7
:1011B800FFF723BB96F9383001337FF496AB0A2644
:1011C80032202EF05DFA4FF4FA750CF0CDFD04468E
:1011D8000CF0CAFD001BB0F57A7FF9D3013DF4D1BC
:1011E80007202EF0D1F84FF47A750CF0BDFD0446B7
:1011F8000CF0BAFD001BB0F57A7FF9D3013DF4D1AC
:10120800013EDDD1A449A54BA548A64A0860DA608D
:1012180007B0BDE8F08FB36913B11A689B881385CE
:1012280040F2E93302E0002B00F0E9800289013B3B
:1012380012F0020F9BB2F6D0C323037340F2E933D6
:1012480002E0002B00F0DB800289013B12F0010F65
:101258009BB2F6D0037B70694FF0060E838904AD0C
:101268004FF47A734FF6FF71FF2703E0013B9BB2FF
:101278008B4233D002899407F8D507734FF47A73F9
:1012880002E0A3B28B4229D00289D20703F1FF34CE
:10129800F7D5027BD2B20DB12A700135BEF1010E2D
:1012A800E8D1B36913B11A689B8893619DF812500D
:1012B8009DF813309DF810409DF811109DF814000A
:1012C8009DF8152043EA05231BB241EA042142EAAE
:1012D800002273873187B287FFF703BB24F050FFE2
:1012E800DFE7EFF3118188F31288D0F808B00368BC
:1012F800DB0344BFCCF80060D0F808B02368DCF802
:101308000020C9B281F3118829681A4407FB01F348
:10131800A3EB0B03B3FBF1F307FB02333AE4EFF360
:10132800118188F31288D0F808B00368DB0344BF42
:10133800CCF80060D0F808B02368DCF80020C9B207
:1013480081F3118829681A4407FB01F3A3EB0B0307
:10135800B3FBF1F307FB0233AAE4EFF3118288F33E
:10136800128881680368DE0303D50123CCF80030B6
:1013780081682368DCF80060D2B282F311882A6899
:1013880006EB030E07FB02F35B1AB3FBF2F307FB52
:101398000E3E71E4EFF3118288F3128881680368C6
:1013A800DE0303D50123CCF8003081682368DCF81C
:1013B8000060D2B282F311882A6806EB030E07FB9D
:1013C80002F35B1AB3FBF2F307FB0E3EFFF7C6BB53
:1013D80024F0D6FEFFF761BA24F0D2FEFFF742BA36
:1013E80024F0CEFEFFF759BB24F0CAFEB7E624F07E
:1013F800C7FEFFF7F9BB24F0C3FEFFF781BB24F05B
:10140800BFFE28E724F0BCFE36E524F0B9FE63E50C
:1014180024F0B6FE7BE524F0B3FEA6E524F0B0FE8A
:10142800BFE524F0ADFEEAE524F0AAFE03E624F0C9
:10143800A7FE2EE624F0A4FE64E424F0A1FEFFF744
:10144800EFBB24F09DFE40E624F09AFE6BE624F004
:1014580097FE73E424F094FE9EE424F091FEC1E428
:1014680024F08EFEECE41049CB691A43CA61FFF7F9
:101478007DBA0E4BF3600123FFF7D3BA0A498B6993
:101488001A438A61FFF772BA07494B691A434A61DE
:10149800FFF76CBA00230020FC9F002000ED00E05D
:1014A800EFBEADDE0400FA05001002409D050008FD
:1014B80007EB0803F02193F878308DF80C3003A877
:1014C80003238DF80E508DF80F9002F808108DF850
:1014D8000D3022F065FFFFF799BA00BF10B490E80D
:1014E8000600047B40690223A3404B6013685DF843
:1014F800044B4FF6FE710B40136023F01FBEF8B586
:10150800174D2B78A52B28D16B78BE2B25D102221D
:1015180029464FF6FF70FFF71FF8124FAC1C2288C0
:101528004AB1A618BE4218D2052A16D92146FFF795
:1015380013F83446F3E721460222FFF70DF802229A
:10154800A118FFF709F80634074B641B1C8041F605
:101558000F53C31A58425841F8BD0020F8BD00BFC8
:1015680000F0030800000408943200202DE9F04F31
:10157800DFF864914F4F8BB00326A7EB09071822B9
:10158800002104A832F0D9F94B4BCDF810900597FB
:101598001A69120604D5494A5A6002F188325A601B
:1015A80001228DF824203422DA60454B454C1B88F3
:1015B800ADF800300222694604A824F0ADFE0222EC
:1015C80069464FF6FF70FEF7C7FFDFF810A18046A7
:1015D8004FF0000B544536D30AAC002524F8245D9F
:1015E8000222214604A824F097FE02222146404602
:1015F800FEF7B2FF40BAC043ADF80800022202A9C4
:1016080004A824F089FE079860B106ABC0F1040273
:101618002946184432F091F9069904A824F022FECC
:10162800079508909DF82430089A23B122490B6940
:1016380043F080030B61013E2DD0002A9FD1FFF7B4
:101648005EFF50B332E065888DF80DB0C5F30B0529
:10165800AB1DADF808302388C3F30B02ADF80A20A0
:101668001B0B062202A904A88DF80C3024F054FEA6
:10167800062202A94046FEF76FFF616880462A46A7
:1016880004A824F049FE616840462A46FEF764FF34
:10169800143480469EE7002AD1D005202BF0ECFFB9
:1016A800094B0A4A1A600A4B0A4ADA600BB0BDE8CD
:1016B800F08F00BF000004080020024023016745A6
:1016C8009F3A0308A0A00308FC9F0020EFBEADDEF0
:1016D80000ED00E00400FA0500F0030814A5030873
:1016E8000378202B024600F10100F9D0092BF7D02E
:1016F8002D2B2CD02B2B03BF5378B7EE000A0246B4
:10170800B7EE000AA3F13001C8B209289FED467A66
:1017180010D8F2EE046A07EE901AF8EEE77A12F89B
:10172800013FE7EE267AA3F13001C8B20928B0EEEE
:10173800677AF0D92E2B4CD003F0DF03452B0BD062
:10174800F7EE007A67EE276A20EE260A704753788C
:10175800BFEE000A0246D5E710B451782D2959D0BA
:101768002B290ABF9178501C901C0024A1F130034A
:10177800092B53D8002303EB830301EB430310F831
:10178800011FA1F13002092AA3F13003F3D9B3F5FF
:101798009A7F28BF4FF49A73072B42D9DFED236A4B
:1017A8001A46F7EE007A083A072A67EEA67AFAD8B8
:1017B80003F007032BB1F2EE046A013B67EEA67A49
:1017C800FBD124B3C7EE276A5DF8044B20EE260A46
:1017D80070475378A3F13001C8B2092802F1010219
:1017E800AAD8F2EE046AF0EE665A07EE901AF8EEFE
:1017F800E77A12F8013F87EEA66AA3F13001C8B272
:10180800092866EEA56A37EE067AEED994E767EE00
:10181800276AD9E7901C91780124A7E7F7EE007AA8
:10182800CFE7F7EE007AC5E70000000020BCBE4C09
:10183800B5EEC00ADFED317AF1EE10FACCBF30EE2A
:10184800270A30EE670ADFED2E7A20EE270A30B538
:10185800FDEEC07A87B017EE904A054684EAE47038
:10186800002303A9A0EBE4700193009302932FF0E7
:10187800ADF8002CACBF20232D2303A88DF8003031
:101888002FF040FF012803A924D002282DD00328D7
:1018980005BF3023684668468DF8013032F055F8A8
:1018A80068462FF02FFF0338C4B2224669462846FF
:1018B80032F082F800232B5528462FF023FF2E22E2
:1018C800431C2A540DEB0401E81832F05BF8284653
:1018D80007B030BD302368468DF801308DF80230EE
:1018E8008DF8033032F031F8DAE7302368468DF8A6
:1018F80001308DF8023032F028F8D1E76F12033A40
:1019080000007A442DE9F041064615460846B6FB24
:10191800F2F43CB905FB1464124B1B5D00F8013B63
:10192800BDE8F081B4FBF2F767B90E4B05FB17472A
:1019380005FB1464DA5D00F8012B1B5D00F8013B20
:10194800BDE8F081B7FBF2F8B8F1000F02D04046CD
:10195800FFF7D8FF05FB1878024B13F8082000F8AA
:10196800012BE3E72C680308104B2DE93048D3E935
:10197800004554EA05020BD10346012200201871E4
:10198800587198719A70DA7018801881BDE830889B
:10199800074B1A6814EB020B45F1000C5A466346D4
:1019A800FEF754FC0120BDE8308800BF4823002022
:1019B80024730020F0B402888578154FC378047921
:1019C8004179A2F2B27202F0030606EB4606013D27
:1019D80005EB8605013B37F815608579008940F2EB
:1019E800B557920807FB0232931903EB430304EB44
:1019F800C303C3EB031301EB8303C3EB031305EB2F
:101A0800830300214FF47A72C2FB0301F0BC7047D4
:101A1800203A0308FAB170B48E18044603E0101A8D
:101A280014D1B14214D014F8012BA2F14103192B9F
:101A380011F8013BA3F1410598BF2032192D03F19C
:101A48002000ECD9D01A01D1002BEAD170BC704724
:101A5800002070BC70471046704700BF4FF0FF323F
:101A6800FFF7D8BFA0F16103192B98BF2038704742
:101A7800A0F14103192B98BF20307047202805D0CA
:101A8800093804288CBF00200120704701207047C6
:101A9800613819288CBF0020012070474138192867
:101AA8008CBF002001207047303809288CBF0020E7
:101AB80001207047A0F13003092B07D920F020003E
:101AC800413819288CBF0020012070470120704739
:101AD80030B402681146531C036011F8024B0160D0
:101AE800D31C517803609378151D05601B0443EAE5
:101AF8000123D078234343EA006030BC704700BF1D
:101B08000368591C1A46016012F8021B02605878D3
:101B180041EA0020704700BF03685A1C0260187829
:101B2800704700BF38B504460068154630F072FDAE
:101B380022682A44226038BD036810B40A0A5C1C73
:101B480004601A7003685A1C026019705DF8044B2F
:101B5800704700BF03685A1C026010B4197003680C
:101B68000A0A5C1C04601A7003680A0C5C1C046096
:101B78001A700368090E5A1C026019705DF8044B4C
:101B8800704700BF03685A1C026019700368090A8D
:101B98005A1C0260197070472DE9F047002488B07C
:101BA80080460F461E46A14605AD531C0393117887
:101BB80039B3252933D1931CCDF81090039350786D
:101BC80030284ED04FF0000AA0F13003DBB2092BC9
:101BD80042D96C2819D0642800F0938024D825288D
:101BE8001CD063D9582876D063281BD13178404659
:101BF800B847039A531C039311780436013400291B
:101C0800D7D1204608B0BDE8F087039B5A1C039241
:101C18001B78642B7CD02AD8252B54D1252140460B
:101C28000134B847039AC0E7732833D044D97528DC
:101C38004FD106F1040E30682B4600220A21764661
:101C4800FEF7CCFA049A0095534639464046FEF70B
:101C5800B7FB039A0444A8E704AA03A92CF0C4FF1D
:101C6800B7E7D31C039390784FF0010AACE7732BC6
:101C780010D05BD9752B3AD0782B96D1A3F15802A6
:101C8800B2FA82F2306852092B4610210436FEF768
:101C9800A5FAD7E73368049A0093394600234046EB
:101CA800FEF78EFB04360444039A7EE70028B9D178
:101CB800204608B0BDE8F0876E28B3D1039A336890
:101CC80004361C6071E72AD9582BD7D0632B8DD0E6
:101CD8006BE77828A6D1A0F15802B2FA82F23068F0
:101CE80052092B461021FEF779FA0436AAE706F1C5
:101CF800040E30682B4600220A217646FEF76EFA5B
:101D0800A0E7331D306829461E46FEF739FA99E7E1
:101D1800331D306829461E46FEF732FA92E7002B3B
:101D28007FF443AF204608B0BDE8F0876E2BC6D0DD
:101D38003BE700BF0EB400B584B005AB019053F883
:101D4800042B0649039301A8FFF726FF019B0022F5
:101D58001A7004B05DF804EB03B07047BD030008C7
:101D68002DE9F04707468CB01E469246002A6AD1F4
:101D7800154614460A8840F2B1739A423AD98B78CC
:101D8800581E0B2836D891F803E00EF1FF301E28B4
:101D980030D891F804C0BCF1170F2BD891F80590F2
:101DA800B9F13B0F26D888793B2823D8B1F80880A9
:101DB800B8F57A7F1ED24FF00108002E34D1098978
:101DC8000491002CB4BF2D212B21002CB8BF6442F4
:101DD800039005910795CDF80890CDF804C0CDF88B
:101DE80000E0384606942F49FFF7A4FF40460CB0A0
:101DF800BDE8F0870023012118468E46ADF824304F
:101E08008DF828308DF829308DF82A30ADF82C302F
:101E180099469C461A4698468DF826108DF8271044
:101E28000B4609A9002ECAD00390CDF80890CDF82A
:101E380004C0CDF800E038461B49FFF77BFF404659
:101E48000CB0BDE8F087194C84FB0234A318D417F2
:101E5800C4EB6314C4EB0415A2EB85052DB2002D69
:101E68000846B8BF6D42FFF7A5FD4FF47A7200230C
:101E78008046894630F010F93C230AFB030A4FF4E8
:101E88007A7200234046494630F006F94FF47A71D9
:101E980092B20023C1FB0A2309A8FEF7D7F924B29E
:101EA80009A967E77468030854680308898888885B
:101EB8000FB430B583B006AB0A490B4853F8042B6E
:101EC800096800680193FFF767FE084C054620681B
:101ED80023F094F90028FAD0284603B0BDE8304032
:101EE80004B07047F0310020F4310020842600202F
:101EF800DFED2B7AB4EEE70AF1EE10FA4ADDDFEDFA
:101F0800296A9FED297A01E0B0EE670AB4EEC70AA4
:101F1800F1EE10FA70EE667AF6DC9FED247AF4EEB4
:101F2800C77AF1EE10FA38D5DFED1E6A9FED207AF8
:101F380001E0F0EE407AF4EEC77AF1EE10FA37EEEF
:101F4800A60AF6D4DFED1B7AB4EEE70AF1EE10FA32
:101F580014DDDFED137A37EEC00A60EE006A9FEDFC
:101F6800166A9FED167ADFED167AA6EE867A20EECF
:101F7800266AE6EE877AA6EE270A7047DFED117A21
:101F8800B4EEE70AF1EE10FA44BFDFED087A37EE57
:101F9800C00AE2E7F0EE407ABFE7B0EE670AD1E7A1
:101FA800DB0F4940DB0FC940E4CB1641DB0F49C0CA
:101FB800E4CB16C1DB0FC93F92E741B99730083C23
:101FC80015A82ABEDB0FC9BF09B909E0194690FB5D
:101FD800F1F301FB13030846002BF7D108467047BD
:101FE8000146FBE707EE901AF8EE677A9FED837AD1
:101FF80027EE800A20EE070AFDEEC07A17EE903A27
:102008002033402B00F28C80DFED7D7AB4EEE70AB6
:10201800F1EE10FA40F3E880B0EE407A9FED796A6D
:10202800DFED796A01E0B0EE677AB4EEE67AF1EEB8
:1020380010FA77EE467AF6DC9FED747AF4EEC77AFA
:10204800F1EE10FA40F1CD809FED6E6ADFED706A17
:1020580001E0F0EE477AF4EEE67AF1EE10FA37EEA8
:10206800867AF6D4DFED6B7AB4EEE77AF1EE10FA01
:1020780051DCDFED697AB4EEE77AF1EE10FA44BF8D
:10208800DFED627A37EEC77A27EE076ADFED635A2B
:10209800DFED637ADFED636A9FED635AE6EE257A3A
:1020A80067EE065AE6EE276AF7EE007AA5EEA67AFC
:1020B800F0EE675AE7EE055AE7EE457A87EEA55A3D
:1020C800DFED547A30EE277AFDEEC76A16EE903AC5
:1020D8002033402B29D99FED557AF6EE006AB7EEEA
:1020E800006AF7EE004AC4EEA57A002383614361D3
:1020F8000362C36180ED045A67EEA66A27EE866A1A
:1021080027EE877AC0ED006AC0ED026A80ED016AA9
:1021180080ED037A7047DFED3A7A37EEC77AB3E796
:10212800B7EE005AF0EE455ACAE7B4EEE70AF1EE08
:1021380010FA5FDD9FED336ADFED336A01E0B0EE40
:10214800677AB4EEE67AF1EE10FA77EE467AF6DCC4
:102158009FED2E7AF4EEC77AF1EE10FA47D59FED8F
:10216800296ADFED2B6A01E0F0EE477AF4EEE67AB1
:10217800F1EE10FA37EE867AF6D4DFED267AB4EE71
:10218800E77AF1EE10FA27DCDFED237AB4EEE77A8E
:10219800F1EE10FA44BFDFED1D7A37EEC77A27EE6D
:1021A800076ADFED1E4ADFED1E6ADFED1E7AE6EEF6
:1021B800246A67EE064AE6EE267AB7EE006AA4EECF
:1021C800A77AF6EE006A36EE476AF8EE007A27EE4E
:1021D800277A66EE266A84E7DFED097A37EEC77A52
:1021E800DDE7B0EE677A3DE7F0EE407A24E7B0EE3F
:1021F800677AC2E7F0EE477AAAE700BF27D4D2365B
:10220800DB0F4940DB0FC940E4CB1641DB0F49C067
:10221800E4CB16C1DB0FC93FDB0FC9BF92E741B959
:102228009730083C15A82ABEF304353F000000800B
:1022380070B406688E4217D90139751E002311F84B
:10224800014F0822634013F0800F4FEA430318BF81
:1022580083F0D503013ADBB2F5D18D42EFD1721C80
:102268000260337070BC70470023F8E710B44C0963
:10227800012250F8243001F01F0102FA01F10B434A
:1022880040F824305DF8044B704700BF4B0901F05B
:102298001F0150F82320012303FA01F1114214BF52
:1022A80018460020704700BF074A084B10781B7873
:1022B800074A834296BFC31AC3F1800300201268FD
:1022C80018441044704700BFA870002025700020F3
:1022D8008C5D0020064A074B10781B7883428ABF22
:1022E800C3F18003C01AC018C0F17F00704700BF57
:1022F800A870002025700020F8B584894FF6FF7675
:102308004FF47A742BB311B30F78013101E0B44262
:1023180017D00589013CAD07A4B2F8D507734FF46F
:102328007A7402E0BCB2B4420BD00589ED0704F11F
:10233800FF37F7D5057BEDB20AB115700132013BC5
:10234800E0E723F01DFF003018BF0120F8BDFF278C
:10235800DFE70120F8BD00BF30B5134C237883B008
:102368001BB90120237003B030BD1049052200239A
:102378000D688DF804208DF8053000BFA86823F09B
:102388007FFD6A4601A902236868FFF7B5FFA868C0
:1023980023F07CFD00BF9DF8013003F0010383F0BA
:1023A8000100237003B030BDF1700020AC70002034
:1023B80070B5064C0646256803E023685B1BB342EC
:1023C80003D8FFF7C9FF0028F7D070BD2473002099
:1023D800F0B51F4C83B0277800234FF0030E00930D
:1023E8000E4615468DF804308DF800E06FB3030EE5
:1023F8008DF801300DF10203010C020A9870197072
:1024080006205A70FFF7D4FFE8B100BF114F3B68B0
:10241800986823F035FD23783A68002B14BF05230C
:102428000423694650680022FFF766FF3B6832467E
:10243800002158682B46FFF75FFF3B68986823F038
:1024480025FD00BF284603B0F0BD0DF10103D3E719
:10245800F0700020AC70002008B540F2E93300E0CD
:102468009BB10289013B12F0020F9BB2F8D00173B5
:1024780040F2E93300E043B10289013B12F0010F59
:102488009BB2F8D0007BC0B208BD23F079FEC0B281
:1024980008BD00BF38B504460D4600BF806823F06C
:1024A800EFFC29466068FFF7D7FFA06823F0EEFC31
:1024B80000BF38BD2DE9F04F89B0B2F1000A029093
:1024C8000491039340F3C5800B46002201EB8A0177
:1024D80053F8040B8B420244FAD1039B0592002B5C
:1024E80000F0AF80059B002B7CD05E4B059A1B68E3
:1024F800DFF8889100920099DAB25118B1F5807F1F
:102508008CBFC2F58072009A0192574A92689A422B
:1025180040F28280554A1178002206928DF81C20DC
:1025280002228DF81820002960D01A0E8DF8192083
:102538000DF11A021C0C190A9370147051700620C0
:10254800FFF736FF0621D9F80000FFF7A3FF484A36
:102558000123137000BFD9F80030986823F090FC6D
:10256800424BD9F800201B785068002B06A90CBFF5
:10257800042305230022FFF7BFFE0024049D029ECA
:10258800019FA34629684FEA840800220B460134BC
:1025980071B1B9422DD2D9F8000031684068FFF70F
:1025A800ABFE2A68336813443360BF1AC5F800B01D
:1025B800A24505F1040506F10406E3D1D9F8003077
:1025C800986823F063FC00BF264B019900981B68AC
:1025D800421A0092234A0B441360039A4AB3009AA2
:1025E800002A88D1059809B0BDE8F08F0DF11902CD
:1025F800A0E7029CD9F8003054F808105868002267
:102608003B46FFF779FE54F808202B683A44DF1B55
:1026180044F808202F60D1E70598009C1549164A10
:10262800001B0590059800230B70137009B0BDE8D6
:10263800F08F059B009A9B1A0593059809B0BDE891
:10264800F08FFFF789FE00287FF44CAF039B0593BA
:10265800C8E7039C1CB9FFF77FFE0594C2E7002377
:102668000593BFE78C5D0020C81F0020F070002094
:10267800F1700020A870002025700020AC700020A8
:1026880070B5104D104E2B7831788B4284B016D02F
:102698000E4A03921A4402928CBF0C46CA1A04A925
:1026A8008CBFC3F180020024012341F8102D02A839
:1026B80002220194FFF7FEFE002333702B7004B052
:1026C80070BD00BF25700020A87000202870002071
:1026D800F0B5124B9D6885B00DB905B0F0BDED0A97
:1026E80014D0002704AE7C196410E0021022694659
:1026F800FFF76EFE0F2809DD6B4653F8042B0132F5
:102708000AD1B342F9D12546AF42ECDBFFF7B8FF57
:10271800034BED021D60E0E7671CF5E7C81F0020CA
:102728008C5D002070B5194C194D23782978994291
:1027380084B027D0174A03921A44029234BF0E4637
:10274800CA1A04A934BFC3F180020026002341F845
:10275800102D02A802220196FFF7ACFE2378184438
:10276800C0B203062B7848BF80F0800083422070F7
:1027780002D0002004B070BD002301202B7023700C
:1027880004B070BD012004B070BD00BF25700020EA
:10279800A87000202870002010B50C4C45F20820C5
:1027A800FFF706FE20680621FFF774FE084B206835
:1027B8000122C7211A70FFF76DFE06480649074A2D
:1027C800002303700B70136010BD00BFAC700020B5
:1027D800F1700020A8700020257000208C5D00207A
:1027E800028822F040021204120C0280028822F0B1
:1027F80038031B041B0C59B141F48071002991FA6C
:10280800A1F2B2FA82F108BF4FF0FF310139C900D5
:102818000B439BB2038003889BB243F040030380C1
:10282800704700BF2DE9F84FDFF8D8B03148DFF81E
:10283800D8A0DFF8D880012308218BF80030FFF7F3
:10284800CFFF2D4B186823F01BFB05212948FFF704
:1028580003FE00212748FFF7FFFD06212548FFF763
:10286800FBFD00212348FFF7F7FD9AF800402148B7
:10287800042144F00104FFF7EFFD21461D48FFF74E
:10288800EBFDB8F80030B3B11C4D1D4F194E0024B4
:1028980095F8019007213046FFF7DEFD494630469E
:1028A800FFF7DAFDB8F8003015F8012F07F8012F07
:1028B80001349C42ECDB07210E48FFF7CDFDFF21D8
:1028C8000C48FFF7C9FD9AF800400A480421FFF7B1
:1028D800C3FD21460748FFF7BFFD074B186823F0E3
:1028E800D5FA02210348FFF77BFF00238BF800305D
:1028F800BDE8F88F0030014030720020B346002058
:10290800D3480020BD4800200C4D00205A0100206B
:10291800F8B5114D114FC1F1030646EA80060821AA
:102928002846FFF75DFF386823F0AAFAF6B21024AC
:10293800E1B22846FFF790FD013431462846FFF7FB
:102948008BFD202CF4D1386823F0A0FA022102482C
:10295800BDE8F84044E700BF003001403072002075
:10296800F8B5444C44480821FFF73AFF206823F0A3
:1029780087FA424B1B78012B6DD058D3022B4ED1CE
:102988003F4D08232B704FF4C3733E4E3E4F3380A8
:1029980002210020FFF7BCFF08213748FFF720FF7E
:1029A800206823F06DFA2D7833480021FFF754FD95
:1029B80029463148FFF750FD344B2F481D78022136
:1029C800FFF74AFD29462C48FFF746FD304B2A48B9
:1029D8001D780321FFF740FD29462748FFF73CFDF6
:1029E8002C4B25481D7804210D43FFF735FD29465A
:1029F8002148FFF731FD206823F048FA02211E48DC
:102A0800FFF7EEFE32882448002130F096FF3B782D
:102A180063B1224B1B7823B300233B70F8BD184DDC
:102A28002B785B06AFD54FF4F073AEE7F8BDA02165
:102A38001148134DFFF710FD00210F48FFF70CFD5B
:102A480000F00603022B03D000F0050001280DD08A
:102A580008232B7097E70A4D48232B704FF4F07327
:102A680093E7FFF7DFFE00233B70F8BD48232B7088
:102A7800D9E700BF307200200030014034720020D6
:102A88005C0100205A010020000000203B72002059
:102A98003C7200200C4D0020D4480020BD48002086
:102AA800F0B55B4B5B4A97B01968914200AF00F0F4
:102AB800A3805949594A00234FF47000C1F888008F
:102AC8003B607B60136843F48033136003E03B682A
:102AD800B3F5A04F09D0136803F400337B603B685B
:102AE80001333B607B68002BF1D04C4B1B6813F41F
:102AF800003318BF01237B607B68012B52D0464C02
:102B0800464B474AE260474A596A11605A6A42F09E
:102B180080725A625A6942F4FC025A610025032203
:102B280007F10801012341F6FF764FF09040FD6060
:102B3800BE603A73BB7321F069FC4FF6FF7307F16F
:102B480008013948BB6021F061FC07F108013748EA
:102B5800374E21F05BFC07F10801364821F056FC9E
:102B680007F10801344821F051FC07F10801334806
:102B780021F04CFC07F1080021F0A2FCBB683049A9
:102B8800304AA1FB031330499B0CF0204FF0070E8D
:102B98005C370B60566084F823009560C2F800E04B
:102BA800BD46F0BD294A1D4B122111605A685A6072
:102BB8005A685A605A6842F480625A605A6822F425
:102BC8007C125A605A6842F4E8125A601A6842F055
:102BD80080721A601A689201FCD559680F4A21F070
:102BE80003015960596841F002015960536803F0C4
:102BF8000C03082BFAD182E700221A6062B6144B44
:102C08001B6883F30888134B1B689847FEE700BFCF
:102C1800FC9F0020EFBEADDE00ED00E0001002409A
:102C28000005FA05807300200004004800080048E9
:102C38003F190100000C004800100048001400482B
:102C480083DE1B4310E000E02873002000200240D0
:102C580000D8FF1F04D8FF1F70B50F4C0F4DC0EBF5
:102C6800C00004EB8004686926693043686182B05B
:102C78009209667BA1600025012101A863618DF896
:102C880004608DF805208DF806508DF8071021F0A6
:102C980087FB02B070BD00BFD81F002000100240A3
:102CA800074BC0EBC00030B403EB8000054C05694E
:102CB80063692B4363610176427630BC704700BF7D
:102CC800D81F0020001002402DE9F04F5E4C54F848
:102CD800204083B0002C71D0A66D984691465B4B7E
:102CE80072682265A160236004F15E014FF480736D
:102CF80004F5AF726161A261E36023610746307E2B
:102D08002CF078F8F068A8B1514B00215A6890422D
:102D180003F11C0300F0928001310C29F6D1002048
:102D28007A1CD2B20C21FFF7BBFF236DF2686263F5
:102D38002433E364B068D8B1454B00215A68904207
:102D480003F11C0378D001310C29F7D100257A1C36
:102D5800D2B20B212846FFF7A3FF2346F27E3D4956
:102D68002846FFF779FF236DB268A2632833A3646E
:102D780094F85D0022F032FC054694F85C0022F0DD
:102D88002DFC18F0080F824696F819B01AD0CDB16C
:102D980018F0110F4FF00B0307F1010714BF4E2174
:102DA8003E21EF715A46AB71284622F0DBFC18F041
:102DB800010F45D0636B5BB3A36B4BB3204603B0E5
:102DC800BDE8F08F18F0010F0CBF4FF02E084FF040
:102DD8004E0819F0020F09D045B10B227B1CAA71CD
:102DE800EB7128465A46414622F0BCFC19F0010F07
:102DF800E0D0BAF1000FDDD001370C238AF8077054
:102E08005A4641468AF80630504622F0ABFCD1E7D4
:102E1800337FB27E8DF804209B090021012201A88E
:102E28008DF805308DF806108DF8072021F0B8FAD6
:102E3800204603B0BDE8F08FCDB288E7C8B26FE78F
:102E4800284623F01DF8B5E7FC310020A43A030812
:102E5800D81F0020E514000800B97047F0B595B0F8
:102E680005462CF0D1F96E4EC368026832600446FC
:102E7800002B00F0C380284622F0B0FB694B586055
:102E880018B1292200238271C371227A664D2E213E
:102E980022F068FC30680AF0F7FD2BF0ABFF3068D1
:102EA800624A038823F001031B041B0C038014A946
:102EB8001E232B8001270F230025138021F84C7D2A
:102EC8002D230293ADF80C50ADF80650ADF80E5016
:102ED8002CF048F9E379ADF8145060229907ADF861
:102EE80016500695ADF81C50ADF81E50ADF82050A0
:102EF800ADF82250049200F1838013F0010F14BF43
:102F0800022200224FF48073ADF81470ADF81C2033
:102F1800ADF82030002304AA6179306806930AF0DE
:102F280013FA306861792CF0FDF83068436C43F48B
:102F38000043436403889BB243F080030380E37932
:102F48009B0768D56179026A04238B4022EA030251
:102F58000262026A134303623268354F13889BB2D8
:102F680043F001031380207C00222921FFF798FEFB
:102F78003049207C00236022FFF76EFEE06838604D
:102F880021F07AF9386803684FF6FE72134003603F
:102F980021F072F909A821F041F9336862792649CC
:102FA80038680A913433134409938022102300258A
:102FB80009A940F22A3E0E920B934FF400724FF487
:102FC80000530D951095139511950F921293ADF826
:102FD80030E021F031F9627933680C2A98BF17493B
:102FE800D86898BF31F812503A6815490543DD6032
:102FF8001368012043F002031360087015B0F0BD98
:1030080013F0010F14BF08222A460423ADF81E202E
:10301800ADF816307EE70122617921F03DF89BE793
:10302800EC5F002000230020E25F0020E05F00202A
:10303800E85F00201D0600084C53002014620308B6
:10304800E45F00200348D0F83C3113B100F59A70D2
:1030580018477047D81F00200348D0F8203113B113
:1030680000F58C7018477047D81F00200348D0F827
:1030780004310BB1FC301847704700BFD81F00203F
:103088000348D0F8E8300BB1E0301847704700BF6C
:10309800D81F00200348D0F8CC300BB1C4301847F3
:1030A800704700BFD81F00200348D0F8B0300BB1DC
:1030B800A8301847704700BFD81F00200348D0F831
:1030C80094300BB18C301847704700BFD81F0020D0
:1030D8000248836F0BB1703018477047D81F002023
:1030E8000248C36D0BB1543018477047D81F0020F1
:1030F8000248036C0BB1383018477047D81F0020BE
:103108000248436A0BB11C3018477047D81F00208B
:103118000248836803B11847704700BFD81F0020D2
:10312800F8B5574C0601A7190546387A2BF062FE08
:103138003B7A03F01F015B090122022B02FA01F21C
:1031480078D0032B71D0012B67D0A31901351879DA
:1031580022F044FAEDB2074610B11223C57183710B
:10316800A319587922F03AFA10B11323C571837163
:10317800A319987922F032FA10B11423C57183711A
:10318800A5190E21EA79384622F0ECFA687922F07E
:1031980025FAEA790E2122F0E5FAA87922F01EFA3A
:1031A800EA790E2122F0DEFAA359364A934251D029
:1031B800354A934259D0354A934240D03444227B11
:1031C800002A2FD1012002249A8822F48052120466
:1031D800120C9A80998889B241F4805199801A8892
:1031E80002F4415242F44572024322431A809A88FB
:1031F80022F470621204120C42F4E0629A809A8BF4
:1032080022F400621204120C07219A8319821A8888
:1032180092B242F040021A80F8BD1D4B996A0A43E7
:103228009A6292E700200446CEE7194B19690A43CF
:103238001A618AE7164BD9680A43DA6085E702F50E
:10324800EA32116941F400411161116921F4004128
:103258001161B3E702F56042D16841F48051D16051
:10326800D16821F48051D160A8E702F5EC321169E8
:1032780041F480411161116921F4804111619DE798
:10328800C07000200030014000380040003C004081
:10329800001002401749184B184A194810B4D1F8C1
:1032A800884044F47004C1F888401C6844F0010464
:1032B8001C605C6822405A601A6822F0847222F40A
:1032C80080321A601A6822F480221A605A6822F43E
:1032D800FE025A60DA6A22F00F02DA621A6B0024E0
:1032E80010404FF0006218639C608A605DF8044BE0
:1032F800704700BF00ED00E0001002400CC07FF8EE
:10330800CCFC00FF2DE9F04F9BB0B0F908500D81BF
:10331800EDB2442D00AF0C46904600F0D38206462D
:1033280043D9812D00F00C8200F29980542D00F0D1
:10333800CE8040F2F1816E2D00F09282802D40F017
:103348002481C34B93F800A00AF1020A1AF0FF0A7D
:1033580000F09980BF4BDFF83483BF4EDFF830B3FD
:103368009A4403F101090A2516E0322D00F09783EB
:10337800A5F13C00C0B2132840F2978300232268CD
:10338800511C216015702268CA4502F101012160B3
:10339800137078D019F8015B0A2DE6D1BBF800301C
:1033A800FF2BA8BFFF23DBB2E9E7052D00F07882E9
:1033B80020D8022D00F0838040F29B81032D00F07D
:1033C8004682042D40F0E1802A46A4492046FEF7B3
:1033D800A9FB00212046FEF7D5FB22680221531CD9
:1033E8000125236028462B466C3711706381BD4642
:1033F800BDE8F08F242D60D040F20C81282D00F01C
:10340800E881382D40F0C1800A68954B0125511C90
:1034180021601570226805215019206011702268FA
:103428000A2150192060117022680021501920606B
:103438001170226819785019206011702268597823
:1034480050192060117022689978531923602B460F
:10345800117028466C376381BD46BDE8F08FA02DFA
:1034680019D040F21B81B82D00F0EF81FE2D40F0FD
:103478008C807C4D05F1080635F8021B2046FEF7C6
:1034880081FBAE42F8D101252B4628466C37638173
:10349800BD46BDE8F08F744B08461968FEF75AFB25
:1034A800724B20461968FEF755FB714B1968204688
:1034B8000125FEF74FFB2B46E7E76E4BF6E70422A4
:1034C8006D4920460125FEF72DFB2B46C1E70B6809
:1034D8006A4ADFF8C081581C1121206019702368DE
:1034E8001278591C21601A70236898F85520591CC5
:1034F80021601A70236898F85420591C21601A70AA
:10350800B8F850102046FEF73DFB23680022591CEE
:1035180021601A7023682822591C21601A70B8F893
:1035280052102046FEF72EFBA8F1020508F14E06C0
:1035380035F8021F2046FEF725FBB542F8D1226870
:103548004F4B0D21501C20605D181170226813F834
:10355800011F501C9D4220601170F7D12368022280
:10356800591C21601A70B8F856102046FEF70AFB5D
:10357800B8F858102046FEF705FB0125B8F85A1090
:103588002046FEF7FFFA2B4663E7214628460DF052
:1035980027F8034600287FF476AF742D00F0C28028
:1035A800772D0DD13268716891421EBF531C33606C
:1035B8001178344A08BF1946204615F039F962E7F0
:1035C800F52D01F07383472D00F0A881392D32685D
:1035D80000F01D8300F29F82212D01F02083292D08
:1035E80040F05D83531C336013780A2B01F0148478
:1035F800502B41F078813046FEF782FADFF8988048
:10360800A8F800003046FEF77BFA0125A8F802006A
:103618002B461EE7202DB8D10B681B4D591C6A7824
:1036280021601A7023682A78591C21601A7023684F
:10363800AA78591C21601A7029892046FEF7A2FA37
:1036480023686A79591C21601A702268A979C6E62C
:10365800C94D0020CC3A0308E4290020BE7200209E
:103668004B5E0020EC4D0020ACF7FF1FB0F7FF1FAA
:10367800B4F7FF1FB85F0020A46803083872002061
:103688002D6D0020F9760108C05000206766666637
:103698000C2A0020D06C0020CC290020822D7FF439
:1036A80074AF0B688B4A8C4D11788C4A581C20607B
:1036B800197011892046FEF765FA894B22681B8824
:1036C800FF2B02F10101A8BFFF2321601370A96835
:1036D80081F3100189B22046FEF754FA296801F3F4
:1036E8000F0189B22046FEF74DFA7E4B2268197801
:1036F80075E6012D7FF449AF0B680022591C216043
:103708001A7023685A1C22601D7022682521531CD8
:1037180023602B4611709CE6522D7FF436AF226849
:1037280000215CE63268716891421EBF531C336009
:1037380011786D4A08BF1946204615F079F8A2E6B7
:103748006A4B1E78033616F0FF063FF49CAE684BB2
:10375800DFF8C0811E4403F1010A4FF00A0920E096
:10376800B9F1500F00F09981B9F1320F00F0B28130
:10377800A9F13C00C0B2132840F2AF8100252946C8
:1037880023685A1C2260204683F80090FEF7FAF955
:1037980029462046FEF7F6F956453FF474AE1AF866
:1037A800019BB9F10A0FDBD1524B9D68196805EBF3
:1037B80085054FF6FF736D009D42A8BF1D469942CF
:1037C800A8BF194625EAE57521EAE171ADB289B2CB
:1037D800D6E70B68DFF84091474E591C022221605A
:1037E8001A7023684FF006085A1C226083F800807C
:1037F80023680A22591C21601A70236801255A1966
:1038080022601D70B9F800102046FEF7BBF9B9F820
:1038180002102046FEF7B6F923685A19226083F889
:10382800008023685022591921601A7023680022E9
:10383800591921601A7031882046FEF7A3F971885A
:103848002046FEF79FF92B4603E62C4B2EE60B6825
:103858005A1C0A601D700B685A1C0A601D705EE7CE
:103868001F4B0A681B881C4DFF2BA8BFFF23511C48
:1038780021601370A96881F3100189B22046FEF710
:1038880081F91F4B20461988FEF77CF9296801F356
:103898000F0189B220460125FEF774F92B46D8E5B9
:1038A8000B2218492046FEF73DF908221649204602
:1038B800FEF738F90125072214492046FEF732F9A8
:1038C8002B46C6E5002A3FF4DEAD114B13600125F7
:1038D8002B46BEE5024F0020D0500020C0500020EB
:1038E800EC4E0020806D0020A9770108C94D00200A
:1038F800DC3A030898290020CC2900204434002011
:10390800446D0020AC680308B8680308C46803085D
:10391800BD050108DC290020505D0020726835686B
:103928007B623046551BFEF7D3F8052D38627B6A5B
:1039380001F25A828026B346012594E80600521AFD
:10394800103AB242B8BF1FFA82FBBA4A396A926883
:103958003A61521A9345396A7B622046FA6088BFF9
:103968001FFA82FBFEF7F6F87B6A002B01F01A8239
:10397800002D41F074812368C7F800D05D71C0B094
:103988000533C7F804D0FB61BBF1000F01F02E83AB
:103998003B6A3A69934281F02E833E6A7D62AA4669
:1039A800A846BC608025FB68A3EB0808A14BB8F5C6
:1039B800807F9B6828BF4FF4807808EB06029A4204
:1039C80088BFA3EB0608FEF75BFE7C6842462146EB
:1039D8003046FEF7FDFCF969B86104EB000C0B7882
:1039E8007B6164452ED2DFF860920CF1FF3C04F154
:1039F800FF3E1EF8013F09EB830219F82340568861
:103A0800ECB100234FF4004204F1FF3832424FEA90
:103A1800520202D00878284308706D0806D10AF1CE
:103A2800010A4D701FFA8AFA01318025D34503D85F
:103A3800E64568D3984566DC01339C42E6D1F445F7
:103A4800D7D1F9617B6ABA6913449BB2D3457B62CB
:103A580006D97B6A3A6A9846D6183B699E42A2D331
:103A6800BC68802D1CBF0AF101031FFA83FA0AF112
:103A7800020189B22046FEF785F82368796A012594
:103A88005A19226020461D70FEF77CF823685344BB
:103A980023602B46D7F800D0DBE4674B85E63388F4
:103AA800FF2BA8BFFF23DBB269E41AF0AFFC0028A4
:103AB8003FF464AC03780A2B2BD8B0F9023088FBAA
:103AC8000312DB17C3EBA2039BB2FF2BA8BFFF2394
:103AD800DBB254E498E8220069E61AF097FC002863
:103AE8003FF44CAE03780A2B3FF648AEB0F90430E9
:103AF800B0F9061003EB830383F3500521EAE17163
:103B0800ADB289B23CE6FB69BC681A463B7D1370CE
:103B1800A7E70023DCE7552D00F09A80572D40F0E9
:103B2800BE80531C336012F8378B07F1270101332D
:103B3800336013F8010C01F8010F9A42F7D1DFF84E
:103B48000CA19AF80050002DFDD13C484FF0010916
:103B5800082106468AF80090FEF742FE384B18689E
:103B680022F08EF9374B2946304683F80090FEF74D
:103B780073FC29463046FEF76FFC09213046FEF7F4
:103B88006BFC41463046FEF767FC07F128084546BE
:103B980007F15E09A5EB080B5FFA8BFB0A2130469B
:103BA800FEF75AFC59463046FEF756FC15F801BB9D
:103BB8000B213046FEF750FC59463046FEF74CFCC8
:103BC800002021F02FFB4D45E4D11C480821054673
:103BD800FEF742FCA0212846FEF73EFCA02128461D
:103BE800FEF73AFC00212846FEF736FC10F02000CC
:103BF800F4D1134B0646186822F048F90125022132
:103C08000E48FEF7EDFD8AF800602B4621E4531CB0
:103C1800336013780A2B01F006813046FDF77CFFEC
:103C28003046FDF779FF01253046FDF775FF2B4635
:103C38000FE400BFC81F0020D02900200030014039
:103C480030720020C5480020EC3A0308BD48002027
:103C5800531C336092F80080B8F1FF0F01F05D81CA
:103C6800B8F1FE0F01F0EE803046FDF749FF96E807
:103C78000C009B1A002B07DD531C336013781BB90B
:103C8800B8F10C0F41F27681B8F1270F00F2938258
:103C9800F84B012523F818002B46FFF7DABB7068AC
:103CA8000B3D811AEF2D00F286820FF2080E5EF8A6
:103CB80025F000BFB94A0008BF410008BF4100080D
:103CC800BF410008BF410008BF410008BF410008CC
:103CD800BF410008BF410008BF410008BF410008BC
:103CE800BF410008BF410008BF410008BF410008AC
:103CF800BF410008BF410008BF410008BF4100089C
:103D0800BF410008BF410008BF410008BF4100088B
:103D1800BF410008454A0008BF4100089B4B000806
:103D2800BF410008714B0008BF410008BF410008AF
:103D3800BF410008494B0008BF410008EF4A00088E
:103D4800BF410008E34B0008BF410008BD4B000815
:103D5800BF410008154C0008BF41000897490008FA
:103D6800BF41000845490008BF410008BF4100089D
:103D7800BF410008BF4100088F340008BF41000858
:103D880019490008BF410008BF410008FF48000862
:103D9800BF410008A5480008BF410008BF4100080E
:103DA800BF410008BF41000899480008BF4100080A
:103DB800BF410008BF41000859480008BF4100083A
:103DC8000B480008BF410008BF410008C947000868
:103DD800BF410008BF410008BF410008BF410008BB
:103DE800BF410008BF410008BF41000879450008ED
:103DF800BF41000805450008BF410008934400087A
:103E0800BF410008F5430008BF410008CD43000842
:103E18007143000855430008BF410008BF4100082E
:103E2800BF410008BF410008BF410008BF4100086A
:103E3800BF410008BF410008BF410008BF4100085A
:103E4800BF410008BF410008BF410008BF4100084A
:103E5800BF410008BF410008BF410008BF4100083A
:103E6800BF410008BF410008BF410008BF4100082A
:103E7800BF410008BF410008BF410008BF4100081A
:103E8800BF410008BF410008BF410008BF4100080A
:103E9800BF410008BF410008BF410008BF410008FA
:103EA800BF410008BF410008BF410008BF410008EA
:103EB800BF410008BF410008BF410008BF410008DA
:103EC800BF410008BF410008BF410008BF410008CA
:103ED800BF410008BF410008BF410008BF410008BA
:103EE800BF410008BF410008BF410008BF410008AA
:103EF800BF410008BF410008BF410008BF4100089A
:103F0800BF410008BF410008BF410008BF41000889
:103F1800BF410008BF410008BF410008BF41000879
:103F2800BF410008BF410008BF410008BF41000869
:103F3800BF410008BF410008BF410008BF41000859
:103F4800BF410008BF410008BF410008BF41000849
:103F5800BF410008BF410008BF410008BF41000839
:103F6800BF4100082B430008BF4100084F47000825
:103F780025470008BF410008BF410008BF410008AD
:103F8800BF410008BF410008BF410008BF41000809
:103F9800BF410008BF410008BF410008BF410008F9
:103FA800BF410008BF4100086B470008BF41000837
:103FB800E7450008BF4100083346000819460008D5
:103FC80009470008BF41000811430008BF41000825
:103FD800E9420008BF4100088D420008BF410008BF
:103FE8005D420008BF410008BF4100083342000895
:103FF80005420008F1410008C9410008A141000834
:1040080077410008BF410008BF410008BF410008D0
:10401800BF410008BF410008BF410008BF41000878
:10402800BF410008BF410008BF410008BF41000868
:10403800BF410008BF410008BF410008BF41000858
:10404800BF41000857410008BF410008BF410008B0
:10405800FF400008BF410008BF410008BF410008F9
:104068009B400008BF410008BF410008BF4100084D
:1040780081400008D06C0020C34B1B78DB0700F19F
:104088009A80012508F0C6FC08F06CFD2B46FFF766
:10409800E0B93046FDF734FD336838851A46591CB7
:1040A800316012F8021B326087F82A105A7887F8B4
:1040B8002B20DA1C32609A7887F82C201A1D32607F
:1040C800DA7887F82D205A1D32601B7987F82E3050
:1040D80007F1280000233B86FDF76CFCAB4AAC4B8C
:1040E8001268801A4FF0010561F10001C3E904016B
:1040F8002B46FFF7AEB9531C336013780F2B5AD8F1
:10410800911C3160C3EBC303A2495078C854D01C3A
:1041180030600B4491785970111D3160D1789970D5
:10412800511D31601179D970911D31605179197122
:10413800D11D31609179597102F108013160D2794C
:104148009A7101251DF0ECFA2B46FFF782B930462B
:10415800FDF7D6FCDFF84482A8F80E003046FDF7DC
:10416800CFFC0125A8F80C002B46FFF772B93046A2
:10417800FDF7C6FCDFF83C82A8F810003046FDF7D2
:10418800BFFCA8F812003046FDF7BAFC0125A8F8D4
:1041980014002B46FFF75DB91346511C316013F824
:1041A800020B3360D31C5178336092781BF0B4FE55
:1041B80000287FF468A94FF0FF352B46FFF749B96F
:1041C8001346511C3160744913F8020B08703360B0
:1041D800724953788B70D31C3360714B92789A7004
:1041E80001252B46FFF735B96E4B6F4918684E22EB
:1041F80001252EF00FFA2B46FFF72BB91146531C59
:1042080033606A4B11F8020B18703160517859709D
:10421800D11C316092789A703046FDF771FC644B7E
:104228000125D8802B46FFF714B93046FDF768FC06
:10423800DFF87C81A8F800003046FDF761FCA8F89B
:1042480002003046FDF75CFC0125A8F804002B4667
:10425800FFF7FFB8DFF8609199F80030002B3FF4C2
:1042680012A9DFF8588100253046FDF749FC17F000
:104278005FF999F80030A8EC010A01359D42F3DB9B
:10428800FFF701B90D2996D1531C33601578072D16
:1042980091D8DFF82C9130464FF00C08FDF730FC30
:1042A80008FB05F809EB0805A8803046FDF728FC4F
:1042B800E8803046FDF724FC336828811A46591CEB
:1042C800316012F8021BA97232605B78EB723046DB
:1042D800FDF7FEFB012549F808002B46FFF7B9B8A2
:1042E800531C33601078060600F1EA86264B1B78CB
:1042F800DD073FF5C8A8032828BF0020012508F0DE
:104308006DFB2B46FFF7A5B81F4B1B78D8073FF569
:10431800BAA8012509F00CF808F024FC2B46FFF791
:1043280098B81346511C316013F8025B3360D31CF4
:10433800507833609178002D00F09086012D7FF43D
:10434800A2A80DF0E3FD2B46FFF783B8531C33609A
:104358001378002B00F088864FF4004001250DF0FB
:104368004DF92B46FFF775B8074B1B7813F0010181
:104378007FF421AF531C3360107801250DF000FD48
:104388002B46FFF766B800BFAB5A00202473002005
:10439800382300205833002014630020605D00207B
:1043A800705D002034510020B05C0308585D002087
:1043B80048460020B0670020C94D00206C35002019
:1043C800983200201346511C3160C04913F8020B83
:1043D800C8703360BE4953784B71D31C3360BD4BF2
:1043E8009278DA7001252B46FFF733B83046FDF78F
:1043F80087FB3046FDF784FB3046FDF781FB3046EE
:10440800FDF78AFB3368B44D1946581C2A6830609A
:1044180011F8020B82F82C003160597882F83610B6
:10442800D91C31609B7882F837303046FDF774FB31
:104438003046FDF771FB3046FDF76EFB3046D5F888
:104448000080FDF75DFBA8F83A003046D5F80080FB
:10445800FDF756FB33687268A8F83800D11A0129AD
:104468000ADD591C2A6831601B7882F82E303046E4
:10447800FDF752FB33687268D31A032B00F3668684
:1044880028681DF079FDFEF7FEBF531C3360924D7E
:10449800DFF86082137888F805303046D5F8009048
:1044A800FDF72EFBA9F820003046D5F80090FDF75F
:1044B80027FB72683368A9F81E00D11A072900F390
:1044C8002986D11A032900F3ED85D21A002A05DDC1
:1044D800591C2A6831601B7882F8263008F0A4FA43
:1044E80024F068FF7D4B1B68002B00F0C685286808
:1044F80001251DF0A9F92B46FEF7ABBF1346511C49
:104508003160DFF8F08113F8021B88F8021033607D
:10451800734953780B70D31C3360724D93782B71A9
:10452800131D3360D378092BA8BF09233046AB701D
:10453800FDF7E6FA336872682880D11A012905DD8B
:104548003046FDF7DDFA33687268E8819A4240F038
:104558009F8508F069FA336872689A423EF493AF0F
:104568005A1C32601B78EB7001252B46FEF771BF91
:104578005D4B1B68002B3EF486AF19F061F8FF28ED
:104588003EF481AF3046FDF7BBFA3F2840F2048580
:10459800DFF86481002588F8005033687268A8F84D
:1045A8000400D21A012A7EF76EAF1A46591C3160F0
:1045B80012F8021B88F8021007F168003260002226
:1045C8005D7800F8402D19F00DF897F82830AB42C7
:1045D8003EF459AF284619F029F8FEF754BF3E4B70
:1045E8001868D31C014621329D1E356013F8035C00
:1045F8000D705D1E356013F8025C4D70336013F862
:10460800015C8D7003339A4201F10301ECD138E764
:10461800364B1B78D9073EF536AF354B4FF4C87289
:1046280001251A802B46FEF714BF09297FF7C3AD71
:10463800DFF8C8801346511CD8F80050316013F8D1
:10464800021B297033605378AB70D31C33609378A6
:10465800642B02F10401A8BF64236B713160D37825
:10466800642B02F10501A8BF6423AB713160137993
:10467800EB71931D33605379642B02F10701A8BFD6
:1046880064232B7231609379EB7002F10803336075
:10469800D3792B713046FDF733FA72683368688135
:1046A800D11A00290CDD591CD8F800003160521AC3
:1046B800002A1978417203DD9A1C32605B784370D6
:1046C800012517F095FD2B46FEF7C3BE605D00205F
:1046D8007C6F0020705D002034510020885D002030
:1046E800545D0020B0670020B05A0020AB5A00206B
:1046F8008246002014630020B45A0020385100205C
:10470800B94B1B78DA073EF5BEAEB84A13780125D7
:1047180043F0040313702B46FEF79BBE531CB448AA
:10472800336001781378002940F031840422027044
:10473800B04A9B00138009F017FBAF4B0125986125
:104748002B46FEF786BEDFF8E88200233046C8F81D
:104758000030FDF7BDF90125C8F800002B46FEF72B
:1047680078BEC1F34705122D3FF625ADC5B107F157
:10477800680307F1260903EB4508CA46A8F1420871
:104788003046FDF7BDF92AF8020FD045F8D19B4B0A
:1047980039F8022F23F8022FD145F9D1112D09D864
:1047A800974A6B00023B13440021223223F8021F70
:1047B8009A42FBD1934A01231D461370FEF749BE66
:1047C800914B1B78012B3EF65EAE1146531C3360AD
:1047D800DFF8608211F8023B88F802303160D31CA0
:1047E80092F801E03360C31A012B917840F3F28309
:1047F8003046FDF785F90125A8F800002B46FEF79D
:1048080028BE531C336092F80080B8F1110F3FF6B0
:10481800D2AC931C33607D4D537805F81830304680
:10482800FDF76EF940F6CA039842A8BF184640F251
:10483800EE23984205EB4801B8BF18460125A0F2BF
:10484800EE222B46192092FBF0F24A70FEF701BEC9
:104858001346511C6E4D316013F8021B29713360E9
:1048680053786B713046FDF74BF9336828805A1C32
:1048780032601B78AB713046FDF742F933686880C7
:104888005A1C32601B78EB7101252B46FEF7E1BDFF
:104898000125FDF781FF2B46FEF7DBBD531C336076
:1048A8005C4B1278DFF890811A700023C8F800304A
:1048B8003046FDF70DF93368D8F800205649574DB2
:1048C80010435A1CC8F8000032601B780B7230463F
:1048D800FDF716F928603046FDF712F96860304692
:1048E800FDF70EF9A8603046FDF70AF93046FDF7E6
:1048F80007F9FEF7C8BD4A4B02F1080101323260E0
:1049080012F8010C03F8010F9142F7D1FEF7BBBD75
:104918001346511C3160434913F8025B8D703360B4
:1049280055784D7083423EF4AEADD31C3360324BA4
:1049380092781A7201252B46FEF78BBD0723B1FB2F
:10494800F3F3C3EBC305491B7FF435ACDBB203F1CA
:10495800FF395FFA89F9002B3EF495ADDFF8C8A05E
:1049680009F101090D46531C336092F900102E4BD2
:104978004FF0000893F902208A4203F1080300F07F
:10498800A78208F10108B8F1060FF3D113E4531C0C
:10499800336013780E2B3FF60EAC911C31605578BE
:1049A800032D3FF608AC2148062101FB03F143180B
:1049B80002F1030E5D71C6F800E095784554111DAB
:1049C8003160D1785970511D316011799970911DFC
:1049D80031605179D970D11D316092791A710125F0
:1049E8002B46FEF736BD00BFAB5A00203C6D0020B9
:1049F8004C380020446D0020382300204A42002013
:104A08004C42002070420020A25F0020E4440020B5
:104A180060460020A45D0020BC71002020320020E8
:104A2800BB710020805D0020E87100205034002018
:104A3800443400203E6D0020B85F0020511C3160D6
:104A480015783B62132D3FF6B6AB911C3160507858
:104A58007A6213F027FF00283FF4ADAB7A6AC249A7
:104A6800007801F82500D01C306001EB85059078AE
:104A78006870101D3060D078A870501D30601279B1
:104A8800EA703B6A01F1500202E004318A4207D021
:104A980008780028F9D18D78C8788542F5D20123A5
:104AA800B24A83F00103012513702B46FEF7D1BCEF
:104AB800AF4B10294FF0000228BF10211A605A602E
:104AC8009A60DA601A7400293EF4DDAC3268013B62
:104AD80011440132326012F8010C03F8010F8A42C6
:104AE800F7D1FEF7D0BC531CA24D336013782B725C
:104AF8003046FDF705F8A8833046FDF701F828830E
:104B08003046FCF7FDFF32686883531C3360127827
:104B1800EA747268D31A032B00F381823368D11ABE
:104B2800052900F36C82D21A002A7EF7ACAC5A1C15
:104B380032601B7885F8213001252B46FEF789BCA9
:104B4800531C33608C4915780D70C01A00287EF705
:104B58009AAC931C33605378003318BF01230125A6
:104B68004B702B46FEF775BC3046FCF7C9FFDFF8E3
:104B78002882C8F800003046FCF7C2FFC8F80400D5
:104B88003046FCF7BDFF0125C8F808002B46FEF7A4
:104B980060BCDFF808820023C8F800303046FCF714
:104BA80097FFD8F8003001250343C8F800302B469A
:104BB800FEF74FBC531C336015781F2D3FF6FBAA38
:104BC80005297FF4F8AA3046FCF782FF6B4B43F8BF
:104BD800250018F0B3FAFEF756BC684D05F14008F9
:104BE8003046FCF78DFF3368A5F88000591C1A463B
:104BF800316012F8021B85F8821032605B7885F804
:104C080083300435A845EBD1FEF73DBC531C336017
:104C1800584B12785A7501252B46FEF71ABC1346D5
:104C2800511C3160564D13F8021B6970336053787C
:104C38002B70D31C33609378AB703046FCF760FF61
:104C480033682881591C1A46316012F8021B6971B1
:104C580032605B78AB7101252B46FEF7FABB494BF6
:104C68003A6A9B68D4F800905A44934280F0C9800D
:104C78003A6AA3EB0208FDF703FD42464946386A43
:104C8800FDF7A6FB236803442360002D3EF4FBAB2D
:104C9800B042BEF6F8AB002100E0236801305A1C90
:104CA800B04222601970F8D1FEF7EDBB3368726824
:104CB8009A4240F0DA80344BFF221A704FF0000A13
:104CC800324D1DF029FF51462022314885F800A0B9
:104CD8002EF033FE87F828A097F82830072B00F22B
:104CE8005481DFF8BC902A4E524697F8283003EBDF
:104CF800430309EBC3035B7CE3B197F8283003EB6C
:104D0800430309EBC30320215B699BB197F8283063
:104D180003EB430309EBC303586946F8220020F06C
:104D2800F3FE2B7856F8230021F0B0F82A780132E8
:104D3800D2B22A7097F828300133DBB287F82830CE
:104D480097F82830072BD0D92368591C21601A708E
:104D5800B8F1000F3EF497AB0E4BC8F800300125B0
:104D68002B46FEF776BB00BFD84300205801002031
:104D780076560020BC710020A45D002070510020F0
:104D8800C0500020C81F0020382300207B7300205B
:104D98003C73002091FF020820320020B85F0020F9
:104DA800F0660020002D7FF45AAF59462046FCF7E4
:104DB800E9FE23685A1C22601D70C74B26689D684F
:104DC8003B6A0BEB0302AA4200F2F680FDF758FC9F
:104DD8005A463146386AFDF7FBFA23680125034431
:104DE80023602B46FEF735BB3046FCF789FE326858
:104DF80071687B6A9142834660D106461D46FEF77C
:104E08009CBDFDF73DFC5A464946386AFDF7E0FA75
:104E18002368034423603BE73046FCF771FEDFF864
:104E2800EC82FEF7EDBB931C3360AC4B51781970E4
:104E3800D11C316091785970111D3160D2789A7007
:104E4800FEF721BB931C33605578022D3FF6B3A9BA
:104E58003046FCF755FEA24B03EB45034FF0FF35F8
:104E6800A3F856002B46FEF7F4BA5A1C19463260CE
:104E78009C4811F8022B027031605B784370042A59
:104E880003D9FF2A7EF44BAC18E797490978994271
:104E980005D8022A7EF443ACFF2B7EF440AC23688D
:104EA80001255A1922601D70B8F1000F3EF4EBAAD3
:104EB8008E4BC8F800302B46FEF7CBBA511C316038
:104EC80012781D46131C064618BF0123FEF735BD90
:104ED8000AEBC80B30468BF80210FCF711FE33685A
:104EE8002AF838001A46591C316012F8021B8BF850
:104EF800031032605A788BF80420DA1C32609A78F2
:104F08008BF806201A1D32600135DB788BF80530E6
:104F1800A9457FF428ADFEF7B6BA931C3360744BED
:104F280051781970D31C3360DFF8B481937888F80E
:104F38005530131D3360D37888F854303046FCF769
:104F4800DFFDA8F850003046FCF7DAFD3046FCF7E4
:104F5800D7FD96E80C009B1A012BA8F852007EF7A3
:104F680092AA3046FCF7CCFD0125A8F85A002B463A
:104F7800FEF76FBA5A4B0030984418BF012001253C
:104F880088F85E002B46FEF764BA5246DCE6042930
:104F98007EF479AAFFF7CCBBC50800F007030135FA
:104FA8000133EDB2DFF868812846194688F80130E8
:104FB80019F0D2F9FFF7EFBA3B6AED1AFDF760FB7B
:104FC8002A463146386AFDF703FA2368034423600A
:104FD800FEF759BA474B1A88012512FB0EF22B46E9
:104FE80092FBF1F2A8F80020FEF733BADA46C7F8C8
:104FF80024B0FEF73CBD7D62AA46FEF738BD5A1CB8
:1050080032601B78EB723046FCF762FD3368E8606B
:105018005A1C32601B782B743368726883E53046FB
:10502800FCF76EFDA8843046FCF76AFD33687268A9
:10503800E884D11A03297FF772AD1A46591C3160EA
:1050480012F8021BA97732605B7885F82030304669
:10505800FCF756FD33687268688460E501251CF02A
:1050680016FE2B46FEF7F5B9234A1368012523F4EB
:10507800004313602B46FEF7ECB920482049214A2B
:10508800214B036001250B6013602B46FEF7E1B945
:105098005A1C32601B78003318BF012388F8073088
:1050A800FFF757BA3046FCF72BFDA8F80E0030463C
:1050B800FCF726FD33687268A8F81000FFF705BAF8
:1050C80000F07F00032828BF002001250CF03AFFDC
:1050D8002B46FEF7BEB900BFC81F00204B5E00205C
:1050E800D06C002038230020C94D0020D5050108C8
:1050F80038720020DE5B00202C510020545900201B
:10510800A8590020105A00205D050008505D0020B5
:10511800B45A00203046FCF7F3FCA8F80A003046E1
:10512800FCF7EEFCA8F80C003046D5F80090FCF728
:10513800E7FCA9F822003046D5F80090FCF7E0FC1F
:1051480033687268A9F82400FFF7BBB93046D5F870
:105158000080FCF7D5FCA8F8320030462E68FCF732
:10516800CFFCB086FFF78CB92DE9F04F2DED0E8BF3
:10517800DFF8F4B097B0DBF8042007905846904762
:10518800002800F08E82BBF8A87000218BF851101F
:10519800002F6DD1BBF93A00DBF82450DBF828105A
:1051A800BBF93860DBF82040BBF93C20DFF8BCA035
:1051B800401B521ACBF830009BF85210CBF8342021
:1051C800341B0BF12C00CBF82C4012F045F8DAF820
:1051D8000020910041F17987DBED0C5A1F4CDBED83
:1051E8000B7A1F4994ED406AD4ED416A94ED427AF6
:1051F800D4F80C2109681B4B0593B8EEE58ADBED62
:105208000D5AF8EEE77AF8EEE58A013277EE867AFB
:1052180038EE268A78EE878A8A42C4ED407A84ED91
:10522800418AC4ED428AC4F80C2101F04A8393F8FC
:1052380000E0BEF1140F02F09B870023D4F814514C
:105248000693062D01F29784DFE815F00416161769
:1052580028152917020CC6168A1500BF60230020DE
:1052680090380020E84D002028630020B065002019
:10527800DE4BDF481A6808934FF47A76B6FBF2F2F1
:10528800C2EB421602EB8602D600DA4BDFF8C8837F
:1052980044780593B6B2B7421D78B8F9060003F012
:1052A8008980DBF87C30BBF93810DBF8602003F12B
:1052B800010E07EE901A0A44BEF1010FCBF87CE00C
:1052C800CBF86020F8EEE77A03F08180DBED1B5A1B
:1052D800DBED1D6A07EE10EA37EEE56AB8EEC75A4D
:1052E800012F86EE057A37EE257A77EEC77A8BEDB1
:1052F8001C7AE7EE866A8BED1B7AF0EE667ACBEDC8
:105308001E6ACBED1D6A03F00384DBF89030BBF90D
:105318003A10DBF8642003F1010E07EE901A0A44F4
:10532800BEF1010FCBF890E0CBF86420F8EEE77AF5
:1053380003F06880DBED205ADBED226A07EE10EA05
:1053480037EEE56AB8EEC75A012F86EE057A37EED2
:10535800257A77EEC77A8BED217AE7EE866A8BEDB0
:10536800207AF0EE667ACBED236ACBED226A03F061
:10537800A783DBF8A430BBF93C10DBF8682003F105
:10538800010E07EE901A0A44BEF1010FCBF8A4E013
:10539800CBF86820F8EEE77A03F04F80DBED255A6A
:1053A800DBED276A07EE10EA37EEE56AB8EEC75A72
:1053B800012F86EE057A37EE257A77EEC77A8BEDE0
:1053C800267AE6EE276A8BED257AF0EE667ACBED43
:1053D800286ACBED276A03F06683874CA8F8060095
:1053E800BBF8A820059B013A1D78ABF8A8200899BE
:1053F8000022072D4A608A60CA6040F0598108F08F
:10540800B3FC059BDFF850821D78079BC01A94F8FF
:105418002831A8F800000993002B40F04F81744A06
:105428005279002A01F07A81744A1278013AD2B28C
:10543800072D84F8282102F01A8200230A93704B62
:10544800D4F83421D3F800A0684B0893079B9FED4C
:105458006D6AD4ED4C9A6C49C4F834319A1A07EE47
:10546800902AF8EE677AB7EE007AC6EE278A00250A
:10547800664BDFF8E891DFF8E881654F06932E4622
:10548800D1ED006A94ED4BDA9FED629ADFED62AAE6
:105498009FED62CA9FED62AADFED62BA9FED62BA24
:1054A80077EE69CA6CEEA6CAF4EEC7CAF1EE10FA36
:1054B80088BFF0EE47CA5D4B99ED008A2B44D3EDC7
:1054C800007AF5EE407AF1EE10FA17D0584B2B44DB
:1054D80093ED007A78EE476AB0EEE66AF4EEC67AA3
:1054E800F1EE10FA08D5F5EEC06AF1EE10FACCBF6D
:1054F80037EE878A37EE678A83ED008A4D4B1A8824
:10550800930739D0022E37D09AF82E104A4B07EE5F
:10551800901A2B4493ED007A4B42F8EEE76A07EEB7
:10552800903A26EE877AF8EEE77AB4EEE77AF1EE6B
:1055380010FA0AD407EE901AF8EE677AF4EEC77AF2
:10554800F1EE10FA88BFF0EE477A3C4B3C4903EB8A
:10555800460331F91600B3F90C30C31A07EE103AB6
:10556800B8EEC77AD007E7EE497A41F17380354B38
:1055780093ED008A27EE888A089B94F868212B44CB
:1055880093ED01EA78EE4EDA002A00F0F7802E4B10
:10559800D4F86C2107991B688A1A9A4240F3EE8066
:1055A8009AF84830022B02F0A181022E04F04584BB
:1055B800264B1B68990700F19780254B87ED00CA99
:1055C8001B689342C0F2CA80F7EE007AF4EEE79ABD
:1055D800F1EE10FA40F1D28008991E4BD1ED017A14
:1055E80093ED007AF0EEE77A3CE000BFA06500207A
:1055F80014630020E84D002060230020545D002043
:105608003451002000247449645A0020645B00204F
:10561800705B0020CDCCCC3DAE47813F0000000040
:105628000000C84200003443610BB63B585A0020C2
:10563800A424002030510020B0240020605D002008
:10564800E0500020405A00206C5A0020DC50002016
:10565800685A0020745A0020EC4D0020982400203D
:105668007C5B0020F4EEC77AF1EE10FA40F18680F8
:10567800D1ED027AF0EEE77AB4EEE77AF1EE10FABD
:105688007CDDD1ED037AF0EEE77AB4EEE77AF1EE5D
:1056980010FA73DD0F4B1B689B075FD50E490F4B44
:1056A80043E00F4B0F4C1D780593072D3FF4A7AE31
:1056B80094F828310993002B3FF4B1AE013B84F8EC
:1056C8002831012D01F0A88217B0BDEC0E8BBDE882
:1056D800F08F00BFDC500020E0500020605D00200B
:1056E800E84D002060230020D34BD449DFF8C8E3FD
:1056F80031F916C09EED008ADFF8C0E387ED00CAD5
:1057080003EB460028EE098AB0F90C00A0EB0C0068
:1057180007EE900AF8EEE77ADEF8000027EE888AAE
:10572800904278EE4EDABFF64FAFB3F90C20B1F9DC
:1057380000E0C348AEEB020E00688EEAEE72A2EB00
:10574800EE7282421ADAB3F90E30B1F90220D21A97
:1057580082EAE273A3EBE27398420FDDB94B1A8831
:10576800002384F86831002A43F06A85B64AB74BAB
:105778001178186881F0010120F08EFBB44B2B449E
:1057880093ED000A069B2DEE000A022E20EE2D0A4C
:10579800A3EC010A069304F00D83AE4BD7ED006A23
:1057A80093ED007AAC4BD3ED007AAC4B93ED006AE5
:1057B800AB4B67EE277A2B4427EEAC7AD3ED007A11
:1057C80067EE277AF0EE665AEDEEA75AB1EE467A02
:1057D800B4EEE57AF1EE10FA08DCB4EEE56AF1EE23
:1057E80010FA8CBFB0EE657AB0EE467A94ED4C6A4A
:1057F800F7EE007AB4EEE76AF1EE10FAACBF0123D7
:10580800002343B1F0EEE66AF0EEC77AF4EEE67AEA
:10581800F1EE10FA01D587ED007A022E04F0AC8281
:10582800904A914B52F826001B68B0EE4E0A9847F2
:105838008E4A8F4B52F826001B6898479AF83730E3
:1058480023B18C4B1B88002B00F06B87B0EE4C8A81
:10585800894B38EE400A2B4493ED008A83ED000A09
:105868009AF8483030EE480A20EE288A002B33D0C8
:10587800824B1B7813F0010300F0B886F7EE007A2C
:10588800F4EEE79AF1EE10FA94F86831C1F2E68482
:10589800002B00F0EB87D4F86C31079AD31A784ABA
:1058A80012689A4218DD774BD3ED007AF0EEEDDA04
:1058B800F4EEE7DAF1EE10FA42F12980614B1A882A
:1058C800002384F86831002A00F09C866E494A69F2
:1058D80012B10A6813604B746C4B94F878212B440E
:1058E80093ED000A2DEE000A20EE088A88ED008A62
:1058F80032B9069B87ED00CA03ED01CA88ED00CADC
:105908000136032E09F1040908F1040807F1040718
:1059180005F104057FF4CFAD059B1A78072A01F03D
:10592800B384012A01F090870023069394F880211C
:10593800002A41F07E81DFF888A1554BDAF8002073
:105948001968D60491F82C0000F10687DFF87491E5
:10595800504AB9F81A3092ED006A4F4A4F4DD2EDCD
:10596800005AD5ED036A4E4A84ED646A07EE103A90
:105978004C4B92ED005AD3ED007AD3ED013AD3EDBA
:10598800024A84ED626AB8EEC77A35EEC64A012249
:1059980036EEC77A84ED614AC4ED655A84F89821D9
:1059A800C7EE055A0A8D534206EE103A3E4BDFED1C
:1059B8003F6A93ED005A3E4B93ED004AB7EE007AEA
:1059C800F4EEC75A35EE045AF1EE10FA88BFF0EE3D
:1059D800475A35EE275AB8EEC66AF4EEE65AF1EEA3
:1059E80010FA07EE902AB4EEC65AB8BFF0EE665A1F
:1059F800F1EE10FAC4ED685AB8EE677A01F1048343
:105A0800B4EEC75AF1EE10FA88BFB0EE475A264BEB
:105A1800DFED286AD3ED017A254B93ED014A77EE45
:105A2800847A25EE265A77EEA37AB4EEE76AF1EE89
:105A380010FA52DC48E000BF605D0020E050002012
:105A4800705A0020FC720020FE72002000730020B3
:105A5800145A00205059002018000020885A0020AD
:105A6800205A00205859002054590020AC590020D1
:105A7800A859002030510020D0240020AB5A002023
:105A88006C5A0020785A0020047300202C5A0020F9
:105A980034510020EC5B0020445D0020044F0020BE
:105AA80050460020705B0020645B0020000000006E
:105AB8007C5B00206F12833A405A0020685A00200D
:105AC800B0650020BC710020B4EEE77AF1EE10FA60
:105AD8008CBFB0EE676AB0EE476AEC4B4A8DD3EDE7
:105AE800027A9FEDEB7A534204EE103A74EEA77AED
:105AF800B8EEC44A26EE076AF4EEC47AF1EE10FA5C
:105B08000AD407EE102AB8EE474AB4EEE74AF1EE97
:105B180010FA88BFB0EE674ADE4ADFEDDD7A5278C8
:105B280024EE274A0AB9B1EE444A002841F0D0854C
:105B3800B7EE003AD84E3278002A02F04B86D749A1
:105B4800DFEDD77AD1ED024AD1ED016A91ED037A02
:105B580066EE244AE5EE264AE4EE074A63EE244A56
:105B6800F4EEE74AF1EE10FAB4BFF0EE673AF0EE61
:105B7800643A98BFF0EE647A012ACDED0E4A02F03D
:105B88004E8691ED067AD1ED052AD1ED076A26EE0B
:105B9800077AA5EE227AA4EE267A23EE077AB4EEE7
:105BA800E77AF1EE10FAB4EEE37A8CBFF0EE676AAA
:105BB800F0EE476AF1EE10FA88BFF0EE676AB4BFFC
:105BC800F0EE637AF0EE477A022A8DED0F7A00F054
:105BD800DE8091ED0A7AD1ED092AD1ED0B3A26EE55
:105BE800077AA5EE227AA4EE237A23EE077AB4EE9A
:105BF800E67AF1EE10FAB4EEE77A8CBFF0EE663A88
:105C0800F0EE473AF1EE10FA98BFF0EE636AA8BFDB
:105C1800F0EE477A032A8DED107A00F0B88091ED06
:105C28000E7AD1ED0D2AD1ED0F3A26EE077AA5EEC0
:105C3800227AA4EE237A23EE077AB4EEE67AF1EE1E
:105C480010FAB4EEE77A8CBFF0EE663AF0EE473A17
:105C5800F1EE10FA98BFF0EE636AA8BFF0EE477A4B
:105C6800042A8DED117A00F09280D1ED123AD1ED2F
:105C7800112A91ED137A66EE233AE5EE223AE4EE24
:105C8800073A63EE233AF4EEE63AF1EE10FAF4EE50
:105C9800E73A8CBFB0EE667AB0EE637AF1EE10FAAE
:105CA80098BFF0EE476AA8BFF0EE637A052ACDEDFB
:105CB800123A6CD0D1ED163AD1ED152A91ED177A3A
:105CC80066EE233AE5EE223AE4EE073A63EE233A2B
:105CD800F4EEE63AF1EE10FAF4EEE73A8CBFB0EEE5
:105CE800667AB0EE637AF1EE10FA98BFF0EE476A82
:105CF800A8BFF0EE637A062ACDED133A47D0D1ED6E
:105D08001A3AD1ED192A91ED1B7A66EE233AE5EE9F
:105D1800223AE4EE073A63EE233AF4EEE63AF1EE7D
:105D280010FAF4EEE73A8CBFB0EE667AB0EE637A1A
:105D3800F1EE10FA98BFF0EE476AA8BFF0EE637A6A
:105D4800072ACDED143A22D091ED1E7AD1ED1D2A05
:105D5800D1ED1F3A26EE077AA5EE227AA3EE847AD1
:105D680027EE037AB4EEE67AF1EE10FAB4EEE77AAB
:105D78008CBFB0EE666AB0EE476AF1EE10FA8DEDB0
:105D8800157A98BFF0EE466AA8BFF0EE477A77EE2C
:105D9800E67AF7EE006AF4EEE67AF1EE10FAC4ED70
:105DA8004C7A43F3D78586EEA77A022ADDED0F7A7F
:105DB80067EE244A67EE877ACDED0E4ACDED0F7A6D
:105DC8002DD0DDED107A67EE877A032ACDED107AB3
:105DD80025D0DDED117A67EE877A042ACDED117AA8
:105DE8001DD0DDED127A67EE877A052ACDED127A9D
:105DF80015D0DDED137A67EE877A062ACDED137A92
:105E08000DD0DDED147A67EE877A072ACDED147A86
:105E180005D0DDED157A27EE877A8DED157A2149C3
:105E2800096811F080530A9301F0CB81F6EE005A0D
:105E3800C4ED685A002A02F09D8494F998311A49F1
:105E480094ED656AC87894ED645ADAF80010DFF8C2
:105E580068E0164FDEED004AB7F906E0B9F81A70A7
:105E68000B9707EE103A124BD4ED616A1D78114B6F
:105E7800D4ED627A1B780893BDEEC66A01F48053AC
:105E880016EE10CABDEEC56A0D9317E0645B0020DC
:105E98006F12833AA45D0020C94D0020C045002040
:105EA80000000000C85B00201C530020506D00203B
:105EB800AB5A0020D4670020BC45002001F48003C1
:105EC80001F01007B8EEC77A0C9305F0010816EE3A
:105ED800101A002840F06487002F41F0D582D34D76
:105EE8009DED0E5A95ED006AD14825EE866AA5EE1D
:105EF800076AB0EE675AA6EE265ABDEEC56A16EED8
:105F080010EA16EE107AE645A8BF67467145C8BF85
:105F18000F4606EE107AB8EEC66A012A80ED006ACE
:105F280000F0DC8095ED046A9DED0F5A25EE866A37
:105F3800A5EE076AB0EE675AA6EE265ABDEEC56A08
:105F480016EE10EA16EE107AE645A8BF67467145C8
:105F5800C8BF0F4606EE107AB8EEC66A022A80ED70
:105F6800016A00F0BB8095ED086A9DED105A25EE98
:105F7800866AA5EE076AB0EE675AA6EE265ABDEE07
:105F8800C56A16EE10EA16EE107AE645A8BF67460F
:105F98007145C8BF0F4606EE107AB8EEC66A032AE6
:105FA80080ED026A00F09A8095ED0C6A9DED115A19
:105FB80025EE866AA5EE076AB0EE675AA6EE265A5F
:105FC800BDEEC56A16EE10EA16EE107AE645A8BFD1
:105FD80067467145C8BF0F4606EE107AB8EEC66A26
:105FE800042A80ED036A79D095ED106A9DED125A66
:105FF80025EE866AA5EE076AB0EE675AA6EE265A1F
:10600800BDEEC56A16EE10EA16EE107AE645A8BF90
:1060180067467145C8BF0F4606EE107AB8EEC66AE5
:10602800052A80ED046A59D095ED146A9DED135A3E
:1060380025EE866AA5EE076AB0EE675AA6EE265ADE
:10604800BDEEC56A16EE10EA16EE107AE645A8BF50
:1060580067467145C8BF0F4606EE107AB8EEC66AA5
:10606800062A80ED056A39D095ED186A9DED145A17
:1060780025EE866AA5EE076AB0EE675AA6EE265A9E
:10608800BDEEC56A16EE10EA16EE107AE645A8BF10
:1060980067467145C8BF0F4606EE107AB8EEC66A65
:1060A800072A80ED066A19D095ED1C6A9DED155AF0
:1060B80065EE865AE7EE055AE6EEA57AFDEEE77A32
:1060C80017EE905AAC45A8BFAC46A942D8BF614666
:1060D80007EE901AF8EEE77AC0ED077AB8F1000FEC
:1060E80000F06C87534A1268002A40F07487524ABD
:1060F800127892B1307868B14D4FDFF85C81002595
:10610800E8B2D8F80030B7EC010A98473078013582
:106118008542F5DB494A12689047059B1A78072A99
:1061280001F0A1800026DAF80020530500F1D1879C
:10613800434B1B78BBB1434AB9F81A30B2F9062071
:106148009A4210DC404B1B78012B01F09583192BE8
:1061580001F092830E2B06D0082B04D03B4D002370
:10616800AB60C4F8403194F8AA5125B1384B1B886C
:106178009F0741F02F8394F8B021002A40F0488708
:1061880099F81E70002F00F02984022F01F0D582A3
:10619800032F41F0CE8299F82030C3EB431103EB73
:1061A8008101C90089B299F81F300233DBB2002A95
:1061B80000F05585002900F0528526480768B1FB94
:1061C800F7F10FB2A4F8E071002B03F0438007EE5B
:1061D800907AF8EEE77AF7EE006A86EEA77A1B4D1A
:1061E800012BD4ED7D6AD5ED007A77EEE67A67EE7D
:1061F800877AC4ED797A3BD0D5ED017AD4ED7E6A01
:1062080077EEE67A022B67EE877AC4ED7A7A2FD09A
:10621800D5ED027AD4ED7F6A77EEE67A032B67EE46
:10622800877AC4ED7B7A23D018E000BFC0450020F0
:10623800985B00204C590020FC6A0020D0670020A1
:1062480058010020506D0020A45D0020044F00205C
:1062580030510020885D0020C8670020D5ED037A02
:10626800D4ED806A77EEE67A67EE877AC4ED7C7AB9
:1062780005990978092903F0ED81002F40F3B483CB
:106288009BB394ED7D7AD4ED797A77EE877A012BFA
:10629800C4ED7D7AC5ED007A21D094ED7E7AD4EDF7
:1062A8007A7A77EE877A022BC4ED7E7AC5ED017A89
:1062B80015D094ED7F7AD4ED7B7A77EE877A032B2D
:1062C800C4ED7F7AC5ED027A09D0D4ED807A94EDD9
:1062D8007C7A77EE877AC4ED807AC5ED037A013B44
:1062E800022BB8BF0223DBB20993099B002A18BF0F
:1062F80002239E46C84BDFEDC96A1A68059B917850
:106308001878137807EE903AF8EEE77AB0EE007A4C
:1063180067EEA67AF4EEC77AF1EE10FA40F35F86DC
:10632800DFEDBF6A37EEC77AB0EE676AA7EE266A76
:10633800F0EE466A95ED007A9FEDBA6A27EE066A96
:10634800F0EEC65A84ED546AC4ED575A99B107EE77
:10635800101AB8EEC75A9FEDB17A66EE064A25EED6
:10636800075AB7EE007A37EE457A64EEA54AA4EEEE
:10637800857A26EE076A9FEDAC7A537926EE877AFE
:1063880027EE067ACBB1DFEDA56A9FEDA86A65EE28
:10639800A65A06EE903AF8EEE66A65EEA65AF4EECC
:1063A800C65AF1EE10FA01F38981B7EE006A76EE6B
:1063B800655AC6EE256A27EE267A0C289FED9C8A38
:1063C800DFED9C6A00F02487B4EEC87AF1EE10FA8B
:1063D80098BFB0EE478AB4EEE68AF1EE10FAB8BF7D
:1063E800B0EE668A84ED4E8ABEF1000F00F0DD80C3
:1063F800B0EE007AF4EEC77AF1EE10FA05DD37EE6A
:10640800C77ADFED876AE7EE267A95ED017ADFED48
:10641800856A27EE267AF0EEC75A84ED557AC4EDE0
:10642800585A99B106EE901A9FED7C6AF8EEE66A22
:1064380027EE075A66EE866AB7EE006A36EE666A97
:1064480025EE255AA5EE266A27EE067ADFED766A4E
:10645800937967EEA67A67EE877AABB107EE103AC2
:10646800B8EEC77A9FED6D6ADFED706A27EE257A80
:1064780027EE067AB4EEE67AF1EE10FA41F31081CF
:10648800DFED6D6A67EEA67A0C2800F0A186DFEDD5
:10649800686A9FED687AF4EEE67AF1EE10FA88BF42
:1064A800F0EE667AF4EEC77AF1EE10FAB8BFF0EEC5
:1064B800477ABEF1010FC4ED4F7A76DD5378DFEDF0
:1064C800576A07EE903AF8EEE77AB0EE007A67EE90
:1064D800A67A537AF4EEC77AF1EE10FA05DD37EEB4
:1064E800C77ADFED4F6AE7EE267A95ED027ADFED9F
:1064F8004D6A27EE267AF0EEC75A84ED567AC4ED37
:10650800595A9BB106EE903A9FED446AF8EEE66A56
:1065180027EE075A66EE866AB7EE006A36EE666AB6
:1065280025EE255AA5EE266A27EE067ADFED3E6AA5
:10653800D37967EEA67A67EE877AFBB107EE103A51
:10654800B8EEC77A9FED356ADFED386A27EE257A0F
:1065580027EE067AB4EEE67AF1EE10FA01F39C80A3
:10656800B5EEC07AF1EE10FA02F1FE82B7EE006ADB
:1065780036EE477AC6EE076A67EEA67A0C2800F070
:106588006586DFED2B6A9FED2B7AF4EEE67AF1EE65
:1065980010FA88BFF0EE667AF4EEC77AF1EE10FAD8
:1065A800B8BFF0EE477AC4ED507A092800F0FC85B0
:1065B80099F82150002D40F0B185002384F8B031BE
:1065C8001E4B1B7823B91E4DAA78002A41F0C180C2
:1065D800059B1D78072D7FF474A807F0C5FB194BA0
:1065E800059A801B1578D880FFF76BB894F8682156
:1065F800002A3FF471A9144A84F868311288002AE5
:106608007FF464A9114A124B1178186881F00101CE
:106618001FF042FCFFF760B9385100200AD7233C2D
:10662800D7A368416F12033B00004843A4707D3F25
:1066380000C0F94400C0F9C40000C842BC480020AA
:106648003E6D0020EC4D0020FC720020FE72002000
:106658000073002094ED577AB1F90000D4ED586A20
:10666800B1F902E0E24AF4EEC76A80EAE0738EEA22
:10667800EE71A3EBE073F1EE10FAA1EBEE71B8BF87
:10668800F0EE476A8B42B8BF0B4607EE103A137814
:10669800B8EEC77A27EE097A002B40F0B880D54BC0
:1066A80093ED006AB4EEEA6AF1EE10FA41F14C801B
:1066B800F7EE005A75EEC65A3BEEC77A65EE8B5A6E
:1066C800CD4BA7EE256A93ED007A26EE076AB5EE64
:1066D800C06AF1EE10FA40F27085CAEE065AB7EEBB
:1066E800007AB0EE476AA6EEE56AF0EE466AF4EE86
:1066F800C76AF1EE10FA88BFF0EE476AF5EEC06A95
:10670800F1EE10FAB8BFF0EE4C6ABC4B93ED007A8C
:1067180067EE877AA7EEA68AFEF72EBF0122FEF75C
:1067280087BEB74BB74A2B4493ED007AD2ED007A77
:10673800B54B67EE277AF7EE006AF4EEE67AF1EEEB
:1067480010FA93ED007A88BFF0EE667A67EE877AE2
:1067580027EE888AFFF77CB8AC4BDFF8EC921A7802
:10676800D5075CBFB9F81820A4F88C21A84AA94D10
:106778001288D5ED037A07EE102AB8EEC77AF4EE40
:10678800C77AF1EE10FA41F2C587A34D2B8807EEC0
:10679800103AB8EEC77AF4EEC77AF1EE10FAC1F201
:1067A80077809E4A9E4D92ED006AD5ED006A94F975
:1067B8009821C4ED646A76EE665A012AC4ED626ACD
:1067C800C4ED615A84ED656A01F0EE85079BC4F853
:1067D8009C31002537EEC77AFCEEE77A914E84EDBE
:1067E800687A17EE902AA4F88C21012296ED005AB7
:1067F80084F898218C4A954241F279878B4BD3EDE6
:10680800007AD3ED013AD3ED024AFFF7C9B87A4BC3
:1068180093ED005AB5EEC05AF1EE10FA40F3CD846C
:10682800834BD3ED004AF5EEC04AF1EE10FA40F37F
:10683800C48434EEC77A66EECA5A87EE246AC5EE77
:10684800856AB7EE007AB4EEC76AF1EE10FA88BF2F
:10685800B0EE476AB5EEC06AF1EE10FA76EE876AD6
:10686800B8BFB0EE4C6A66EE266A40E7714AD2EDD0
:10687800007AB0EEC87AB4EEE77AF1EE10FA7FF754
:106888002BA86D4AD2ED007AB0EEED7AB4EEE77A35
:10689800F1EE10FA7FF720A8684AD9ED007A92ED58
:1068A800007AF0EEE77AF4EEC77AF1EE10FA7FF5A7
:1068B80013A801220799C4F86C1184F86821FEF71F
:1068C800EEBF07EE102A1978DFF88081C4F80C7142
:1068D800B8EEC77AF7EE006A132986EE879AB8F9F8
:1068E8000400B4F810619BED070A01F0E984544AEA
:1068F800544992ED001AD2ED053A92ED122A92ED22
:10690800173AD2ED091AD2ED0E4A92ED016A92EDCC
:10691800064A92ED0A7AD2ED0F5AD2ED132AD2ED39
:10692800186A92ED045AD2ED030A67EE897A69EE85
:10693800288A29EE088AE1EE273A01EB8607002526
:10694800A2EE283AC4F80051C4F80451E1EE884A8E
:10695800A6EE274AE7EE085A92ED167A92ED0D6AEE
:1069680092ED021AD2ED0C1AC7ED003AE2EEA86ACF
:1069780025EE635A27EE437A92ED0B2AD2ED152ABB
:10698800C7ED204AA0EEE34A26EE646AD2ED143A37
:1069980082ED054AA1EE275AF0EE477AE1EEE45A75
:1069A800A2EE086AE2EEC36AE3EEA87A82ED065A1E
:1069B800C2ED0E5A82ED0F6A87ED403AC2ED176AB2
:1069C800C2ED187AC4F80851721C02F01F02A4F82C
:1069D8001021A8F80400059BFEF729BCA4F8E07173
:1069E800002A3FF4EDAD0B4D4FF0020E82E400BFDC
:1069F8004C5A0020545A0020485A0020445A00207B
:106A0800BC2400203C5A0020385A0020AB5A0020F1
:106A180054460020044F002056460020445D0020C4
:106A2800404600205C4600208FD00300705B0020A9
:106A3800505A00207C5A0020785A0020805A0020A2
:106A4800203B0020B4380020BC710020EC4D002011
:106A5800BC4A1178D4F81871BB4B9FEDBC7AFE0084
:106A68009A1982ED007A002979D0B948B0EE476AC0
:106A7800F0EE476A0022F0EC017A013267EEA77A5D
:106A880005EE902AB4EEE77AF1EE10FAF8EEE55A40
:106A9800B8BFB0EE677A8A4276EEA76AA7EEA56A13
:106AA800E9D1F5EEC06A9A19F1EE10FA82ED007A92
:106AB80055DDC6EE265AA74AA7490988F7EE007A97
:106AC80075EEE75AD2ED007A65EEA77AFDEEE77A21
:106AD80017EE902A812A42F353808A42A8BF0A46B9
:106AE80007EE902AF8EEE77A9C4AF01902EB80024A
:106AF80092ED057AD2ED003A92ED066A92ED014ADE
:106B0800D2ED046AD2ED034A92ED025AA3EEA77AB7
:106B1800A4EE276A66EEC76AA7EE646ABDEEC77A76
:106B2800E5EE276A17EE100A812882ED056AC2EDA4
:106B3800066A42F322808142A8BF014607EE901AF6
:106B4800F8EEE77AFCEEE77ACDED087ABDF820207A
:106B580099198A801FB9BEF1130F02F0E786BEF1BA
:106B6800150F41F0ED801E44DFF81082B28828F836
:106B78001720D4F814517A4A013582FB053251198D
:106B8800EA17C2EBA102C2EBC202AD1AC4F8145153
:106B98007448D4F81C11079B734D02682D78C4F80B
:106BA8001C31591A0A440260002D64D107EE901A6C
:106BB8006E4EDFF8E0916E4FB8EEE78A06F5F07595
:106BC80006F51378F6EC017A9BED070ADBF8083234
:106BD800F8EEE77A284627EE800A9847A5F1E00004
:106BE800DBF828319847A5F17000DBF89831984711
:106BF800D6F8EC00DBF8AC309847D7ED007AA9EC72
:106C0800010AE0EE087A2435A845E7EC017AD9D1E3
:106C1800059B1D78FEF749BD564B574A19681288DF
:106C2800564BC96919805A8017B0BDEC0E8BBDE868
:106C3800F08F534B534E1A7812F0010F327840F010
:106C48003983002A00F03E8592004F494F48DFF80B
:106C580048A1DFF848912BF0DDFCFFF743BAB4F800
:106C6800E071013F3FB2002FA4F8E0717FF7B8AEA2
:106C7800474DFFF705BB07EE901A3C4D454BDFF833
:106C8800FC80DFF8EC900694F8EEE78A05F5B87614
:106C980000271C46CDF82480059BDBED077A1B787E
:106CA800172B00F0A08195ED007AB8EEC78A082B63
:106CB80028EE278A07D1B0EE480A08932BF080FE09
:106CC800089BA8F80000DAF8002092000BD5002FE6
:106CD80003F00281B0EE480ADBF8083206F17000D2
:106CE8009847B0EE408AB0EE480ADBF82831A6F1A2
:106CF80070009847DBF8983130469847059B1B7819
:106D0800032BB0EE408A00F07A81D5F8F000DBF86A
:106D1800AC30B0EE480A9847D9ED007AA4EC010AE5
:106D2800E0EE287A0137032F06F1240608F102085D
:106D380005F10405E9EC017AAED1059B069C1D78A6
:106D4800FEF7B3BC963800208C3B00200000000002
:106D5800602300209838002094380020B43A00209E
:106D680093244992804500208C38002054630020E9
:106D7800844500208C6F002096320020EC4D0020C6
:106D8800AB5A0020C94D00206C350020985B0020CC
:106D9800044F0020A4650020B0650020BC710020CD
:106DA800002F00F09186B8F1000F42F0A982089BED
:106DB800CD4D002B42F0F68095ED006A9DED0E5A00
:106DC800CA4825EE866AFDEEE44AA5EE076AB0EEEB
:106DD800675AA6EE265A14EE901ABDEEC56A16EE4C
:106DE80010EA16EE107AE645A8BF67467145C8BF97
:106DF8000F4606EE107AB8EEC66A012A80ED006AE0
:106E080000F0DF8095ED046A9DED0F5A25EE866A45
:106E1800A5EE076AB0EE675AA6EE265ABDEEC56A19
:106E280016EE10EA16EE107AE645A8BF67468E45BC
:106E3800B8BF0F4606EE107AB8EEC66A022A80ED91
:106E4800016A00F0BE8095ED086A9DED105A25EEA6
:106E5800866AA5EE076AB0EE675AA6EE265ABDEE18
:106E6800C56A16EE10EA16EE107AE645A8BF674620
:106E78008E45B8BF0F4606EE107AB8EEC66A032AEA
:106E880080ED026A00F09D8095ED0C6A9DED115A27
:106E980025EE866AA5EE076AB0EE675AA6EE265A70
:106EA800BDEEC56A16EE10EA16EE107AE645A8BFE2
:106EB80067468E45B8BF0F4606EE107AB8EEC66A2A
:106EC800042A80ED036A7CD095ED106A9DED125A74
:106ED80025EE866AA5EE076AB0EE675AA6EE265A30
:106EE800BDEEC56A16EE10EA16EE107AE645A8BFA2
:106EF80067468E45B8BF0F4606EE107AB8EEC66AEA
:106F0800052A80ED046A5CD095ED146A9DED135A4C
:106F180025EE866AA5EE076AB0EE675AA6EE265AEF
:106F2800BDEEC56A16EE10EA16EE107AE645A8BF61
:106F380067468E45B8BF0F4606EE107AB8EEC66AA9
:106F4800062A80ED056A3CD095ED186A9DED145A25
:106F580025EE866AA5EE076AB0EE675AA6EE265AAF
:106F6800BDEEC56A16EE10EA16EE107AE645A8BF21
:106F780067468E45B8BF0F4606EE107AB8EEC66A69
:106F8800072A80ED066A1CD095ED1C6A9DED155AFE
:106F980065EE865AE7EE055AE6EEA57AFDEEE77A43
:106FA80017EE905AAC45A8BFAC46A942D8BF614677
:106FB80007EE901AF8EEE77AC0ED077A002A3FF458
:106FC80091A892004A4949482BF024FB494A126883
:106FD800002A3FF48CA819F0D7FFFFF788B8F0EE25
:106FE800676AFFF7A7B995ED007A0BEB4702B8EE91
:106FF800C78A128FA8F8002028EE278A63E62BF0AC
:10700800DFFCA8F8000080E6B0EE465AFEF7FFBCA9
:1070180039493A4BD1F8EC101B6844F6206081429C
:10702800A8BF0146B1F57A7FB8BF4FF47A7189B22B
:1070380013F0100FA4F8B211DAF8003000F023842E
:10704800DB0441F1A1852E4BD3F800E0BEF8327085
:107058007F082C4D2C48D4F8B431D5ED037AA0FB29
:1070680001018809642191FBF0F11429BDEEE77A4A
:1070780004EB4305A8BF142101338B42C4F8B43193
:1070880017EE10CAA4BF0023C4F8B43104EB4303BD
:10709800A5F8B8C1B3F9B83107EE103AB8EEC77A17
:1070A80077EEC77AFDEEE77ACDED067ABDF91810CE
:1070B80081EAE173A3EBE173BB4201F32D87134926
:1070C8004FF07E530B60FFF75BB8114B0593114CE3
:1070D8005EE5DBF80830002B3FF42AA80E49A1F141
:1070E8004C009847FFF724B8C0450020985B002063
:1070F8006C3500204C59002064080020C85B002033
:1071080034510020044F0020D34D62101800002095
:10711800E84D002060230020746300201E21CE4823
:10712800FBF7B4F800283FF448AACC4B1B88580654
:107138003FF543AA94F80432AB4242F01C82C84B94
:10714800D4ED827AD3ED016A94ED505ADFEDC55A39
:107158009FEDC56A27EEC57A68EE277AA8EE267AEB
:10716800E5EE267AB4EEE57AF1EE10FA88BFB0EED5
:10717800657AB4EEC67AF1EE10FAF4EEE57AB8BFA5
:10718800B0EE467AF1EE10FA88BFF0EE657AF4EECA
:10719800C67AF1EE10FAB8BFF0EE467A84ED4E7A70
:1071A800C4ED507AFFF709BAFDEEC87AAF4A17EE78
:1071B800903A9780D380FFF7FBB9DFEDAD6AFFF710
:1071C800A4BADAF8001049023EF530AEFEF732BE36
:1071D8009FEDA47ADFEDA46AA449F4EEC77AF1EE34
:1071E80010FA98BFB0EE677AFDEEE77AB4EEE67A69
:1071F800F1EE10FA17EE903AB8BFB0EE667ABEF12B
:10720800010F84ED4F7A4B803FF758A9FFF7D0B9AB
:10721800B4EEC87AF1EE10FA98BFB0EE478ABDEE28
:10722800C77AB4EEE68ADFF844C2F1EE10FA17EE38
:10723800103AB8BFB0EE668A84ED4E8AACF80030DA
:10724800BEF1000F7FF4D4A8FFF7B2B9BDEEE77A1C
:10725800864B17EE102A9A80FFF793B9002B3EF45D
:107268003BABFEF718BB06F07FFD059B7F491A78FC
:10727800069B072AA0EB030088807EF453AF06F034
:1072880073FD0646FEF74FBF06F06EFD059BDFF85F
:10729800DC811A780A9B012AA0EB0300A8F80200F7
:1072A80000F0D482072A7EF43FAB06F05DFD06901D
:1072B800FEF73CBB002A00F00582D4ED583A94ED65
:1072C800574AD4ED627A6B4994ED617A91ED005A90
:1072D800D4ED555A94ED546A674D6848F4EEC43AB3
:1072E800F3EE046AF1EE10FA77EEA64A00F11E8377
:1072F80095ED026A26EE656AB0EE674AA6EE074A81
:10730800B4EEE44A34EE666AF1EE10FA48BFB0EE25
:10731800456A012A80ED006A00F0D48195ED066A7D
:1073280026EE656AB0EE674AA6EE074AB4EEE44A6E
:1073380034EE666AF1EE10FA48BFB0EE456A022AEA
:1073480080ED016A00F0BE8195ED0A6A26EE656A55
:10735800B0EE674AA6EE074AB4EEE44A34EE666A2F
:10736800F1EE10FA48BFB0EE456A032A80ED026AD2
:1073780000F0A88195ED0E6A26EE656AB0EE674AC0
:10738800A6EE074AB4EEE44A34EE666AF1EE10FA65
:1073980048BFB0EE456A042A80ED036A00F0928186
:1073A80095ED126A26EE656AB0EE674AA6EE074AC0
:1073B800B4EEE44A34EE666AF1EE10FA48BFB0EE75
:1073C800456A052A80ED046A00F07C8195ED166A0D
:1073D80026EE656AB0EE674AA6EE074AB4EEE44ABE
:1073E80074EE666AF1EE10FA48BFF0EE456A062AB6
:1073F800C0ED056A00F06681D5ED1A6A66EEE56AA9
:10740800B0EE674AA6EE874AB3EE046AB4EEE44AE1
:1074180074EE466AF1EE10FA48BFF0EE456A072AA4
:10742800C0ED066A00F04E81D5ED1E6ADFF850A067
:10743800DFF8509066EEE55AE5EE877AF4EEE74A13
:1074480077EEC67AF1EE10FAC8BFF0EE457AC0EDD5
:10745800077AFEF747BE00BFC85B00203051002006
:107468001800002000C0F94400C0F9C4EC4D002009
:1074780000000000BC450020C0450020985B0020AB
:10748800B0650020BC710020B8F1000F41F0028205
:10749800DB4D9DED0E5A95ED006ADA4825EE866AB9
:1074A800A5EE076AB0EE675AA6EE265ABDEEC56A83
:1074B80016EE10EA16EE107AE645A8BF6746714543
:1074C800C8BF0F4606EE107AB8EEC66A012A80EDEC
:1074D800006A3FF476AD95ED046A9DED0F5A25EEEE
:1074E800866AA5EE076AB0EE675AA6EE265ABDEE82
:1074F800C56A16EE10EA16EE107AE645A8BF67468A
:107508007145C8BF0F4606EE107AB8EEC66A022A61
:1075180080ED016A3FF455AD95ED086A9DED105A6E
:1075280025EE866AA5EE076AB0EE675AA6EE265AD9
:10753800BDEEC56A16EE10EA16EE107AE645A8BF4B
:1075480067467145C8BF0F4606EE107AB8EEC66AA0
:10755800032A80ED026A3FF434AD95ED0C6A9DED87
:10756800115A25EE866AA5EE076AB0EE675AA6EEAE
:10757800265ABDEEC56A16EE10EA16EE107AE645F2
:10758800A8BF67467145C8BF0F4606EE107AB8EE29
:10759800C66A042A80ED036A3FF413AD95ED106ABC
:1075A8009DED125A25EE866AA5EE076AB0EE675A77
:1075B800A6EE265ABDEEC56A16EE10EA16EE107A49
:1075C800E645A8BF67467145C8BF0F4606EE107A64
:1075D800B8EEC66A052A80ED046A3FF4F2AC95ED70
:1075E800146A9DED135A25EE866AA5EE076AB0EE79
:1075F800675AA6EE265ABDEEC56A16EE10EA16EED2
:10760800107AE645A8BF67467145C8BF0F4606EE23
:10761800107AB8EEC66A062A80ED056A3FF4D1AC46
:1076280095ED186A9DED145A25EE866AA5EE076A4F
:10763800B0EE675AA6EE265ABDEEC56A16EE10EAF7
:1076480016EE107AE645A8BF67467145C8BF0F46D3
:1076580006EE107AB8EEC66A072A80ED066A3FF48D
:10766800B0AC95ED1C6A9DED155A65EE865AE7EEAD
:10767800055AE6EEA57AFDEEE77A17EE905AAC4584
:10768800A8BFAC46A942C8BF8C4607EE90CAF8EE20
:10769800E77AC0ED077A91E4DFED5B6AFEF76CBF2D
:1076A800B5EEC07AF1EE10FA01F15A82B7EE006A2F
:1076B80036EE477AC6EE076AFEF7E4BEDFED526A99
:1076C800FEF779BEDFF878A1DFF87891FEF70ABDFA
:1076D8004E494A79002A3EF42BAA4D4A1278002ACC
:1076E8003EF426AA0B784B49DFED4B4A07EE903A59
:1076F8000B88B8EE677A07EE902A06EE903AF8EE15
:10770800E77AF8EE666A67EE277AB7EE007A87EED0
:10771800A63AB4EEE43AF1EE10FA88BFB0EE643A55
:10772800B4EEC73AF1EE10FAB8BFB0EE473AFEF73A
:1077380001BA3A4B5988FEF736BDB4F8B21101F5D3
:107748007A7189B2FEF72FBD354B93ED006AFEF7CB
:10775800BEBF344F3B78013B0D2B24D8DFE813F034
:10776800F506BB07E606CB0623002300A4078F0710
:1077780034070E0067075B07860702072A4B1B784A
:10778800002B02F0F5801A2014F0CEFC002842F0FD
:10779800EF80264B1B78002B42F0EA8009233B70D0
:1077A8001FF07AFAAA78012A00F063852B79012B59
:1077B80001F05985022B7EF40BAF3B78012B7EF448
:1077C80007AF1A4B1B78002B7EF402AF20F0B4F9F8
:1077D800FEF7FEBE164B9FED177AD3ED087AF4EE4E
:1077E800C77AF1EE10FA00F2F9849FED137A134D7F
:1077F800D5ED037A77EE877AC5ED037AFEF7BBBC41
:10780800C0450020985B00200000C842C0500020FE
:10781800024F0020EC4E0020713DAA3F3442002068
:10782800485A0020A25F0020A65D0020A75D002026
:10783800584500208FC2753C00000000044F00200E
:10784800B0650020BC710020DFF8708206F08CFA69
:107858009049D4F87C2109680690821A511AC4F814
:107868007C01A8F80420A8F80610FEF75FB806F017
:107878007BFA0A90FDF7E3BD874B9B7B002B3EF418
:107888006DACFEF770BCDD003FF5DAABFEF778BCF7
:10789800B4F88C51954240F2028594F8A451002D19
:1078A80040F06E877D4A7E4E92ED007AD6ED007AE2
:1078B80094F99821C4ED647A77EE676A012AC4EDD9
:1078C800627AC4ED616A84ED657A02F03D80079BB7
:1078D800C4F89C31734A9FED747A92ED005A84ED96
:1078E800687A012284F89821FEF784BF6F4B1B88C1
:1078F800002B40F0E8856E4A6E4B117818681EF030
:10790800CBFAD4F86C21079B9A1AFDF74EBE6A4B46
:10791800D9ED007A93ED007AF0EEE77AF4EEC77AC3
:10792800F1EE10FA7DF7D8AFFDF7C8BFD5ED015AD3
:1079380065EEC65AB0EE674AA5EE874AB4EEE44A49
:1079480074EE665AF1EE10FA48BFF0EE455A012A75
:10795800C0ED005A3FF4B6AED5ED055A65EEC65AED
:10796800B0EE674AA5EE874AB4EEE44A74EE665A6A
:10797800F1EE10FA48BFF0EE455A022AC0ED015A5E
:107988003FF4A0AED5ED095A65EEC65AB0EE674A87
:10799800A5EE874AB4EEE44A74EE665AF1EE10FAA0
:1079A80048BFF0EE455A032AC0ED025A3FF48AAEAA
:1079B800D5ED0D5A65EEC65AB0EE674AA5EE874A70
:1079C800B4EEE44A74EE665AF1EE10FA48BFF0EEEF
:1079D800455A042AC0ED035A3FF474AED5ED115A46
:1079E80065EEC65AB0EE674AA5EE874AB4EEE44A99
:1079F80074EE665AF1EE10FA48BFF0EE455A052AC1
:107A0800C0ED045A3FF45EAED5ED155A65EEC65A80
:107A1800B0EE674AA5EE874AB4EEE44A74EE666AA9
:107A2800F1EE10FA48BFF0EE456A062AC0ED056A85
:107A38003FF448AED5ED196A66EEC66AB0EE674AFD
:107A4800A6EE874AF3EE045AB4EEE44A74EE656A89
:107A5800F1EE10FA48BFF0EE456A072AC0ED066A53
:107A68003FF430AED5ED1D6ADFF854A0DFF854902E
:107A780026EEC66AE6EE077AF4EEE47A77EEE57A61
:107A8800F1EE10FAB8BFF0EE457AC0ED077AFEF7CE
:107A980029BB00BF885D002014610020445D0020E0
:107AA800404600205C46002000000000FC720020D8
:107AB800FE72002000730020805A0020EC4D002048
:107AC800B0650020BC710020089BD94D002B41F007
:107AD8008D8095ED006A9DED0E5AD64825EE866A92
:107AE800FDEEE44AA5EE076AB0EE675AA6EE265AFE
:107AF80014EE901ABDEEC56A16EE10EA16EE107A6C
:107B0800E645A8BF67467145C8BF0F4606EE107A1E
:107B1800B8EEC66A012A80ED006A3EF4DFAA95ED48
:107B2800046A9DED0F5A25EE866AA5EE076AB0EE47
:107B3800675AA6EE265ABDEEC56A16EE10EA16EE8C
:107B4800107AE645A8BF67468E45B8BF0F4606EED1
:107B5800107AB8EEC66A022A80ED016A3EF4BEAA1F
:107B680095ED086A9DED105A25EE866AA5EE076A1E
:107B7800B0EE675AA6EE265ABDEEC56A16EE10EAB2
:107B880016EE107AE645A8BF67468E45B8BF0F4681
:107B980006EE107AB8EEC66A032A80ED026A3EF451
:107BA8009DAA95ED0C6A9DED115A25EE866AA5EE03
:107BB800076AB0EE675AA6EE265ABDEEC56A16EEFB
:107BC80010EA16EE107AE645A8BF67468E45B8BF9C
:107BD8000F4606EE107AB8EEC66A042A80ED036AEC
:107BE8003EF47CAA95ED106A9DED125A25EE866A40
:107BF800A5EE076AB0EE675AA6EE265ABDEEC56A2C
:107C080016EE10EA16EE107AE645A8BF67468E45CE
:107C1800B8BF0F4606EE107AB8EEC66A052A80EDA0
:107C2800046A3EF45BAA95ED146A9DED135A25EE9D
:107C3800866AA5EE076AB0EE675AA6EE265ABDEE2A
:107C4800C56A16EE10EA16EE107AE645A8BF674632
:107C58008E45B8BF0F4606EE107AB8EEC66A062AF9
:107C680080ED056A3EF43AAA95ED186A9DED145A1E
:107C780025EE866AA5EE076AB0EE675AA6EE265A82
:107C8800BDEEC56A16EE10EA16EE107AE645A8BFF4
:107C980067468E45B8BF0F46FEF7FEB9664ED4ED6F
:107CA800017A94ED006A3188726977EEA77AF0EE6E
:107CB800006AB0EE677AA6EE267A4E1E04EBC6017D
:107CC800D6EE267A08391032F6EE003A27EE237AF5
:107CD80067EEA37A84ED207AC4ED217A574C2746C3
:107CE80004F1800091ED027A91ED036AD7ED036A01
:107CF800D7ED027A52ED014A12ED025A37EE674A81
:107D080076EEC65A77EE277AE4EE845A013EA1F160
:107D18000801E5EE047A07F1080702F1080236EED9
:107D2800267A00F10800E4EE877AE5EE475A67EE16
:107D3800A37A25EEA37AC0ED007A80ED017AD1D13D
:107D4800BEF1140F7EF417AF06F00EF8069BDFF8AD
:107D58000081C01AA8F80200D4F81451FEF70BBF2E
:107D6800D4F81831B4F810C1354ACCF120095FFABB
:107D780089F90CEB431702EB87075FEA990201F0D8
:107D8800F285013216012F482F4907EB060807F143
:107D9800100212ED024A12ED035A12ED016A12EDB9
:107DA800047A50ED024A50ED035A50ED016A50ED45
:107DB800047A64EE244A65EE255A66EE266A67EE72
:107DC800277A1032904541ED024A41ED035A41EDC0
:107DD800016A41ED047A00F1100001F11001D8D1D7
:107DE8001A48A6F110010F4400EB0108214419F0CC
:107DF800030209D0B7EC017AF8EC017A67EE277A2A
:107E0800013AE1EC017AF5D1BCF1000F41F0318083
:107E1800BEF1140F7EF4AFAE05F0A6FF069BDFF8A7
:107E28003080D4F81451C01AA8F80200FEF7A3BE97
:107E3800C0450020985B00209C380020602300206B
:107E4800B4380020443A002070230020343A00203F
:107E5800EC4D0020D04E318873684FEA51094FEA43
:107E680089005FEAD10C04EB000204EB810500F005
:107E7800A18000F110010CF1010CC84F02EB0C1CA1
:107E88002944103203F1100E05F1100050ED032AB9
:107E980050ED043A17ED043A17ED032A50ED026A43
:107EA80010ED016A17ED021A57ED010A11ED044AA7
:107EB80011ED035A52ED044A52ED035A12ED027ABB
:107EC80052ED017A51ED021A11ED010A73EE238A7F
:107ED80032EE228A47ED048A07ED038A71EE268A7C
:107EE80030EE868A47ED028A07ED018A74EE848AAD
:107EF80035EE858A42ED048A02ED038A77EE218AFF
:107F080037EE808A42ED028A02ED018A73EE633A07
:107F180075EE655A1EED035A32EE623A74EE644A03
:107F280025EE638A1EED044A23EE052A64EE652ACF
:107F3800A3EE048A1032944524EE843AA3EE842AF0
:107F480007F110070EF1100EA5EE853A00F11000AA
:107F580001F11001E4EE852A00ED078A00ED082AF8
:107F680001ED073A41ED082A5EED055A1EED065A65
:107F780071EE666A30EEC66A31EEC77A70EE677ADD
:107F880026EE253A65EEE63A25EE674A67EE054A9B
:107F9800E6EE053AA6EE853AA7EE254AE7EEA54AAB
:107FA80000ED063A40ED053A01ED064A41ED054A75
:107FB8007FF46CAF1FFA89F91A464946784825F0CC
:107FC8006FFE72684946284625F06AFE059B1A78B6
:107FD800142A7FF4C1AEB7E6D4F818517149724833
:107FE800724BEA00114415448A88196800EE102A79
:107FF800643AC82AA8BFC822782AB8BF782207EEF0
:10800800902AB8EEC07AF8EEE77A00EB850577EEAD
:10801800670A77EE876A67EE877A20EEA67AB8EE67
:10802800400AC7EE870A2846D5F81490D5F8188074
:10803800EF692E6A26F022FA059BC5F8149093F88A
:1080480000E0C5F81880BEF1140FEF612E6201F050
:10805800A484D4F81821564BD4F81451013283FB68
:108068000213A3EBE27303EB4303D31A0135C4F8FD
:108078001831C4F8145175E6474E4948B268B189B9
:1080880029F0E0FA059B93F800E0BEF1140F01F027
:108098009184D4F814510135C4F81451FFE5454EC4
:1080A80031785FEA910C01F0AC85434F0CF101097E
:1080B8004FEA491907EB090807F12002A7F17000F8
:1080C80012ED076A52ED056A12ED037A52ED017A54
:1080D80052ED025A12ED084A52ED064A12ED045AC0
:1080E80026EE066A66EEA66A27EE077A67EEA77A94
:1080F800A4EE046A20329045E4EEA46A00F1100070
:10810800A5EE057AE5EEA57AF1EEC65AB1EEE66A75
:10811800F1EEC76AB1EEE77A40ED085A00ED076A5A
:1081280040ED066A00ED057ACAD1A9F120023A4469
:1081380004EB0C1711F0030018BF08320FD052EDF2
:10814800017A12ED027A67EEA77A0138E7EE077A2C
:1081580002F10802B1EEE77AA7EC017AEFD1BEF19D
:10816800140F01F00A840135C4F81451FEF772BCEB
:1081780005F0FAFD059B069093F800E0BEF1140F98
:1081880005BFDFF83880D4F81451D4F81451A8F892
:108198000050FDF756B800BF9C380020702300201F
:1081A800602300208C3B002034650020A06500205F
:1081B8005655555596380020E0230020EC4D0020F8
:1081C800306E99BC2716983DA40DC93F843459BE1A
:1081D800DB0F4940D06D393A00000000F0EEE76A45
:1081E800B7EE005A35EE665A1FED0B4A5FED0B5A93
:1081F8001FED0A6A1FED0C7A94ED6B0AF1EEC54A81
:10820800E6EE845AF5EEC07AA6EEA56AF1EE10FA0B
:10821800A6EE867A48BF5FED127A27EE247A48BF29
:1082280037EEC77A27EE000A2AF0CAFBB0F5617F5D
:1082380000F38D8607EE900AF8EEE76A5FED1B7A89
:1082480066EEA76A07EE905ABDEEE67AF8EEE77A90
:1082580017EE103A2033402B41F281841FED220A99
:108268002AF0AEFB00B207EE900AB8EEE77AFFF705
:10827800BEBAC249C24B89681B6899423FF696AAA2
:108288003B780C3B022B7EF6A3A9BE4C3A702378B0
:10829800002B3EF49DA900232370FEF799B9BA4A32
:1082A80002F1500503E00432954200F06982137828
:1082B800262BF8D19678D3789E42F4D2FFF7EDBA00
:1082C800B24DB34F95ED004A95ED057AD5ED014ACB
:1082D80095ED066AD5ED046A95ED035AD5ED025A77
:1082E80067EE897A07EB8602A4EE277AA4EEA76ADE
:1082F80066EEC76AA5EE476AE5EEA76A20EE070AAA
:1083080085ED056AC5ED066A82ED007A29EE088AD0
:108318002AF056FB69EE288AD5ED0E5AD5ED176A74
:1083280095ED091AD5ED121A95ED0F5A95ED187AB3
:1083380095ED0A2AD5ED132A95ED0D6AD5ED167A35
:1083480095ED0C3AD5ED0B3A95ED154AD5ED144A55
:10835800E1EE085A002207EB8601E8EEA16A00B2B6
:10836800C4F80021A2EE085AC4F80421C4F8082170
:10837800A8EEA27A26EE656A67EEE67AA3EE655A5B
:10838800A3EE886AA6EEC47AE8EEA47A85ED0E5AC2
:10839800C1ED205A85ED0F6AC1ED406A85ED177A67
:1083A800C5ED187AFEF710BBD4F89C51079B5D1BEE
:1083B800FEF710BABBF93820CBF8201007EE902A48
:1083C8000121F8EEE77ACBF86020CBF87C10002288
:1083D800012FCBED1C7ACBED1B7ACBF8742001F082
:1083E8009D82B7427CF491AFBBF93A20CBF8642068
:1083F80007EE902A00210122F8EEE77ACBF8241044
:10840800CBF890200022012FCBED217ACBED207AFA
:10841800CBF8882001F08682B7427CF4AAAFBBF97A
:108428003C20CBF8682007EE902A00210122F8EEC4
:10843800E77ACBF82810CBF8A4200022012FCBED47
:10844800267ACBED257ACBF89C207CF4C6AF9FED3D
:10845800518A032D49D04CB107EE904AF8EEE77ADD
:10846800F4EEC87AF1EE10FA01F1D0834A4A4B4C87
:108478001168DBF86820A8F8060094F8200102EBE0
:10848800560292FBF6F60022CBF828608A620A634D
:10849800CA6228B1424A126832F480637CF4A0AF01
:1084A800404A126812F4003241F030823E481146C8
:1084B800835C012B02F10C0200F07783013118294B
:1084C800F6D1FCF78DBF39494B69002B3DF46DA8F7
:1084D8003748384B008893FBF0F00B684FF0010EDB
:1084E800186081F811E0FDF760B8B0EE480A2AF08C
:1084F80067FA00B2AFE724F017FF2F4A0292A2F101
:108508000C03252101930091A2F10A035021163A88
:1085180049201FF0F7F8A8B9284BAA7818604FF03F
:10852800FF31596007233B70FFF73DB9DFF88C80B6
:1085380024F0FAFE224AD8F80430126864339342D1
:10854800C1F07C83AA78FFF72EB91E4B1B78D90798
:1085580001F16A831F2013F0E7FD0028F2D00C23F5
:108568003B70EFE71F20069213F0DEFD069A002805
:108578007FF419A901233B70FFF715B9C81F002024
:108588008C5D0020A75D0020D8430020203B002000
:10859800B4380020000000008C6F00206023002009
:1085A8002C51002044340020805403080473002018
:1085B8001C73002020A10700563F0308485D0020D7
:1085C80024730020AB5A00201A2013F0ADFD0028B8
:1085D8003FF4E6A89B4B1B88002B7FF4E1A89A4B3D
:1085E8004520D3F8008024F067FF0E2024F064FFB4
:1085F80040461DF0D5FFDDF81C8040461DF0D0FF39
:10860800924A934B12681A6040460A233B701EF048
:1086180091F8FFF7C5B8012A01D1FAF7BDF80D2383
:1086280013203B700FF070FFAA78FFF7BCB8894B96
:1086380089495B680968C8338B4205D324F09AFEE0
:10864800AA7800283FF4AFA8032A93D1DFF8408224
:10865800D8F800000FF05CFA804B1B780022022B40
:10866800C8F8002001F00384AA7883E7012A01F002
:10867800D4820E2313203B700FF046FF62E724F0EC
:1086880053FE1EF03BFB00283FF45CAF24F072FE63
:1086980000283FF457AF6D4A6D4B12681A600A23E1
:1086A8003B70AA78FFF77FB824F03EFE6C4B0021A0
:1086B80005208DE80300A3F10802029153201FF062
:1086C80021F800287FF43EAF624BAA78186008238F
:1086D8003B70FFF768B8604B5E491B684B606148A8
:1086E80000230B60032103603970FFF75CB8DFEDEE
:1086F8005E7A5E4B94ED687AC3ED007AC3ED017A39
:10870800C3ED027A5A4BF0EE674AF0EE673A196801
:10871800FDF746B9574A584DD2ED006A574A95EDCC
:10872800006A1278C4ED646A84ED656A002A00F074
:108738001F8276EE665A94F99821C4ED615A013287
:10874800C4ED626A00F08985079BC4F89C31002556
:1087580037EE677AFCEEE77A494E84ED687A17EED1
:10876800902AA4F88C21FF2296ED005A84F89821CB
:10877800FEF740B8434B1D7805F00108FDF7AEBC85
:108788003C4A3D4DD2ED007A3C4A95ED007A12788C
:10879800C4ED647A84ED657A002A00F0658377EE8B
:1087A800676A94F99821C4ED616A0132C4ED627A6E
:1087B80000F0DB86079BC4F89C3100259FED2A7AE0
:1087C8002F4E84ED687AFF2296ED005A84F898219E
:1087D800FEF710B82C49DFED2D7A0968C4ED4C7A04
:1087E80011F080530A9340F0A683DAF8001011F4D0
:1087F80080030A9300F0CF8100230A93B6EE007A33
:1088080067EE877AF4EEE57AF1EE10FAC8BFF0EE7B
:10881800675A40F39083C4ED685AFDF70BBB73EEBB
:10882800E77AB7EE007AF4EEC77AF1EE10FAC4ED03
:108838004C7A41F38F8084EEA77A8DED0E7AFDF79E
:10884800EEBA00BFD85B0020D45B0020BC5B0020E0
:10885800B85B0020485D002024730020845D002060
:10886800044103081C70002000000000705B002019
:1088780034510020EC5B002044460020D4670020DF
:1088880058460020AB5A0020C85B0020000000803A
:1088980020700020D14D0D9B9DED0E5A95ED006A7C
:1088A800002B00F01B8725EE866ACD48A5EE076AE7
:1088B800B0EE675AA6EE265ABDEEC56A16EE10EA65
:1088C80016EE107AE645A8BF67467145C8BF0F4641
:1088D80006EE107AB8EEC66A012A80ED006A3DF409
:1088E80001AC95ED046A9DED0F5A25EE866AA5EE5A
:1088F800076AB0EE675AA6EE265ABDEEC56A16EEAE
:1089080010EA16EE107AE645A8BF67467145C8BF5B
:108918000F4606EE107AB8EEC66A022A80ED016AA2
:108928003DF4E0AB95ED086A9DED105A25EE866A98
:10893800A5EE076AB0EE675AA6EE265ABDEEC56ADE
:1089480016EE10EA16EE107AE645A8BF674671459E
:10895800C8BF0F4606EE107AB8EEC66A032A80ED45
:10896800026A3DF4BFAB95ED0C6A9DED115A25EEF8
:10897800866AA5EE076AB0EE675AA6EE265ABDEEDD
:10898800C56A16EE10EA16EE107AE645A8BF6746E5
:108998007145C8BF0F4606EE107AB8EEC66A042ABB
:1089A80080ED036A3DF49EAB95ED106A9DED125A79
:1089B80025EE866AA5EE076AB0EE675AA6EE265A35
:1089C800BDEEC56A16EE10EA16EE107AE645A8BFA7
:1089D80067467145C8BF0F4606EE107AB8EEC66AFC
:1089E800052A80ED046A3DF47DAB95ED146A9DED92
:1089F800135A25EE866AA5EE076AB0EE675AA6EE08
:108A0800265ABDEEC56A16EE10EA16EE107AE6454D
:108A1800A8BF67467145C8BF0F4606EE107AB8EE84
:108A2800C66A062A80ED056A3DF45CAB95ED186AC6
:108A38009DED145A25EE866AA5EE076AB0EE675AD0
:108A4800A6EE265ABDEEC56A16EE10EA16EE107AA4
:108A5800E645A8BF67467145C8BF0F4606EE107ABF
:108A6800B8EEC66A072A80ED066A3DF43BAB95ED81
:108A78001C6A9DED155A65EE865AE5EE075AE6EE34
:108A8800A57AFDEEE77A17EE902A9445A8BF94469A
:108A98008A42A8BF614607EE901AF8EEE77AC0ED61
:108AA800077AFDF71FBBBEF1010F7FF7D0AC07EEC9
:108AB800103AB8EEC77AC7EE876AB1EEE68AC8E41C
:108AC800BEF1010F40F32E8707EE103AB8EEC77AD1
:108AD800C7EE876AB1EEE68A032D13D04CB107EED4
:108AE800904AF8EEE77AF4EEC87AF1EE10FA01F15E
:108AF8008D80DBF8642002EB560292FBF6F2CBF88D
:108B0800242089E4B0EE480A29F05AFF00B2E5E7CC
:108B1800BEF1010F40F3028707EE103AB8EEC77AAC
:108B2800C7EE876AB1EEE68A032D13D04CB107EE83
:108B3800904AF8EEE77AF4EEC87AF1EE10FA01F10D
:108B48006580DBF8602002EB560292FBF6F2CBF868
:108B5800202046E4B0EE480A29F032FF00B2E5E7EB
:108B6800F7EE006AFDF78EBCF7EE006AFDF704BD6C
:108B780076EEC65AF0EE466ADDE58222FDF7E8BFDA
:108B8800DFED187AFDF7B0BF174BD3F800E0BEF958
:108B98003270FEF75EBAB6EE007AF4EEC75AF1EE1E
:108BA80010FA3FF72BAEFDF745B9D4F824614A0017
:108BB8003EB1551800EB850576786D78B542BCF462
:108BC8000FAC0A4400EB82000022C4F82401A4F888
:108BD8001022C4F81422FCF703BC00BFC0450020D3
:108BE800985B0020000002433451002095ED006A94
:108BF8009DED0E4AE34825EE866AFDEEE43AA4EEC2
:108C0800076AB0EE674AA6EE264A13EE901AB4EE4B
:108C1800C45AF1EE10FAB0EE446A88BFB0EE646A46
:108C2800BDEEC66A16EE10EA16EE107AE645A8BF43
:108C380067467145C8BF0F4606EE107AB8EEC66A99
:108C4800012A80ED006A3DF449AA95ED046A9DED7C
:108C58000F4A25EE866AA4EE076AB0EE674AA6EECA
:108C6800264AB4EEC45AF1EE10FAB0EE446A88BF50
:108C7800B0EE646ABDEEC66A16EE10EA16EE107A19
:108C8800E645A8BF67468E45B8BF0F4606EE107A80
:108C9800B8EEC66A022A80ED016A3DF41FAA95ED76
:108CA800086A9DED104A25EE866AA4EE076AB0EEC2
:108CB800674AA6EE264AB4EEC45AF1EE10FAB0EEB0
:108CC800446A88BFB0EE646ABDEEC66A16EE10EA62
:108CD80016EE107AE645A8BF67468E45B8BF0F4620
:108CE80006EE107AB8EEC66A032A80ED026A3DF4F1
:108CF800F5A995ED0C6A9DED114A25EE866AA4EE5C
:108D0800076AB0EE674AA6EE264AB4EEC45AF1EEF8
:108D180010FAB0EE446A88BFB0EE646ABDEEC66A67
:108D280016EE10EA16EE107AE645A8BF67468E459D
:108D3800B8BF0F4606EE107AB8EEC66A042A80ED70
:108D4800036A3DF4CBA995ED106A9DED124A25EE14
:108D5800866AA4EE076AB0EE674AA6EE264AB4EE23
:108D6800C45AF1EE10FAB0EE446A88BFB0EE646AF5
:108D7800BDEEC66A16EE10EA16EE107AE645A8BFF2
:108D880067468E45B8BF0F4606EE107AB8EEC66A3B
:108D9800052A80ED046A3DF4A1A995ED146A9DEDBC
:108DA800134A25EE866AA4EE076AB0EE674AA6EE75
:108DB800264AB4EEC45AF1EE10FAB0EE446A88BFFF
:108DC800B0EE646ABDEEC66A16EE10EA16EE107AC8
:108DD800E645A8BF67468E45B8BF0F4606EE107A2F
:108DE800B8EEC66A062A80ED056A3DF477A995EDC6
:108DF800186A9DED144A25EE866AA4EE076AB0EE5D
:108E0800674AA6EE264AB4EEC45AF1EE10FAB0EE5E
:108E1800446A88BFB0EE646ABDEEC66A16EE10EA10
:108E280016EE107AE645A8BF67468E45B8BF0F46CE
:108E380006EE107AB8EEC66A072A80ED066A3DF497
:108E48004DA995ED1C6A9DED154A65EE865AE7EE2B
:108E5800045AE6EEA57AB4EEE75AF1EE10FAC8BF66
:108E6800F0EE647AFDF72AB977EEC76AF0EE477A32
:108E780097E4454A4FEA89075FEA9C09384402EBC0
:108E8800C313274437D009F101094FEA091903EB45
:108E9800090803F1100200F1100607F1100112EDA4
:108EA800024A12ED035A12ED016A12ED047A56EDE8
:108EB800024A56ED035A56ED016A56ED047A64EEFD
:108EC800244A65EE255A66EE266A67EE277A10323E
:108ED800904541ED024A41ED035A41ED016A41EDE9
:108EE800047A06F1100601F11001D8D1A9F1100990
:108EF8004B4448444F441CF0030C3EF489AFB3EC98
:108F0800017AF0EC017A67EE277ABCF1010CE7EC04
:108F1800017AF4D1FEF77CBFBEF834309FED1B7A9E
:108F280007EE903AF8EEE77A194B67EE877AC3EDC9
:108F3800007AFDF725B9B7EE007A77EE677AF4EE96
:108F4800E75AF1EE10FA88BFF0EE675A63E407EECD
:108F5800905ADFED106AF8EEE77A66EEA65A9FEDB2
:108F68000E5A9FED0E6A9FED0E7AA5EE856A26EEE3
:108F7800A55AA5EE867AE5EE076A26EEA70AFFF758
:108F88006FB900BF985B0020B43800206F12833A95
:108F98001800002084F9223F92E741B99730083C35
:108FA80015A82ABE95ED006A9DED0E4ACC4825EE1F
:108FB800866AFDEEE43AA4EE076AB0EE674AA6EECA
:108FC800264A13EE907AB4EEC45AF1EE10FAB0EED7
:108FD800446A88BFB0EE646ABDEEC66A16EE10EA4F
:108FE80016EE101AE645A8BF61467745C8BF394650
:108FF80006EE101AB8EEC66A012A80ED006A3DF442
:10900800E0AF95ED046A9DED0F4A25EE866AA4EE61
:10901800076AB0EE674AA6EE264AB4EEC45AF1EEE5
:1090280010FAB0EE446A88BFB0EE646ABDEEC66A54
:1090380016EE10EA16EE101AE645A8BF6146BE45C0
:10904800B8BF394606EE101AB8EEC66A022A80ED95
:10905800016A3DF4B6AF95ED086A9DED104A25EE1C
:10906800866AA4EE076AB0EE674AA6EE264AB4EE10
:10907800C45AF1EE10FAB0EE446A88BFB0EE646AE2
:10908800BDEEC66A16EE10EA16EE101AE645A8BF3F
:109098006146BE45B8BF394606EE101AB8EEC66A34
:1090A800032A80ED026A3DF48CAF95ED0C6A9DEDC4
:1090B800114A25EE866AA4EE076AB0EE674AA6EE64
:1090C800264AB4EEC45AF1EE10FAB0EE446A88BFEC
:1090D800B0EE646ABDEEC66A16EE10EA16EE101A15
:1090E800E645A8BF6146BE45B8BF394606EE101A28
:1090F800B8EEC66A042A80ED036A3DF462AF95EDC6
:10910800106A9DED124A25EE866AA4EE076AB0EE53
:10911800674AA6EE264AB4EEC45AF1EE10FAB0EE4B
:10912800446A88BFB0EE646ABDEEC66A16EE10EAFD
:1091380016EE101AE645A8BF6146BE45B8BF3946C7
:1091480006EE101AB8EEC66A052A80ED046A3DF4E8
:1091580038AF95ED146A9DED134A25EE866AA4EEA4
:10916800076AB0EE674AA6EE264AB4EEC45AF1EE94
:1091780010FAB0EE446A88BFB0EE646ABDEEC66A03
:1091880016EE10EA16EE101AE645A8BF6146BE456F
:10919800B8BF394606EE101AB8EEC66A062A80ED40
:1091A800056A3DF40EAF95ED186A9DED144A25EE5B
:1091B800866AA4EE076AB0EE674AA6EE264AB4EEBF
:1091C800C45AF1EE10FAB0EE446A88BFB0EE646A91
:1091D800BDEEC66A16EE10EA16EE101AE645A8BFEE
:1091E8006146BE45B8BF394606EE101AB8EEC66AE3
:1091F800072A80ED066A3DF4E4AE95ED1C6A9DED04
:10920800154A65EE865AE7EE045AE6EEA57AB4EEFC
:10921800E75AF1EE10FAC8BFF0EE647AFDEEE77A8D
:1092280017EE901A8C45A8BF8C468F42D8BF674668
:1092380007EE907AF8EEE77AC0ED077AFDF7BEBE42
:1092480028494A69002A3CF499AA0A6813604B74B1
:10925800FCF794BA244DFDF70BB8D4F89C51079B42
:109268005D1BFFF775BA214B1B78DA0704D412F09F
:10927800F5FD002840F068851D4DD4F80C222B68B8
:109288009A423EF69AAA3B78012B3DF4A1A9194CC3
:109298002278002A3DF49CA90B2B19D801229A4068
:1092A80040F6030112EA01087EF4F5AF12F4C06F2C
:1092B8000ED0093B012B0BD8452024F0FDF8FF20E8
:1092C80024F0FAF80C4824F069F8404624F0F4F841
:1092D8000A4B2A685A600B233B70FEF7DCBF00BFBD
:1092E800985B002004730020044F0020AB5A002034
:1092F80024730020A75D0020D0680308485D002083
:109308000D9B002B00F07183E34D9DED0E4A95ED0A
:10931800006A089B25EE866AA4EE076AB0EE674AE3
:10932800A6EE264AB0EE446A33B1B4EE445AF1EEE2
:1093380010FAC8BFB0EE646AFDEEE44ABDEEC66A34
:1093480014EE907A16EE101A8F4214EE90EA00F39B
:10935800F3846145A8BF614606EE101ACF48B8EEFF
:10936800C66A012A80ED006A3CF4BCAE95ED046A39
:10937800DDED0F4A089B25EE866AA4EE876AF0EEBB
:10938800674AE6EE264AB0EE646A002B00F0CA840B
:10939800B4EEE45AF1EE10FA40F3C484394661455C
:1093A800A8BF614606EE101AB8EEC66A022A80ED1A
:1093B800016A3CF497AE95ED086ADDED104A089B0A
:1093C80025EE866AA4EE876AF0EE674AE6EE264A3C
:1093D800B0EE646A002B00F09B84B4EEE45AF1EE20
:1093E80010FA40F3958439466145A8BF614606EEF8
:1093F800101AB8EEC66A032A80ED026A3CF472AE0F
:1094080095ED0C6ADDED114A089B25EE866AA4EEFF
:10941800876AF0EE674AE6EE264AB0EE646A002BE9
:1094280000F06C84B4EEE45AF1EE10FA40F366846E
:1094380039466145A8BF614606EE101AB8EEC66AFD
:10944800042A80ED036A3CF44DAE95ED106ADDED1B
:10945800124A089B25EE866AA4EE876AF0EE674AF0
:10946800E6EE264AB0EE646A002B00F03D84B4EEC6
:10947800E45AF1EE10FA40F3378439466145A8BF43
:10948800614606EE101AB8EEC66A052A80ED046A2F
:109498003CF428AE95ED146ADDED134A089B25EEE1
:1094A800866AA4EE876AF0EE674AE6EE264AB0EED0
:1094B800646A002B00F00E84B4EEE45AF1EE10FA60
:1094C80040F3088439466145A8BF614606EE101A84
:1094D800B8EEC66A062A80ED056A3CF403AE95ED3F
:1094E800186ADDED144A089B25EE866AA4EE876AA1
:1094F800F0EE674AE6EE264AB0EE646A002B00F00A
:10950800E083B4EEE45AF1EE10FA40F3DA83394618
:109518006145A8BF614606EE101AB8EEC66A072A6A
:1095280080ED066A3CF4DEAD95ED1C6ADDED154A6A
:10953800089B65EE865AE4EE875AE5EEA67A002B7C
:1095480000F0B783F4EEC57AF1EE10FA40F1B1837A
:109558003A466245A8BF6246964607EE90EAF8EE9C
:10956800E77AC0ED077AFCF7BDBDD4F89C51079B9C
:109578005D1BFFF723B907EE905ADFED496A9FEDAF
:10958800497A84F80452F8EEE77A67EEA67A77EE1D
:10959800876ABDEEE66A16EE103A2033402B40F299
:1095A8009782DFED416A414BBDEEE77AC3ED016A70
:1095B80017EE103A2033402B00F260829FED3C7A80
:1095C800F4EEC77AF1EE10FA40F3CA83DFED395AA8
:1095D8009FED396A01E0F0EE477AF4EEC67AF1EED3
:1095E80010FA37EEE57AF6DCDFED347AB4EEE77A96
:1095F800F1EE10FA40F1B183DFED2E5A9FED306A9B
:1096080001E0B0EE677AB4EEC67AF1EE10FA77EEC2
:10961800257AF6D49FED237AF4EEC77AF1EE10FAA4
:1096280040F3E3829FED227A77EE677A67EEA75AD6
:109638009FED245A9FED246A9FED247AA5EE856A52
:1096480027EEA55AA5EE867AE5EE077AC4ED827A6A
:10965800FDF77ABD95ED000A0893069229F0B0F956
:109668001B49DFF870E0D1F8EC10DFF86CC0069AFF
:10967800ACF800008EFB013EC917C1EBAE1107EE36
:10968800901AF8EEE77A089BFDEEE77A17EE901A43
:10969800ACF80210FCF7F1BDC0450020985B002033
:1096A80035FA8E3CDB0FC93F00000000180000208F
:1096B800DB0F4940DB0FC940E4CB1641DB0F49C043
:1096C800E4CB16C192E741B99730083C15A82ABEE9
:1096D80064080020D34D6210EC4D002025EE866A08
:1096E800A5EE076AB0EE675AA6EE265ABDEEC56A21
:1096F80016EE100A814200F36C816045A8BF6046EF
:1097080006EE100A0A9BB8EEC66A002B00F0FF832B
:10971800DC48012A80ED006A3CF4E4AC95ED046A6B
:109728009DED0F5A25EE866AA5EE076AB0EE675AD8
:10973800A6EE265ABDEEC56A16EE107AB94200F3B7
:1097480046816745A8BF674606EE107A0A9BB8EEC1
:10975800C66A002B00F09883022A80ED016A3CF467
:10976800C1AC95ED086A9DED105A25EE866AA5EE06
:10977800076AB0EE675AA6EE265ABDEEC56A16EE1F
:10978800107AB94200F32D816745A8BF674606EEF7
:10979800107A0A9BB8EEC66A002B00F09383032A5E
:1097A80080ED026A3CF49EAC95ED0C6A9DED115A71
:1097B80025EE866AA5EE076AB0EE675AA6EE265A27
:1097C800BDEEC56A16EE107AB94200F30881674506
:1097D800A8BF674606EE107A0A9BB8EEC66A002B49
:1097E80000F06683042A80ED036A3CF47BAC95EDB7
:1097F800106A9DED125A25EE866AA5EE076AB0EE4C
:10980800675AA6EE265ABDEEC56A16EE107AB94218
:1098180000F3E3806745A8BF674606EE107A0A9B07
:10982800B8EEC66A002B00F0B182052A80ED046A02
:109838003CF458AC95ED146A9DED135A25EE866AF2
:10984800A5EE076AB0EE675AA6EE265ABDEEC56ABF
:1098580016EE107AB94200F3BE806745A8BF674686
:1098680006EE107A0A9BB8EEC66A002B00F0168343
:10987800062A80ED056A3CF435AC95ED186A9DED35
:10988800145A25EE866AA5EE076AB0EE675AA6EE68
:10989800265ABDEEC56A16EE107AB94200F3A380C7
:1098A8006745A8BF674606EE107A0A9BB8EEC66AF7
:1098B800002B00F07582072A80ED066A3CF412AC92
:1098C80095ED1C6A9DED155A65EE865AE7EE055A28
:1098D800E5EEA67AFDEEE77A17EE902A914203DCD0
:1098E8006245A8BF6246114607EE901A0A9BF8EE39
:1098F800E77A002B7FF435AE0C9B002B7FF431AE5A
:109908000B9B9E45B8BFF0EE647A2AE65E4A127851
:10991800032A00F015820022FEF7C8BD9FED5B8A7E
:10992800FFF702B99FED598AFFF7D6B89FED580A9D
:10993800DFF8708125EE800A29F042F8D4F8145136
:10994800A8F80600FDF717B9D4F89C51079B5D1BD2
:10995800FDF7C0BF4F49096811F080530A937EF4A0
:109968004DAFFEF742BF4C484C498046FEF73FBA20
:1099780007981CF0DFFEFDF713BF04F0F5F9059B0F
:10998800DFF8208193F800E0069B3178D4F8145171
:10999800C01AA8F80400FEF7E6BB04F0E5F9059B39
:1099A800DFF8008193F800E0069BC01AA8F80200CF
:1099B800FEF74FBB04F0D8F9059BDFF8E88093F871
:1099C80000E0069BC01AA8F80200FEF762BB0F462B
:1099D800BAE6084694E60F4642E70F461DE70F46EB
:1099E800F8E60F46D3E60F465DE70EA9BDEEE46A3A
:1099F80001EB820290462A48089A224D0A9B089455
:109A080016EE107A05E04145A5EC016A00F1100058
:109A180031D090ED006AB1EC014A25EE866AA7EED6
:109A2800046AB0EE674AA6EE864AB0EE446A32B1DE
:109A3800B4EE445AF1EE10FAC8BFB0EE646ABDEE57
:109A4800C64A06EE107A14EE104AA74206DC14EE57
:109A5800104A6445A8BF644606EE104AB8EEC66AC6
:109A6800002BD0D10C9C002CCDD10B9CA645B8BFA7
:109A7800B0EE646AC7E7089CFCF734BBDFED037AF5
:109A8800E4E500BF985B0020806D00200000000026
:109A98000000C842C85B0020343A00206023002040
:109AA800C0450020EC4D002092E741B99730083CB2
:109AB80015A82ABEE4CB1641DB0FC940E4CB16C17A
:109AC800DB0FC93FDB0F4940DB0FC9BFDB0F49C0C4
:109AD800F4EEC77AF1EE10FA40F355815FED0A5AB9
:109AE8001FED0C6A01E0F0EE476AF4EEC66AF1EE8B
:109AF80010FA36EEE57AF6DC5FED0C6AB4EEE67A3B
:109B0800F1EE10FA40F12F815FED155A1FED156A3D
:109B180001E0B0EE667AB4EEC67AF1EE10FA77EEAE
:109B2800256AF6D41FED1A7AF4EEC76AF1EE10FA38
:109B380040F3B3801FED1D7A77EE666A66EEA65A8B
:109B48001FED275A1FED276A1FED277AA5EE856AB4
:109B580026EEA55AA5EE867AE5EE076A23E51FEDFF
:109B6800277AF4EEC76AF1EE10FA40F38A815FEDC6
:109B78002E5A1FED306A01E0F0EE476AF4EEC66A2D
:109B8800F1EE10FA36EEE57AF6DC5FED306AB4EE07
:109B9800E67AF1EE10FA40F171815FED395A1FED66
:109BA800396A01E0B0EE667AB4EEC67AF1EE10FAE0
:109BB80077EE256AF6D41FED3E7AF4EEC76AF1EE29
:109BC80010FA05DD1FED417A77EE666AFFF7C5B931
:109BD8001FED437AF4EEC76AF1EE10FA44BF1FEDA9
:109BE800457A77EE666AFFF7B8B91FED497AF4EE61
:109BF800C77AF1EE10FA44BF1FED4C7A77EE677A18
:109C080014E5C84F07F18002FEF794BAA8F80600D9
:109C1800ABF8A860C34CFBF7EABBF8F79DFB00283C
:109C28003EF490ACFEF725BD802027F05BF808B124
:109C38000DF09AFF1DF030FEFEF78CBC402023F09B
:109C480049FB00287EF47EACD8F80030DFF814A376
:109C5800DFF814B34FF040090EE023F02DFCDBF8D9
:109C68000020D8F80030013A0133B9F10109CBF8E6
:109C78000020C8F8003079D01AF803301846002BB5
:109C8800EBD100234FF0FF32C8F800300423C8F8A6
:109C980004203B70AA78FDF786BD9FEDA37AF4EE09
:109CA800C76AF1EE10FA44BF9FEDA07A77EE666AB4
:109CB80044E7FDEEE77A17EE902ABA42FFF64DAC7C
:109CC80047E4BDEEC66A16EE101AB942BFF620ACDC
:109CD800394620E4BDEEC66A16EE101AB942BFF640
:109CE800F2AB3946FFF7F2BBBDEEC66A16EE101AA4
:109CF800B942BFF6C3AB3946FFF7C3BBBDEEC66A70
:109D080016EE101AB942BFF694AB3946FFF794BB6A
:109D1800BDEEC66A16EE101AB942BFF665AB3946F3
:109D2800FFF765BBBDEEC66A16EE101AB942BFF65C
:109D380036AB3946FFF736BB14EE901AFFF70CBB6B
:109D48000EF0C6FBFBF74CBB794B1B6803F59C5325
:109D58000833C4F80C32FDF730BDF0EE477A59E409
:109D6800B0EE677A40E4F0EE476ADBE61AF80330B3
:109D7800002B7EF4E7AB84E794F87831002B7BF472
:109D8800CBADFBF7B6BDB0EE667AB5E60C9B002B03
:109D98007FF44BAD0B9B9E45B8BFB0EE646A44E5BB
:109DA8000C9B002B7FF487AD0B9B9E45B8BFB0EE94
:109DB800646A80E55F4A604B10681B6898475F4B90
:109DC800D7ED006A93ED007A5D4BD3ED007A5D4BD9
:109DD80083ED020A5C4B67EE277A2B4427EEAC7AB8
:109DE800D3ED007A594B67EE277AF0EE665AEDEE1E
:109DF800A75A93ED006AB1EE467AB4EEE57AF1EE31
:109E080010FA08DCF4EEC65AF1EE10FA8CBFB0EE88
:109E1800467AB0EE657A4E4B1B78012B02D0192B8F
:109E28007BF4E4ACDFED4B7AF4EEE7DAF1EE10FA0E
:109E3800CCBF01230023FBF7E4BC474BD3ED007AEA
:109E4800B1EE677AF4EEC7DAF1EE10FA13D4F4EE55
:109E5800E7DAF1EE10FA88BFF0EE67DA3F4B87EDEC
:109E680000CA1B689342BBF6AFABFBF713BC0EF0FE
:109E780089FAFEF7F9BBF0EE47DAEFE7F0EE476A4A
:109E880099E6B0EE667A80E60C9B002B7FF464AC12
:109E98000B9B9E45B8BFB0EE646A5DE40C9B002B3B
:109EA8007FF4E6AC0B9B9E45B8BFB0EE646ADFE476
:109EB8000C9B002B7FF496AC0B9B9E45B8BFB0EE75
:109EC800646A8FE40C9B002B7FF469AC0B9B9E4566
:109ED800B8BFB0EE646A62E4132B05D1B0EE480A4D
:109EE80028F06EFD099B1880B0EE480ADBF80832AE
:109EF8001B489847059B1B78132BB0EE408A7CF4CF
:109F0800F2AE28F05DFD099B5880FCF7ECBE0C9B77
:109F1800002B7FF4FDAB0B9B9E45B8BFB0EE646A87
:109F2800FFF7F6BB60230020DB0FC9BFDB0F49C07A
:109F380024730020FC590020105A0020180000202B
:109F480050590020645B0020205A0020885A0020C5
:109F5800B458002000009642845A0020685A002015
:109F680034650020F03E03081C7000202DE9F04FF6
:109F78002DED068BA04BA14A1C7897B000F59C41AB
:109F8800203181460B911160002C00F0EA869C4A32
:109F98001268904240F283809A4A069216689A495B
:109FA8009A4A0591013C1C70994B049206F480561C
:109FB8000893002E40F08180964B1B78022B01F00D
:109FC8009481042B01F08381012B01F03781924B9E
:109FD8009945089B9B7800F29685002B40F0978561
:109FE8008E4B0793069B1E6816F4805740F08786B1
:109FF800DFF860A2049BB3F90610059B5D8BA942AC
:10A00800B4BF00250125864B1B6813F080535ED032
:10A01800079A127812F001025FD00598408C8842A6
:10A0280041F3B882002D5ED17E4C94F88C10002943
:10A0380059D17D487D49006890F82D0000240C60B6
:10A048004C608C607A4900284ED10870002A4FD0A5
:10A05800F0064DD5774A1278D10649D4002F47D15A
:10A06800002B45D1720243D4734B1B78002B02F0AE
:10A078001C82724B9B78002D42F09A823BB1704A49
:10A08800704B12681B689B1A002BC2F2708210205A
:10A09800644C0EF039FA012384F88D3028E0594BCE
:10A0A80006931E68594B584A049306F48056584B39
:10A0B80005920893002E3FF47FAF00215848F8F727
:10A0C800E5F800287FF478AF18F062FD74E77402B1
:10A0D8009ED4079A127802F00102524C002184F8AB
:10A0E8008C10002DA5D0524901200870002AAFD14C
:10A0F800554B1A78002A40F0BD800599049C488B7E
:10A10800B4F90070898BB4F90240B842B4BF802614
:10A11800002646F04003B942D8BF33469B0843F0B7
:10A128008006A042B8BF3346049F43F04006A142D0
:10A13800C8BF33469B08B7F90440B7F9066043F037
:10A148008007A042B8BF3B4643F04007A142C8BFC2
:10A158003B469B0843F08007324C8642C8BF3B46CB
:10A1680043F0400794F88EE08E42B8BF3B469E45C8
:10A1780001F04A84A4F8902084F892202E4984F8AB
:10A188008E300E78002E01F04B835F2B01F0BE83DA
:10A198006F2B01F0FD83079B1B78DE076AD494F8C8
:10A1A8009210002966D1B4F99030322B62DD94F810
:10A1B8008E200120572A84F892004DD0069B1B68F8
:10A1C8005D0741F199825A2A41F0968294F89430B9
:10A1D800002B42F0508194F8963083F0010384F804
:10A1E8009630002B42F0DC810C200EF08DF9174BD5
:10A1F800174D099341E000BF7043002048420020FA
:10A208006C430020B0650020BC710020506D002018
:10A218001C5300204C380020404B4C00AB5A002007
:10A22800C85B00207C25002034510020705B002092
:10A23800D82400203C6D002058010020805D0020BB
:10A2480024730020945A00205B4D002038510020D0
:10A258003051002028440020884B894A19684FF45F
:10A268007A73B3FBF1F3C3EB431103EB8103DB0018
:10A27800A2F8A830834B844D0993069B1B685F079F
:10A2880000F1B4860DF15009804E0A950022C9F8F4
:10A2980004203446149240F6330B4FF0190840F26C
:10A2A8008337049D02E00434544522D0A178E37832
:10A2B800994218FB0170F6D294F801E00EF1040EF1
:10A2C80018FB037135F91E305B45A8BF5B46B3F533
:10A2D800617FB8BF4FF461739842E4DA9942E2DBD8
:10A2E80021782729DFD848460434F7F7BFFF5445BB
:10A2F800DCD1674A0A9D1378664A99E8030082E828
:10A308000300002B40F0F085634B1A78002A00F018
:10A318006A8501215F48F7F7B9FF002840F0E78216
:10A32800089BDB78002B40F0E2825C4B0A932B8879
:10A338001FB227F001071FFA87F84345A5F80080E8
:10A3480001F00280564F4FF002090E204FF0140A18
:10A358004FF0FF0B87F8009087F801A087F802B04C
:10A368000EF0D2F849464B48B5F80080F7F78EFF53
:10A37800002841F09A8228F002039BB243452B80C3
:10A388000BD0474B02201421FF2218700E20597061
:10A398009A700EF0B9F8B5F80080424B424A197825
:10A3A80050680B9318F0030F08BF81F00201C1F346
:10A3B80040010C921BF070FD24213648F7F766FF28
:10A3C80030B9079A13785F0744BF23F0040313706A
:10A3D8000A9B1B6813F00A0F11D006212D48F7F7C6
:10A3E80055FF002801F0AD802B88580641F12582E1
:10A3F80007212848F7F74AFF002840F0C8870C21B2
:10A408002448F7F743FF2A88002800F0508342F4D5
:10A4180080739A422B8009D0214B022214211A7092
:10A428000E20FF2259709A700EF06EF81F4B1B78A1
:10A43800082B00F048830E2B00F04583069BD3F8C9
:10A44800008018F4806F6BD0194B1B79002B00F03B
:10A45800308214210F48F7F719FF002840F02E82A8
:10A4680021F0FEFE01200DF057FF002855D0DFF83F
:10A4780044A000274FF0CC0BA14620E0A0650020A7
:10A48800286300203851002030510020D843002094
:10A49800D4670020C85B0020BC480020DC500020A6
:10A4A80090350020EC720020F0720020A45D00209E
:10A4B800F44E00201C7C0020DFB2022F2CD80BFBAE
:10A4C80007F87B1C5AF80840002CF5D1032290F9B4
:10A4D800023002940192C278E24951F82220009297
:10A4E80018462246234601210DF056FB034607EB8A
:10A4F800470000EB00100A9353B121460AEB800095
:10A50800CC2229F01AFA0A9B4AF808300137FFB220
:10A5180024F016FC0028D0D14C46069BD3F80080C6
:10A52800079B93F800A0D04B1AF0010A00F0418273
:10A5380001221A70099B04991B68B1F906105A89FF
:10A54800CA4801279142077080F21982C84B4FF020
:10A558007E521A60059BC74FB3F81890049B97F971
:10A568000420B3F90030387897F801C0002AA3EB2B
:10A57800090714BF01224FF0FF32002FB8BF7F42F6
:10A58800B7F5FA7FA8BF4FF4FA77B84280F2F481A2
:10A598003F1A07EE907AF8EEE77AB74F4B45C7EDCA
:10A5A800007A03DAF1EE677AC7ED007A049BB3F913
:10A5B80002E0AEEB0903002BB8BF5B42B3F5FA7FAC
:10A5C800A8BF4FF4FA73984280F2D3811B1A07EEA2
:10A5D800903AF8EEE77AF145C7ED017A03DDF1EE3E
:10A5E800677AC7ED017A049BB3F90400A0EB09036D
:10A5F800002BB8BF5B42B3F5FA7FA8BF4FF4FA73DC
:10A608006345CCBFA3EB0C03002302FB03F207EE68
:10A61800902AF8EEE77A4845C7ED027ABCBFF1EE1A
:10A62800677AC7ED027A18F4805800F07F81B1F597
:10A63800FA6F924BA8BF4FF4FA61B1F57A7F1A7896
:10A64800B8BF4FF47A71A1F57A71002A41F01D81E3
:10A658008B4ADFF844E282FB0130CB17C3EB60136F
:10A66800581C6FF0630C3EF910003EF913E00CFB28
:10A678000313A0EB0E0003FB00F382FB0312DB17AE
:10A68800C3EB62139E440FFA8EFE07EE90EAB8EE13
:10A69800E78A87ED038AB8F1000F40F066842B88BB
:10A6A8005A0640F1FB807749774A91ED018AD2ED4D
:10A6B800019A92ED026A91ED034A92ED030A91ED37
:10A6C800029A92ED007AD1ED005AD7ED011A97ED72
:10A6D800002A6E4A6E4938EE445A79EEC63A77EE49
:10A6E800007A65EE233A75EEC96A75EE890A37EE87
:10A6F800401A66EEA76AB0EE633AA0EE813A13F00C
:10A708000303B0EE665A78EE044A79EE867AA0EE34
:10A71800815AF0EE638AA4EEA73AD4EEA78AA4EE93
:10A72800E75A33EE263AF0EE687AF0EE674AF6EE2C
:10A73800008A35EE88AAE0EEC14A28EEC33A35EE23
:10A74800635A77EE293A77EEE67AAAEE233A25EEAF
:10A75800285A76EE403A34EE49AAE0EE817A74EE51
:10A76800A64AAAEE235A34EE094A37EE697A64EE0D
:10A77800A84A63EE036AE4EE074A75EEC85A36EE55
:10A78800006A67EEA87AB0EE667A95EE057AE5EE8D
:10A79800056AE5EE867AB1EE648AF0EE665AF0EE66
:10A7A800476AB1EE674AE8EE246A63EE270A67EE65
:10A7B800A43AE4EE275AB1EE450AB0EE609AB0EE3C
:10A7C800631AA4EE277A23EE244AE7EEA76AA5EED9
:10A7D800249AA0EE031AE8EE245AB0EE448A31EE29
:10A7E800A16AE0EE240AA5EE278A66EEA16A72EE57
:10A7F800028AE5EE033A61EE211A26EE096AA4EE12
:10A80800A47AA0EE274A0CBFD7ED022ADFED212A51
:10A8180082ED005AA2EE256AE8EEA06AE2EE081A76
:10A8280073EEA33A27EE227A34EE044AF0EE005A89
:10A83800E3EEA26AA4EE226AA1EEA57AC7ED016A48
:10A84800C1ED366A81ED356A87ED006A81ED377AA8
:10A8580082ED013AC2ED027AC2ED034AF3B987EDFF
:10A86800027A1BE03C630308AC5A00201025002044
:10A878008C240020585D0020044F00203C2A002032
:10A888001F85EB518801002010010020480100209D
:10A898007C2500200000000068460020BAF1000F67
:10A8A80040F0248111F094FE17B0BDEC068BBDE892
:10A8B800F08F079B1B78D9077FF5D2AD4FF40F7047
:10A8C80026F010FA00283FF428AE0DF04DF94FF4A9
:10A8D8000F7026F0B1F900283FF41FAE0DF044F9CF
:10A8E8004FF40F7026F0A8F90028EED115E69A4B20
:10A8F8000A931B689B077FF51AADB5F8008018F01E
:10A90800010F7FF438AD48F0010398452B803FF4E0
:10A9180032AD924B022214211A700E20FF22597078
:10A928009A700DF0F1FDB5F8008024E5059B5A8B6F
:10A938009142C0F20685B1F5FA6FD4BFC2EB0101AE
:10A94800C2F5FA614FF47A7303FB01F18448037886
:10A95800C2F5FA62B1FBF2F1002B3FF479AE43780D
:10A96800804A01FB03F182FB0123C917C1EB631184
:10A978006EE6DFED7D7A2EE6DFED7B7A0DE6B1F54A
:10A98800FA6F80F2D784187A8B1A03FB00F3C2F5AA
:10A99800FA6293FBF2F3C3F1640307EE903AF8EE20
:10A9A800E77A9FED727A724B67EE877AC3ED007A89
:10A9B800D0E51B780693002B7FF4BCAD6D4A126876
:10A9C800002A3FF4B7AD6C4A079212F8030CDFF87F
:10A9D800E0B11146D71E11F06FFB9BF80090079A63
:10A9E800002800F03086069BB9F1000F53D107F11B
:10A9F8000801787911F060FB002841F026855F494D
:10AA0800B87A11F059FB002800F03086B9F1020F2E
:10AA180041F017855A49F87B11F04EFB002841F0A8
:10AA28000C855849387D11F047FB002800F0308626
:10AA3800B9F1040F41F0FD845349787E11F03CFBD5
:10AA4800002841F0F2845149B87F11F035FB002805
:10AA580000F03086B9F1060F41F0E3844C4997F8CD
:10AA6800230011F029FB002841F0D784494997F8C1
:10AA7800280011F021FB002800F03086B9F1080FFA
:10AA880041F0C784444997F82D0011F015FB0028C0
:10AA98003FF450AD09231A4602EB820217443F4A9D
:10AAA8007878B9788BF800301070517042E522F44C
:10AAB80080739BB29A422B807FF4AEAC384B1B78E4
:10AAC800082B7FF4B8AC2A8822F040039BB29A4244
:10AAD8002B803FF4B3AC214B022214211A700E20B4
:10AAE800FF2259709A700DF00FFDA7E40B9B19789F
:10AAF8000C9B01F0010118681BF0CEF917B0BDECF2
:10AB0800068BBDE8F08F13B9089A01239370254B83
:10AB1800089A1D7892F8214007931B2011F004FB36
:10AB2800012C05F00108814600F0088705F00205B0
:10AB3800089A1D4E92F82030DFF878A01B4F09952F
:10AB48009346052B00F29E87DFE813F0BE00B400A1
:10AB58003600FC00FE00F100DC500020903500209B
:10AB68003C2A00201F85EB51000000000AD7233C37
:10AB78008C240020B05A00203A35002044350020AB
:10AB8800493500204E350020533500205835002027
:10AB98005D3500206235002067350020B45A00205A
:10ABA800A45D0020AB5A0020604600202C510020F4
:10ABB8002000002058010020012C04BF05238BF839
:10ABC8002030B8F1000F12D0059B3088B3F9181067
:10ABD8000022134661F30F0260F31F4261F30F0373
:10ABE800049861F31F430360032342600993BF4D38
:10ABF800DBF814102A68914280F0028647F230513F
:10AC08000322CBF81C108BF82020022006F0F6FC5B
:10AC180017F0BEFF2968DBF81C200A440421CBF892
:10AC280018208BF82010012C40F07D872A68DBF86B
:10AC38001810914280F026879AF8000020B911F088
:10AC480073FA002840F01E873A6822F002023A6040
:10AC58002A687388642101FB03234FF48060002273
:10AC6800CBF810308BF820208BF8032006F096FCE8
:10AC78009BF8203065E711F05DFA012807D19B4D5C
:10AC880072882B68642101FB0233CBF81030B9F1CC
:10AC9800000F02D0B379002B4BD1012C00F0F286C3
:10ACA800924DDBF810102A689142C0F031870123D9
:10ACB8008BF82030012C3AD0F379012B46D011F0D3
:10ACC800B9F99BF820303CE7B8F1000FD3D1099DC2
:10ACD8004FF48060B9F1000F00F0568306F076FC5F
:10ACE800089A00231361002D3FF47CA928460DF033
:10ACF8000BFC069B1E6816F480573FF479A91D21AA
:10AD08007B48F7F7C3FA00287FF472A9794B03F15F
:10AD1800500A03E004339A4500F0BA861A78262AC6
:10AD2800F8D19978DA789142F4D2FFF763B96F4D88
:10AD38008EE711F07FF903224FF47A738BF8202005
:10AD4800CBF81C30694D60E7684D6CE711F072F97B
:10AD5800032240F6B8338BF82020CBF81C30634D23
:10AD680053E7654F3B78002B01F06382634BDFF8B4
:10AD78009881DFF898B1DFF898A1059345465E46BB
:10AD8800049099460EE019F804109847032C28DC23
:10AD980088B93B782AF8020F01349C4205F1040572
:10ADA80080F24981072CE1B23046DBF80430EADD55
:10ADB800984700B2EDE738F824206B88801A4FF4E2
:10ADC8007A719B1A01FB00F040F6CA0290FBF3F07F
:10ADD8000844904240F2EE23A8BF10469842B8BFFC
:10ADE800184600B2D5E7DFF82C91DFF82CA1444FC4
:10ADF8000A9209F15A084FF0010B494619F8010C5B
:10AE080011F05AF900B399F8040099F8023099F84A
:10AE180003E000EB400107EB8101013BD1F8A020E2
:10AE280003EB4303534493420ED097F8CC20C1F868
:10AE3800A0300BFA00F022EA00000A9B81F89CE09F
:10AE4800C1F8A43087F8CC0009F10609C145D4D16E
:10AE58002C4B264A1B780A93099BDFF8C0A012687E
:10AE68001B680B93AAF19C094FF0000B9046DAF887
:10AE7800043083B31F7877B3DAF80820A8EB02020E
:10AE8800002A0CDB99F8CC20012101FA0BF122EA07
:10AE9800010208F5FA7189F8CC20CAF808100A9A54
:10AEA800CAB19AF8002059780432D2B2002940F089
:10AEB800B58305990498098B30F9122001F1C8006F
:10AEC800824240F3F78599F8CC109A7841FA0BF34F
:10AED800D80740F181860BF1010BBBF1040F0AF191
:10AEE8000C0AC4D1FFF715BA024B1DE024730020E9
:10AEF800C85B0020D84300209C440020BC7100207F
:10AF08007C250020ED520020B0440020344200206F
:10AF18007A250020513400202441030818260020F7
:10AF280004339C423FF4F0A919782329F8D1987882
:10AF3800DA789042F4D2AD48F7F7A8F900283FF440
:10AF4800E3A9AB4B1B6813F4003341F001820022E4
:10AF5800A84B1046995C142902F10C0201F0FE80FE
:10AF680001301828F6D1FFF7CFB91D219F48F7F710
:10AF78008DF928B100F060BD0436B4423FF48FABC0
:10AF880031782629F8D1B278F3789A42F4D2089B1E
:10AF9800DB78002B7FF483AB9448F7F777F9DFED84
:10AFA800967A002801F0498138EE678A934A9449D5
:10AFB800FDEEC87ACDED047ABDF910301B0382FB93
:10AFC8000302DB17C3EBA212C9F57A731BB203FBAA
:10AFD80002F343F30F334B4407EE903AF8EEE77A67
:10AFE8000123C7ED037A0B70FFF759BB854C94F822
:10AFF80096305BB1079B1B78DE0707D5049BB3F936
:10B008000620059B5B8B9A4200F3D885112177486F
:10B01800F7F73CF9002800F0AB8294F89A302BB986
:10B0280094F8943013B93223A4F89830012384F8A3
:10B038009A30FFF727B9DDF81090734A06926F49E6
:10B04800126842F2010AA1FB091B12EA0A0A4FEA36
:10B058009B1B00F08A826D4D6D486E4C6E492E78B0
:10B068000078267008701EB16B490E7886F00106CC
:10B07800644C0F2184F82410002B00F0E683059D12
:10B08800664BB5F826C0B5F824E0059D1093184620
:10B098002D8B0078624B129594F825500995614DD7
:10B0A8000495A3FB00535B0803EB4303C31ADBB20D
:10B0B8000F90CDF834C002F480520C9304F12800AC
:10B0C8000BF59673CDF8449097F80080DDF824903E
:10B0D800DFF860C10994534C0E91139200210A9332
:10B0E8000896CDF81CE0089B002B00F02B83099BE9
:10B0F800079D33F911201FFA82FEAE454FEA41033E
:10B1080003D30D9DAE4540F262835CF82120934540
:10B1180080F02283E25EBAF1000F40F037830131FC
:10B128004145E25200F10600DDDB0E9A099C3E4BD8
:10B1380084F824200F2A49460CBF01220022DDF89A
:10B14800449084F825101A7000F08683374B3049F4
:10B15800314ADFF8E4B008931C46042001230B7041
:10B16800137006F04BFADBF80030A1686268E36000
:10B178005B1A934284BF002384F82130069B3C78F5
:10B188001E68002C01F07A80059A294DB2F824E057
:10B19800178B244916F48056284640F09983324686
:10B1A8000EE0437803EB830303EB830303F2EE2300
:10B1B8009BB20132A24221F8023B00F102000ED0FC
:10B1C80015F81230002B00F00683022BE9D001326B
:10B1D8000B8821F8023BA24200F10200F0D1109A3C
:10B1E800137801331370FEF7E4BE00BFC85B00207C
:10B1F800443400208054030800007A44D34D621080
:10B20800042500207C250020B06500201042002085
:10B2180000010020ED520020010100208D43002094
:10B22800ABAAAAAA506D0020D05B00201C530020B6
:10B23800E44400209043002024730020D84CD4F824
:10B248008830A9EB0303002BFEF6C1AED54AD64BD6
:10B25800527C059933F812308A7DDFEDD46A9FED70
:10B26800D46AC97D9BB207EE102A07EE903AB8EE71
:10B27800C77AF8EEE77A27EE267A67EE867A0B9A8F
:10B28800C4F88820C7EE876A40F2FF32FCEEE67AFF
:10B29800CDED077ABDF81C30934228BF134609B19B
:10B2A800D31A9BB2C348C44D0178C44C35F8116019
:10B2B800226825F81130921B13440131C04D2360D8
:10B2C80001F00F021B0902702B80FEF780BE02F00E
:10B2D8004BFDBC4BBC4A1B68C31A93427EF777AE42
:10B2E800B74B00221A80FEF772BE059A0499537D67
:10B2F800D27D013B31F913301AB1C3F53B630833F2
:10B308001BB2A3F57A7307EE903A9FEDB07AAC4A78
:10B31800F8EEE77A40F2FF3167EE877AFCEEE77ADB
:10B32800CDED077ABDF81C308B4228BF0B46138041
:10B33800FEF74DBE1B7AC3F1640307EE903AFFF7A0
:10B348002EBB4146FFF702BB0221A148F6F79EFF3C
:10B3580000283FF410A82F8018F0020F7FF41DA8D2
:10B3680048F0020343452B803FF417A8994B02226B
:10B3780014211A700E20FF2259709A700DF0C4F82B
:10B38800B5F80080FFF709B806F008F9A8E4924A72
:10B39800B2F90030002BB8BF5B42B3F5E17FBFF6CE
:10B3A8002EA8B2F90230002BB8BF5B42B3F5E17F9B
:10B3B800BFF625A8894B93ED096AD3ED076A93ED8B
:10B3C800057AD3ED037A76EE866A77EE877A76EE9B
:10B3D800A66AB7EE007A37EE666A77EEA77AB0EE1D
:10B3E800C66AF0EEE75AB4EEE56AF1EE10FAB4BFB9
:10B3F800B0EE655AB0EE465AB5EE405AF1EE10FA84
:10B4080040F0AD839FED767AB4EEE56AF1EE10FA7E
:10B4180044BF9FED746A36EE477AB7EE006AF4EEE1
:10B42800C66AF1EE10FAC8BFDFED6F6AF5EEC07AB2
:10B43800C8BF36EEC77AF1EE10FA48BFB1EE477AC8
:10B44800F6EE007A27EE677ADFED667A77EE276AFE
:10B45800BDEEE66A16EE103A2033402B40F23686EF
:10B46800DFED626A624ADFED617AC2ED006AFDEEE5
:10B47800C76AC2ED017A16EE903A2033402BC2ED2E
:10B48800027A49D8DFED587AB4EEE77AF1EE10FA8D
:10B4980040F3ED879FED576ADFED576A01E0B0EEA4
:10B4A800677AB4EEE67AF1EE10FA77EE467AF6DCD1
:10B4B8009FED527AF4EEC77AF1EE10FA40F1EF8779
:10B4C8009FED4C6ADFED4E6A01E0F0EE477AF4EE4C
:10B4D800E67AF1EE10FA37EE867AF6D4DFED417AA5
:10B4E800B4EEE77AF1EE10FA40F37486DFED3E7AB7
:10B4F80037EEC77A27EE076ADFED425ADFED426A78
:10B50800DFED427AE6EE256A67EE065AE6EE267A1F
:10B51800A5EEA77AF0EE477A3D4BC2ED037A1A689A
:10B5280012F4003240F04E863A4B1046995C0A29D4
:10B5380002F10C0200F04B8501301828F6D1FEF715
:10B548005EBF2A8822F040039BB29A422B803EF4C9
:10B558004FAF204B022214211A700E20FF2259707F
:10B568009A700CF0D1FFFEF743BF2B490E787AE5AD
:10B5780094F89430002B3EF485AE079B1B7813F0AB
:10B5880001037EF47FAE012284F8943084F895207C
:10B59800FEF778BE024C012184F88C10FEF7A3BD9B
:10B5A8007C250020C4720020E47200200000C842FC
:10B5B800000080444D3800205438002050380020C6
:10B5C800446D00205023002060E316006F12833F73
:10B5D800C85B002090350020E050002020010020AA
:10B5E800A7DFA834DB0FC93FDB0F4940000000008C
:10B5F80088010020DB0FC940E4CB1641DB0F49C0AE
:10B60800E4CB16C192E741B99730083C15A82ABE89
:10B618004434002080540308ED520020012900F032
:10B62800FD8499F8CC20012303FA0BF30BF1010BED
:10B638001343BBF1040F89F8CC300AF10C0A7FF4EC
:10B6480016ACFEF766BE511D787910F035FD00285E
:10B658003FF4D5A9B9F1010F40F0F78607F10D01C4
:10B66800B87A10F029FD002840F0EB86B549F87B40
:10B6780010F022FD00283FF4D4A9B9F1030F40F0DF
:10B68800DC86B149387D10F017FD002840F0D186DE
:10B69800AE49787E10F010FD00283FF4D4A9B9F126
:10B6A800050F40F0C286AA49B87F10F005FD0028B2
:10B6B80040F0B786A74997F8230010F0FDFC002852
:10B6C8003FF4D4A9B9F1070F40F0A786A24997F82B
:10B6D800280010F0F1FC002840F09B869F4997F85D
:10B6E8002D0010F0E9FC00283EF424AFB9F1090F51
:10B6F8003EF420AFFFF7CEB95D2A00F05F855B2AE4
:10B7080000F06F825E2A00F01086562A00F011863B
:10B71800972A00F03386A72A00F0FD85904D2B88E4
:10B728009B0740F0AF85A2F1B703072B00F28B828D
:10B73800DFE813F07D028902890289027102890219
:10B7480065026502079B002B3FD05CF821209345DA
:10B758004FEA4103FFF4DEAC824A824DD25C05EB2E
:10B76800030E002A00F09480022A47D19EF8012097
:10B7780002EB820202EB820202F2EE2292B203296B
:10B7880033DD12B2BAF1000F3FF4C9AC0C9D20F8BA
:10B798001520B9F1000F03D10F9D022D7FF6BFAC24
:10B7A800B0F802900288B0F804E04A4496446E4A21
:10B7B8000FFA8EFE82FB0E526C4DA2EBEE7225F84C
:10B7C80003E012B24FF00109A9E41A464B000A9DA2
:10B7D8004CF821509FE4D3B2022B04D9032B7FF4F9
:10B7E800F6AC7346E5E43B46E3E4012505FA01FEC1
:10B7F8000E9D25EA0E0512B20E958CE4E25ABEE7BC
:10B808005B4A1278002A7FF4F9A9B8F1000F3FF4D7
:10B81800F5A9012C40F036819BF82030FFF791B94B
:10B8280031465448F6F732FD002800F0C98084F804
:10B83800936017F0DDFDFEF7AEBC43F04002934283
:10B848002A807FF486AEFEF7D3BD4B4B4B4A10924D
:10B8580001221A704A4B04931B214648F6F716FD3D
:10B8680000287FF473AC474BDFF820B108931946E2
:10B87800DBF80030CA688B609B1AC82B00F2308551
:10B88800069B1E6806F48056A9E45B78FFF768B843
:10B89800CAB2022A40F2B683032AAFD1129A139D84
:10B8A800079E002D08BF324669E728F0010292B2D0
:10B8B80042452A803FF450AD0E2087F8009087F863
:10B8C80001A087F802B00CF01FFEB5F8008043E530
:10B8D80000220FE0437803EB830303EB830303F2B7
:10B8E800EE239BB20132A24221F8023B00F1020092
:10B8F8003FF475AC15F812301BB1022BEAD00B8857
:10B90800F0E7D3B2032BFAD83B46EBE7B2F5FA7F60
:10B91800FEF6B0AC94F89230002B7EF4ABAC079BEB
:10B928001B7801210B4084F8921000F0B48317F0C3
:10B938002FF9154B0A4D0993FEF79FBC0025FFF719
:10B94800F7B800BF493500204E3500205335002098
:10B95800583500205D35002062350020673500200D
:10B9680030510020E444002056555555EC25002060
:10B97800C8240020C85B0020D05B00208D43002035
:10B98800506D00201C5300203851002024730020E3
:10B99800B2F5FA7FFEF66EAC94F89230002B7EF486
:10B9A80069AC079A12780121D70784F8921000F140
:10B9B8001E8417F01DFDBF4BBF4D0993FEF75DBCFC
:10B9C800079BBE4A1B781060DB077EF5E8ABBC4BD3
:10B9D8001B78002B3EF44EAC089BDB78002B7EF4E2
:10B9E80049AC94F893300133DBB2032B84F89330DD
:10B9F8007EF640ACB34B5B7813B9002D7EF43AACBD
:10BA080017F0C6F8FEF7C7BBAF4AB0491068B4F9DB
:10BA18009020C66981FB06018911F617701A00F596
:10BA2800FF407F3082423EF7A9AB891B0A4412B21D
:10BA3800A4F89020FEF7A2BB089BDB78002B7FF4CC
:10BA48009FAADFEDA37AA14938EE678AC9F5FA63A0
:10BA5800FDEEC87A1BB2CDED047ABDF910201203B1
:10BA680081FB0201D217C2EBA11203FB02F343F3DD
:10BA78000F334B4407EE903AB8EEE78A87ED038A16
:10BA8800FFF77EBA099D002D3EF4ACAAFFF72EB948
:10BA9800904A059BD588049A1B8BB2F906105A1B4D
:10BAA800914240F388802B449942B4BF0025012578
:10BAB800FEF7A9BAC8398A4242DA99F8CC109A78BE
:10BAC80041FA0BF3D9073FF506AA524201200C921E
:10BAD8000CF000FE7B1E0C9A162B00F27C81DFE82E
:10BAE80013F0FE011202E601370226024B02D101D1
:10BAF800BC01A70192017D017A0137026C014B025A
:10BB0800D101BC01570143012F0160021901D40082
:10BB180010F090FA032140F6B8328BF82010CBF8D9
:10BB28001C20FFF772B8AB460899DBF80020CB69F8
:10BB3800099D13448B61002D3EF454AAFFF7D6B833
:10BB480099F8CC30012202FA0BF223EA020308F535
:10BB5800FA7289F8CC30CAF80820FFF7BCB9B4EEFD
:10BB6800E56AF1EE10FA8CBFB0EE654AB0EE464ACF
:10BB7800C4EE054A9FED582A9FED585ADFED581A32
:10BB8800DFED582A9FED583ADFED583A9FED584AB5
:10BB9800A4EE825AE4EEE12AA4EE857AA4EEA23A53
:10BBA800B0EE475AB0EE637AA4EE837AA4EE874AE1
:10BBB80084EE057A28E40125FEF725BA00214D48D0
:10BBC800F6F764FB00287FF421AA322384F8960054
:10BBD800A4F89830FFF71ABA002A0CBF01200220F7
:10BBE80075E7454B012202204449454C0B60314B17
:10BBF8002270314D09930CF06DFDFEF73EBB2D4AC6
:10BC08003F4B099211463F4A0A6002225A7010F0CF
:10BC1800EFFAFEF732BB274A394B099211463A4AE6
:10BC28000A6000225A7010F0E3FAFEF726BB214A98
:10BC3800334B09921146354A0A6001225A7010F0B6
:10BC4800D7FAFEF71ABB9E2A00F06D849D2A00F0F1
:10BC58006284AE2A00F05784AD2A00F04C84EF2AA3
:10BC680000F04684FD2A00F04084FB2A00F02D8471
:10BC7800FE2A00F06084F72A00F08F847B2A00F007
:10BC8800EC830C4B0993FEF7F8BAD9F8D000204B97
:10BC980090F836109B7811446429A8BF642121EAE2
:10BCA800E17180F83610002B40F0698416F064F9D1
:10BCB800B7E400BF3851002030510020985A0020C6
:10BCC800ED520020805D00208C6F0020D34D621063
:10BCD80000007A444846002099FB243F69A2163E9A
:10BCE80039094E3DE3B59E3E88FA163E45FE7F3F34
:10BCF800A7DFA834C85B0020AE5E002034510020C6
:10BD0800B8720020845F00206C5F0020785F0020FC
:10BD18003E6D0020D9F8D000BC4B90F837109B78C6
:10BD28001144FE29A8BFFE2121EAE17180F83710ED
:10BD3800002BBBD0162010F041FAD9F8D000B5E797
:10BD4800D9F8D000B14B81781144C829A8BFC821BF
:10BD580021EAE17181709B78002BA7D0142010F0A4
:10BD68002DFAD9F8D000A1E7D9F8D000A74B41782F
:10BD78001144C829A8BFC82121EAE17141709B7804
:10BD8800002B93D0132010F019FAD9F8D0008DE7C2
:10BD9800D9F8D0009D4B01781144C829A8BFC82103
:10BDA80021EAE17101709B78002B3FF47FAF1220EC
:10BDB80010F004FAD9F8D00078E7944B0B989B78E8
:10BDC800417911446429A8BF642121EAE1714171D4
:10BDD800002B40F0C583D9F8D00067E7D9F8D00028
:10BDE8008A4B017A9B781144C829A8BFC82121EA47
:10BDF800E1710172002B3FF459AF0B2010F0DEF90E
:10BE0800D9F8D00052E7D9F8D000804BC1799B7897
:10BE18001144C829A8BFC82121EAE171C171002BCA
:10BE28003FF444AF0A2010F0C9F9D9F8D0003DE733
:10BE3800D9F8D000754B81799B781144C829A8BFDF
:10BE4800C82121EAE1718171002B3FF42FAF09204D
:10BE580010F0B4F9D9F8D00028E7D9F8D0006B4B26
:10BE6800417993F802E01144C829A8BFC82121EA02
:10BE7800E1714171BEF1000F40F06083112F7FF432
:10BE880062AF13E7D9F8D000604B017993F802E06C
:10BE98001144C829A8BFC82121EAE1710171BEF186
:10BEA800000F40F09183102F7FF461AFFEE60B99ED
:10BEB800564B0F790C931744642FA8BF642727EAC1
:10BEC800E7770F7110F094F90C9B9B78002B82D0C8
:10BED8000320394610F072F9D9F8D000E6E60B983D
:10BEE8004A4B01781144FA29A8BFFA2121EAE171E5
:10BEF80001709B78002B3FF46EAF012010F05EF9C3
:10BF0800D9F8D000D2E60B98404B817811446429C7
:10BF1800A8BF642121EAE17181709B78002B3FF46E
:10BF28005AAF022010F04AF9D9F8D000BEE60B98B3
:10BF3800364BC1799B78114481F30801C171002BFC
:10BF48003FF449AF052010F039F9D9F8D000ADE633
:10BF58000B982E4B817993F802E011446429A8BF0D
:10BF6800642121EAE1718171BEF1000F40F0F08295
:10BF78000D2F7FF423AF2EE7D9F8D000234BC178DB
:10BF880093F802E01144C829A8BFC82121EAE17149
:10BF9800C170BEF1000F40F0F6820F2F7FF4FBAEA8
:10BFA80084E60B98194B41781144B1F5967FA8BFE8
:10BFB8004FF4967121EAE17141709B78002B3FF4B0
:10BFC8000AAF152010F0FAF8D9F8D0006EE610493B
:10BFD800D1F800E04200BEF1000F08D0171803EBBB
:10BFE80087079EF801E07F787745BEF408AA1044D9
:10BFF800084F094A03EB800300200B60388010606B
:10C00800FEF7FDB9129AFFF7BABB00BF3E6D0020DC
:10C0180084240020702500207425002004999B7832
:10C0280031F91220B2F5617F4FF4966191FBF3F379
:10C03800C0F2E48040F633019142A8BF11460C2FAC
:10C04800A1F5617191FBF3F100F0DE81182F7FF407
:10C05800E8AAC9B2C8290B46A8BFC823D9F8D02076
:10C06800D77DD8B2B8423FF4DCAADF1BC84BD075E5
:10C0780048BF0737FF109B780137FFB23BB9002F45
:10C088003FF4CFAA38460CF025FBFFF7CABA1820B0
:10C0980010F094F8F3E7BF49096811F4003140F053
:10C0A8006081BD4B08465D5C0F2D01F10C0170D01D
:10C0B80001301828F7D10023FA3A84F89230B74BA8
:10C0C800A4F89020B64D0993FEF7D7B8B4EEE77AF6
:10C0D800F1EE10FA40F3E081DFEDB25A9FEDB26A5B
:10C0E80001E0F0EE676AF4EEC66AF1EE10FA76EE59
:10C0F800E57AF6DCDFEDAD6AF4EEE67AF1EE10FAF9
:10C1080040F1C781DFEDA75A9FEDA96A01E0F0EE83
:10C11800667AF4EEC67AF1EE10FA77EEA56AF6D4EE
:10C12800DFEDA47AF4EEE76AF1EE10FA40F3E78067
:10C13800DFEDA17A77EEE66A66EEA65A9FED9F5A82
:10C148009FED9F6ADFED9F7AA5EE856A26EEA55AD8
:10C15800E5EE867AE5EE276AFFF784B99A49D1F8C1
:10C1680000E04200BEF1000F08D0171803EB870764
:10C178009EF801E07F787745BEF4C6A80244934F45
:10C18800934803EB820300220B603A800260FEF7BB
:10C19800BBB88D490F68450037B12E1803EB8606EA
:10C1A8007F787678BE4286D20544884E884803EB6D
:10C1B800850300250B60358005607CE7854B0022F0
:10C1C800012011E5844B1B78032B00F042810022EB
:10C1D800FFF7AAB9DFED817AB4EEE77AF1EE10FA4B
:10C1E80044BFDFED727A37EEC77AFFF783B97C4A2E
:10C1F8006B4D1360694B0993FEF73FB80C2F40F065
:10C20800B78000273946774B0D915B78BB423FF4E6
:10C2180008AA5F4B0C93384605F094FE0C9B0D99C9
:10C228009B781BB1C9B20C200FF0C8FF0137FFB2D1
:10C2380025E76D4A0592FEF700BF38EE678A6B4B1B
:10C248006B491870FDEEC87AC9F5FA63CDED047A2A
:10C25800BDF91020120381FB0201D217C2EBA11213
:10C268001BB203FB02F343F30F334B4407EE903A40
:10C27800F8EEE77AC7ED037AFEF711BA06F48056AE
:10C28800FEF7ADBF0023BB2A149300F0BF80B72A86
:10C2980000F0E980BE2A00F00681BD2A7FF4D3AC05
:10C2A8004FF6FE71534A3D48D68909909089334428
:10C2B8000144D38191810DF00BFBF5F757F90DF08F
:10C2C800EFFA00F04FFC01200CF004FAB4F89030BB
:10C2D8000022FA3BA4F8903084F89220FDF7CDBFF5
:10C2E800454A069B1E68136823F004031360089AE6
:10C2F800012306F4805682F82130FEF770BFDFED87
:10C30800377AF4EEE76AF1EE10FA44BFDFED277AE8
:10C3180077EEE66A10E7394A214D137843F00403B3
:10C3280013701E4B0993FDF7A8BF354B022203205B
:10C338005AE40DF0CDFAF5F719F90DF0B1FA00F05D
:10C3480011FC01200CF0C6F994F88E20FFF7E0B933
:10C35800214B1B78032B7EF4FAAD0CF0B9F8FDF7EE
:10C36800D3BF1D490978032900F08E80194698E645
:10C37800182F7FF456A900210B466FE6214B084D74
:10C388004FF4C8721A80054B0993FDF776BF00BFBA
:10C398003E6D0020443400208054030838510020AA
:10C3A80030510020DB0FC940E4CB1641DB0F49C0F8
:10C3B800E4CB16C1DB0FC93FDB0F494092E741B917
:10C3C8009730083C15A82ABE842400207025002038
:10C3D80074250020605E0020806D0020DB0FC9BF3F
:10C3E800985A0020B8720020BC7100200425002053
:10C3F800D34D6210605D00202C5100203C6D002060
:10C40800FC5E002082460020CFB2FCE619460223DB
:10C4180048E708231A46FEF73FBB07231A46FEF7EC
:10C428003BBB06231A46FEF737BB05231A46FEF721
:10C4380033BB04231A46FEF72FBB03231A46FEF725
:10C448002BBB02231A46FEF727BB01231A46FEF729
:10C4580023BB0CF03DF8FDF7D2BF4FF4FA61022080
:10C4680005F08EFC0DE419464FF6FE731AE7F0EE60
:10C47800477AFFF71DB8594B84F8941084F8950053
:10C48800574D0993FEF7B3BD0CF022F8B4F990208C
:10C4980011E6F0EE676A43E6F0EE667A2AE6B0EE59
:10C4A800677AFFF71BB80221FCE6002D3DF4EFADDB
:10C4B8004C4C94F88D30002B3DF41AAE0CF008F873
:10C4C800002384F88D30FDF713BE0021022005F00B
:10C4D80057FCB4F89030414A0992963B0022A4F8E0
:10C4E800903084F89220FDF7C8BE00210120EEE7C5
:10C4F80000210846EBE7FF21002018F02DFA94F8F8
:10C508008E20FFF7ACBB0121002018F025FA94F823
:10C518008E20FFF7A1BB0021FF2018F01DFA94F828
:10C528008E20FFF796BB0021012018F015FA94F829
:10C538008E20FFF78BBB00210320C8E711200D9345
:10C548000C920FF03BFED9F8D0000D9B0C9A95E4A5
:10C558000D200D930C920FF031FE0D9B0C9A07E500
:10C568000E200FF02BFED9F8D000FFF79FBB1D4C13
:10C5780016F00EFB002384F88D30FDF7B9BD1720A7
:10C588000FF01CFE27E40F200D930C920FF016FEFF
:10C59800D9F8D0000D9B0C9AFFE40021042096E7FF
:10C5A8000B200BF0B1FF0D4B0D4D0993FDF765BE48
:10C5B800002B3FF47DAF0C490C4A09684FF47A70A0
:10C5C80000FB0313136073E710200D930C920FF018
:10C5D800F5FDD9F8D0000D9B0C9A64E43851002081
:10C5E800305100207C25002024730020945A00201C
:10C5F80038B50B4C23688BB15A68821A002A054655
:10C6080004DA0CE05A68AA1A002A07DB9A68226042
:10C6180018461A6890472368002BF3D138BD38BDF7
:10C62800744300200B4B002210B4027203F18C04F7
:10C63800012102E0072A09DC9979890702D51979CD
:10C64800815401329C4203F11403F3D15DF8044B89
:10C65800704700BF606403081F230370704700BF62
:10C66800012310B410211224112244704171C270A8
:10C6780003720370037183705DF8044B704700BF49
:10C688002C22022302704370704700BF2DE9F04747
:10C698008C4B1B78DB07074644D58B4B8B4D1C789E
:10C6A8008B4E012C59D01CD3022C07D189498A4AB8
:10C6B80009881288914201D901241C70EB7AE3B1F0
:10C6C8002B89D3B1854B1B78BBB105F05DFC0028E5
:10C6D80000F09B802B7B83422CBF0121002131700D
:10C6E8000CE07C497E4A098810886A7B801A884257
:10C6F800E2DAEB7A0024002BE2D131782A79632A36
:10C7080006D8022C774E00F0BA803378002B5DD122
:10C71800754AAB7A8C4238BF0C461470002B4CD14A
:10C72800BDE8F0876B4B694D19885B88E878CB1AB0
:10C7380083EAE3728142A2EBE3721DD32B788B422A
:10C748001AD3614B1C78E01E012861D96749097822
:10C7580002294FD0012C5E4EA5D15F4A5D4912884F
:10C76800687B0988121A914239DD5D4A12888A422B
:10C77800A4D200241C70A1E7B1EB400FE1DC524BBE
:10C788001C78E11E012940F29480022ADEDC574918
:10C798004F4E0878DFF84481DFF844C1DFF838E10C
:10C7A80000210324022834701C7088F80010ACF8AB
:10C7B8000010AEF8001081D11FE0012C71D0022CBE
:10C7C8000BD10720BDE8F0470BF09EBE7068381A01
:10C7D800474B984258DD72709AE7BDE8F08702240B
:10C7E8001C706BE7022AD2DD4049097802294FF014
:10C7F800040464D13949364E09783E48022ACCBF30
:10C8080000220122C28081804BE70221317075E746
:10C81800022A9BDC95F800C091FBFCFC0CF1010C92
:10C82800BCF1080FDFF8B4A0304EA87895F801E005
:10C8380096F800802A4CDFF8A090254EA8BF4FF04C
:10C84800080C8AF800C01FFA8CFA10FB0AF01EFBCD
:10C858000AFE80B2DFF88CA02080A9F800E000244E
:10C868004FF0640EB8F1020F34701C70CAF804401F
:10C878008AF801E07FF439AF0FFA8CF1BDE7307820
:10C88800A0B9012377603370C2F164021A4B00FB30
:10C8980002F083FB0023C017A0EBA3506430707034
:10C8A80036E70820BDE8F0470BF02EBE7368F81A8B
:10C8B8008EE7032C96D10D49097802299AD0044EA7
:10C8C800FCE600BFAB5A0020342A0020C0500020EC
:10C8D800442A0020EC4E0020382A0020024F002075
:10C8E800362A00203C2A0020806D0020E84D0020D8
:10C8F8007F969800EC4D00206BCA5F6B2DE9F047DE
:10C908000569C3681D4028D00F4606464FF0004809
:10C918004FF00009B5FA85F328FA03F2D2431B3B1E
:10C9280032611540042B16D8DFE803F031292119AC
:10C9380003007B6A002B32D003F1FF3A1FFA8AFA10
:10C94800C7F824903C6A34B123682046514698477A
:10C958006468002CF8D1002DDCD1BDE8F087386878
:10C96800716B036889B29847002DD3D1F5E77868D1
:10C97800B16B036889B29847002DCBD1EDE7B86851
:10C98800F16B036889B29847002DC3D1E5E7F868D1
:10C99800316C036889B29847002DBBD1DDE7F36A93
:10C9A8001FFA83FACEE700BF08B50121022019F06B
:10C9B8007DFA094B1B7803F00503052B08D00021ED
:10C9C800012019F073FA0021084619F06FFAFEE702
:10C9D8000EF0C2FEF3E700BFF8310020022828BF9E
:10C9E800022010B4084C094B207000EB8002C0EB09
:10C9F800C20207495DF8044B013003EB4203C0B2A1
:10CA08000B600BF067BE00BFB8720020605E0020AC
:10CA18003451002008B50CF05BFFF4F7A7FDBDE822
:10CA280008400CF03DBF00BF38B5434B5A8999897F
:10CA3800914224BF00225A81198ADA89914224BF7F
:10CA48000022DA81DA788AB3072A2FD03B493C4D95
:10CA580091F85300012400210A282C709C70D97188
:10CA68003DD00C2865D0DFED377A8ABB364C9FED78
:10CA7800370AA278002918BFF0EE407A062A04D8AF
:10CA8800334901EB820191ED000A217959B3013A4A
:10CA9800032A4DD8F7EE007A87EE800A25F090FF3A
:10CAA8002388984228BF1846208038BDD97921B1FB
:10CAB80098780428B8BF04209870204890F853004C
:10CAC8000A280CD00C28CED1DFED227A002ACDD04E
:10CAD800072ACBD00A282CD1DFED1F7AC6E70A2017
:10CAE800DFED1E7AC1E79B78154A07EE103A1178F8
:10CAF800B8EEC77A27EE277A07EE901AF8EEE77AAB
:10CB080067EE877AB4EEE70AF1EE10FA10DDC0EEB0
:10CB1800077AFDEEE77A17EE903A102BA8BF10239C
:10CB2800012BB8BF0123DBB28B4238BF0B46137011
:10CB380038BDDFED0B7A99E71463002028630020E5
:10CB4800545D00206F120339B06700206F1203385C
:10CB58006C4103080AD7A3390F506E3A5304E938D9
:10CB68006F12833A2DE9F047A84FA94E0CF0B0FE9A
:10CB7800BE421ED2DFF81483DFF81493444625889A
:10CB880062197DB14A450DD2052D0BD933886188CC
:10CB9800C3F30B03994200F0DE801446258862191E
:10CBA800002DEFD171683046143619F0CEFBBE4225
:10CBB800E4D3984A1378A3F1170102290FD99649AB
:10CBC80011F83300002840F0F280D8000144497879
:10CBD80029B1924911F83330002B00F01081904BA5
:10CBE8005A78022A40F2DD8000228E495A701A785B
:10CBF8008D48022A016000F2D08002EB82018B4B43
:10CC0800C2EBC10203EB4203998C5A8C884C9142C7
:10CC1800236001D300225A84864B9A78042A00F0B4
:10CC2800E58032B91A88B2F5F07F84BF4FF4F0720C
:10CC38001A80814DFFF7F8FE2B68804A1A40002AB7
:10CC480000F0E080D80700F1CC80590400F1C480DE
:10CC58001A0700F1BC809B0400F1B28021F020FD8E
:10CC680010B977480AF04AFD802019F0A5FB4FF467
:10CC7800007019F0A1FB4FF4003019F09DFB4FF440
:10CC8800001019F099FB4FF0007019F095FB4FF068
:10CC9800806019F091FB0FF0ABFA0021302269484F
:10CCA80026F04BFE206815F00FF8674B276803F154
:10CCB800500102E0043399426DD01A78002AF9D164
:10CCC8009C78D8788442F5D26049614B0D796149E6
:10CCD80061480A70614E624C0460C822642111FBED
:10CCE8000521002259609A60DA601A615A619A61D6
:10CCF800DA6183F8202083F8212037600AF02AFBC4
:10CD0800584B9FED595A1B88584A9FED596A5079DC
:10CD1800584906EE903AF8EEE66A1388C5EE265AA8
:10CD280007EE103A53881279C1ED005A07EE903A8F
:10CD3800B8EEC77A504BF8EEE77A18725A7227EEB7
:10CD4800067A67EE867ABDE8F04783ED017AC3ED8F
:10CD5800007A0CF0A5BD63799B077FF41EAF71685C
:10CD680094F804A0304619F0F0FA3388BAEB133F70
:10CD780004D01436BE42FFF401AF1AE77388706816
:10CD8800AA1FC3F30B039A4204F10601A8BF1A466F
:10CD980025F040FCEDE7012296E700221A70234BAC
:10CDA80032E7204902EB420201EB82011FE7D8007B
:10CDB8000C186468002C7FF409AF1724147005E779
:10CDC8002E4819F0F9FA402019F0F6FA46E72C48EF
:10CDD80019F0F2FA2B683EE72A4819F0EDFA2B68A9
:10CDE80036E7294819F0E8FA2B682EE79A8AB2F54F
:10CDF8007A7FBFF41EAF4FF47A729A8219E718232C
:10CE08001370ECE643F008032B601BE714A5030836
:10CE1800A0A00308A45D00201C650308845E030825
:10CE2800B87200206C5F002038510020605E00203E
:10CE380034510020B0670020B85F0020096000026C
:10CE4800E871002018260020D84300206046002002
:10CE58001C530020580100205C2600204C2600208E
:10CE6800665D002008250020C0C9FB483C2300203F
:10CE780017B7D1380C250020A04500200940000232
:10CE880001600002092000020860000202F00308A5
:10CE98000000040808B50CF01BFDF4F767FB0CF064
:10CEA800FFFCFFF75FFE0120BDE808400BF012BC55
:10CEB8002DE9F047B54C82B06368204698470028B2
:10CEC80000F0BF80B24B1B780122042B84F83C2071
:10CED80000F0BA80B4F91610B4F91820B4F91A3071
:10CEE80021636263A363AB4B1B88002B69D0AA4DF7
:10CEF800D4ED0C7AD5ED004A95ED050A95ED015A69
:10CF080095ED067AD5ED035A95ED026AF8EEE76AD3
:10CF1800D5ED047AA4EEA60AA5EE267A67EEC07AC5
:10CF2800A5EEC07AE6EE267A85ED057AC5ED067A95
:10CF380025F046FDD4ED0D6AD5ED094A95ED0E0AAA
:10CF480095ED0A5A95ED0F7AD5ED0D7AD5ED0C5A77
:10CF580095ED0B6A2063F8EEE66AA4EEA60AA5EE44
:10CF6800267A67EEC07AA5EEC07AE6EE267A85EDD7
:10CF78000E7AC5ED0F7A25F023FDD4ED0E6AD5EDB6
:10CF8800124A95ED170A95ED135A95ED187AD5EDD5
:10CF9800167AD5ED155A95ED146A6063F8EEE66ACF
:10CFA800A6EEA40AA6EE857A67EEC07AA0EE657AA8
:10CFB800E6EE867A85ED177AC5ED187A25F000FD3C
:10CFC800A063764FA17F76480AF046F93B88002B8C
:10CFD8007CD1744E3568744B1B685B0742D4B5F935
:10CFE8000070216B636BA06B704A714E92ED026A00
:10CFF800D2ED006AD2ED015AC91B2163B5F902705E
:10D00800DB1B6363B5F904703568C01B07EE900A33
:10D01800B8EEE75A07EE901AB8EEE77A07EE903ABC
:10D02800F8EEE77A36EE056A36EE877A77EEA57A75
:10D038000135A06382ED026A82ED007AC2ED017AC1
:10D04800356002B0BDE8F0875A4BB4F91600B4F960
:10D058001810B4F91A2018802063598061639A80E7
:10D06800A26340E7544F3B88322B7ED0002B5BD124
:10D0780052480378002BB2D0DFF848E1F169326AF0
:10D088008EFB01730027C9170770C1EB23118EFBB4
:10D098000203D217C2EB2312736A29806A80A08A1E
:10D0A80047498EFB03E2DB17C3EB22131B1AAB8045
:10D0B800CF600CF00DFCF4F759FA0CF0F1FBFFF718
:10D0C80051FD01200BF006FB356888E7354E226BD1
:10D0D8003568B3F5C87F4FF0000323632B80398888
:10D0E80018BF7068B7F8008008BF0020B1F5C87F86
:10D0F80018BFB368616B02440B440020B8F5C87FC1
:10D1080060637260B36068803AD0D4F838E0F16840
:10D11800A0637144B8F1010FA880F16054D008F100
:10D12800FF38A7F8008056E7F169226B00232363D4
:10D138002B80B7F800E00A44BEF1320F616B6363DD
:10D148006B80F261A26B6BD0706A0190306AA36346
:10D158000144019831620244BEF1010FAB80726252
:10D1680063D00EF1FF333B8082E7154B2988D868DE
:10D178006A88AB883182B0617282B3820021D4E7B9
:10D18800A36BF360A063A880C9E700BFE850002044
:10D19800E84D0020C83B0020CC3B00208246002000
:10D1A800185100205C260020B0650020944500201E
:10D1B80090450020EC4D0020142600201126002068
:10D1C800605D00201F85EB51DFF80CC1DFF8F8E047
:10D1D800C8328CFB02A9C833D217C2EBE9128CFB08
:10D1E80003A9DB17C3EBE913C8316B802A808CFBDA
:10D1F800013CA28ACB17C3EBEC139B1AAB80CEF889
:10D208000C000CF065FBF4F7B1F90CF049FBFFF7E3
:10D21800A9FC40460BF05EFAB7F8008035687EE757
:10D22800A36331627262AB809BE7234A234812688A
:10D238002349037012F4003281F800E032D113461A
:10D248002049C85C0B2803F10C030ED00132182AC0
:10D25800F7D1338A2B80728A1B4B6A80B18AB269F4
:10D26800A980B7F800E0DA607BE71848D0F800C07A
:10D278005300BCF1000F09D003EB020E01EB8E0E38
:10D288009CF801C09EF801E0E645E2D21344DFF8BD
:10D298004CE00F4A01EB830100230160AEF8003037
:10D2A8001360D6E70B4A1278032A01D01A46C7E75B
:10D2B8000BF00EF93568CCE7443400201626002020
:10D2C8001026002080540308605D0020842400207C
:10D2D80074250020806D00201F85EB5170250020EB
:10D2E80038B50C4C0C4DAC4206D26168204614345B
:10D2F80019F02BF8AC42F8D3084A094B094C1460D2
:10D30800002209491A705A7008480860BDE8384078
:10D318000FF014BFA0A0030814A50308345100207F
:10D32800B8720020605E0020385100206C5F002039
:10D3380008B5FFF7D5FF0CF0CBFAF4F717F9BDE8FD
:10D3480008400CF0ADBA00BFF0B50C292BD8DFE8C7
:10D3580001F06F2A2A2A4C2A2A2A2B2A2A2A07006D
:10D36800046AB2F80CE097881668674D24F4805474
:10D378000462036A4468C16923F4005343EA0E3324
:10D3880021F4E641A84243EA073341EA062100F0C6
:10D39800B58005F50065A84200F0B0809268446049
:10D3A800C16102640362F0BD046A96899588D2F867
:10D3B80000E0554F24F480740462036A4468C1692C
:10D3C80023F4007343EA062321F07301B84243EAC9
:10D3D800052341EA0E017ED04C4DA8427BD09268CD
:10D3E8004460C161C2630362F0BD046A968995888E
:10D3F800D2F800E0444F24F010040462036A446841
:10D40800816923F0200321F0807143EA061321F497
:10D41800E641B84243EA051341EA0E2148D03B4DA4
:10D42800A84245D092684460816182630362F0BD7E
:10D43800046A9389B2F804E01768334E24F00104B3
:10D448000462056A4468816943EA0E0321F4803165
:10D4580025F002059BB221F07301B04243EA0503AF
:10D4680041EA070114D0294DA84211D005F54065BD
:10D47800A8420DD005F58065A84209D005F580655C
:10D48800A84205D092684460816142630362F0BD9E
:10D49800D689158A578A23F0080333433D43D68833
:10D4A80024F4407423F00403ADB233432C43E9E77A
:10D4B800D589178AD68823F0800343EA051324F414
:10D4C8004064558A23F0400344EA870443EA06137C
:10D4D80044EA8504A6E7D589178AD68823F4006329
:10D4E80043EA052324F44054558A23F4806344EA2C
:10D4F800071443EA062344EA051470E7158A24F45E
:10D50800804444EA851449E7002C01400034014076
:10D518002DE9F04FC822002183B07948794CDFF813
:10D528000892794D794E7A4FDFF8008226F005FA95
:10D5380078487949DFF8F8E1DFF8F8C10022135993
:10D54800834200F0C280B3F1804F00F0CA80AB4242
:10D5580000F0C980B34200F0C880BB4200F0C78029
:10D56800734500F0C680634500F0C580434500F070
:10D57800C480DFF8C4A153457AD00AF5806A5345C0
:10D5880008BF092375D01432A02AD8D15D4C634D49
:10D59800634E614F04F1A00802E01434A04564D042
:10D5A800A379002BF9D023794FEA131909F1FF3930
:10D5B800B9F1050F03F00F03EFD835F8190040FA59
:10D5C80003F2D207E9D54FF0010A0AFA03F3013B47
:10D5D800184024F0B1FD16F809305249184411EBEF
:10D5E800C002DAD051F83000DFF850E1217A00F1BA
:10D5F80038439B0A1EF8033003F01F0E5B09022B09
:10D608000AFA0EFA63D0032B66D0012B58D0938800
:10D618000093B3FA83F3C3F11F039BB2DA0800EB5C
:10D62800820203F00703D2F820E09B004FF00F0CB2
:10D638000CFA03FC2EEA0C0EC2F820E0D2F820E027
:10D6480001FA03F343EA0E03136269460023022238
:10D6580014348DF804208DF805308DF806308DF8D7
:10D66800073016F0D3FEA0459AD103B0BDE8F08F7D
:10D67800082309EBC3034FF0010B93F820A00AF02D
:10D688001F034FEA5A1ABAF1020F0BFA03F311D02B
:10D69800BAF1030F08D0DA457FF475AFD1F814A0BA
:10D6A80043EA0A034B616EE7D1F81CA043EA0A0378
:10D6B800CB6168E7D1F818A043EA0A038B6162E7F7
:10D6C8007B694AEA03037B61A1E70023D1E7BB69D1
:10D6D8004AEA0303BB619AE7FB694AEA0303FB6171
:10D6E80095E70123C5E70223C3E70323C1E7042322
:10D6F800BFE70523BDE70623BBE70723B9E700BF5C
:10D70800F470002060640308000400400008004032
:10D7180000100040002C014000100240E86103089E
:10D72800F4610308E46100206C41030800400140F3
:10D73800001400400034014000440140FC6103082B
:10D7480001490248FFF7DAB8947100200048014007
:10D7580001490248FFF7D2B8447100200034014063
:10D7680001490248FFF7CAB844710020003401405B
:10D7780002494FF08040FFF7C1B800BF1C7100207C
:10D7880010B5064C06482146FFF7B8F804F17801B1
:10D798000448BDE81040FFF7B1B800BFF47000209E
:10D7A800002C01400044014001490248FFF7A6B897
:10D7B800F4700020002C01402DE9F04104684A4D26
:10D7C800A30AAB4272D009D8B3F5801F6AD0023DD4
:10D7D800AB425AD14FF0200E002608E0434DAB4231
:10D7E80068D00135AB4252D14FF0C00E04264779BC
:10D7F8004FEA970C002961D0B000634685190227CB
:10D80800D4F80C809F400CEB4503BFB2384D03F1B0
:10D81800040C47EA080745F8231045F82C20E76070
:10D82800EFF31181502282F31288821905EBC202AC
:10D83800136973B313620433821905EBC202576983
:10D8480017B11F6053690433821905EBC202976947
:10D8580017B11F6093690433821905EBC202D769B7
:10D8680017B11F60D36904330027CAB21F6082F35F
:10D878001188304405EBC000036A6BB9E3684FF6C2
:10D88800FE721340E360BDE8F081BDE8F081BDE8B9
:10D89800F08105EB0E03CFE7E36843F00103E36093
:10D8A800BDE8F0814FF0480E0126A0E74FF0700E5A
:10D8B80002269CE74FF0980E032698E7BF0802233C
:10D8C80006FA03F0BB40DB43E768094D9BB23B40D7
:10D8D80087190CEB470CE3600CF1040345F82C1096
:10D8E80045F823209CE700BF4D00100051001000B0
:10D8F800F470002030B503685C4D18885C4CB4FBAC
:10D90800F2F20139013AAB4294B283B089B282B2E1
:10D9180066D05848834263D0B3F1804F60D0A0F5F9
:10D92800983083425CD000F58060834258D05248DA
:10D9380083425BD000F5806083427DD022F4407240
:10D9480000F58C3092B283421A80D9621C850ED0C1
:10D95800484A93420BD002F54062934207D002F541
:10D968008062934203D002F58062934201D1002283
:10D978001A8601225A611A883C4992B242F0010281
:10D988008B421A8062D0B3F1804F61D03B4A9342F8
:10D9980060D002F5806293425ED002F50062934245
:10D9A8005CD002F5806293425AD002F590329342DD
:10D9B80058D002F54062934256D002F580629342F5
:10D9C8001ED002F58062934208BF092219D002A82E
:10D9D8004FF0012340F8043D16F0E2FC03B030BDDF
:10D9E800254822F07002834292B2A3D101201A8006
:10D9F800D9621C8558611A8892B202431A80C5E719
:10DA080008221F4B03EBC20301A893F821408DF8AD
:10DA18000440012300228DF805308DF807308DF879
:10DA2800062016F0BDFC1B2CD8D1164B019301A87B
:10DA380016F0B6FC03B030BD01201A80D9621C85EF
:10DA480058611A8892B202431A809CE70022D8E7EC
:10DA58000122D6E70222D4E70322D2E70422D0E744
:10DA68000522CEE70622CCE70722CAE7002C0140B0
:10DA780000A24A04003401400010004000040040A5
:10DA88006C41030819010001204B98422DD0B0F1D8
:10DA9800804F2CD0A3F5943398422AD003F58063A5
:10DAA800984228D003F50063984226D003F5806396
:10DAB800984224D003F59033984222D003F540636E
:10DAC800984220D003F58063984207D003F580631D
:10DAD800984208BF092202D00020704708220C4B48
:10DAE80003EBC20393F8200070470022F7E70122F6
:10DAF800F5E70222F3E70322F1E70422EFE7052224
:10DB0800EDE70622EBE70722E9E700BF002C01401A
:10DB18006C4103082DE9F04F013085B0C3B203937F
:10DB28000B4602918B4C8C4E002B00F09A803220D1
:10DB38008A4D8B4FDFF82C9221F0A2FD4FF4FA7A30
:10DB48004FF0100C4FF47A70D9F80430C3F308037F
:10DB5800002B40F0DE80EFF31183002B40F0D980DA
:10DB68002968A26800BF2B689942F9D1D7F800E06C
:10DB780000FB0EF39B1AB3FBFEF300FB01314FF0E1
:10DB8800010E0191D9F80430C3F30803002B40F0CB
:10DB98008780EFF31183002B40F082802B68A16807
:10DBA80000BF2A689342F9D1D7F800B000FB0BF206
:10DBB800521AB2FBFBF200FB0323019A9B1AB3F53E
:10DBC8007A7FDFD3BAF1010ABED1039B002B40F064
:10DBD800BD804FF47A7ADFF88C9150464FF0100CE4
:10DBE800D9F80430C3F30803002B75D1EFF3118380
:10DBF800002B71D12968A26800BF2B689942F9D11E
:10DC0800D7F800E000FB0EF39B1AB3FBFEF300FB12
:10DC180001314FF0010E0191D9F80430C3F3080324
:10DC280013BBEFF31183FBB92B68A16800BF2A6807
:10DC38009342F9D1D7F800B000FB0BF2521AB2FBAD
:10DC4800FBF200FB0323019A9B1AB3F57A7FE3D317
:10DC5800BAF1010AC4D1029B013B0293002B7FF465
:10DC680066AF05B0BDE8F08FEFF311888CF312882A
:10DC7800A1682368DB0344BFC6F800E0A1682B68ED
:10DC880032685FFA88F888F31188D7F800801A4458
:10DC980000FB08F35B1AB3FBF8F300FB0233D2E78F
:10DCA800EFF311888CF31288A1682368DB0344BF63
:10DCB800C6F800E0A1682B6832685FFA88F888F334
:10DCC8001188D7F800801A4400FB08F35B1AB3FBED
:10DCD800F8F300FB023370E7EFF311828CF312883C
:10DCE800D4F808E02368D90303D501233360D4F8B6
:10DCF80008E02B683168D2B282F311883A68194477
:10DD080000FB02F3A3EB0E03B3FBF2F300FB0131BC
:10DD18007FE7EFF311828CF31288D4F808E02368C8
:10DD2800D90303D501233360D4F808E02B683168A0
:10DD3800D2B282F311883A68194400FB02F3A3EBCC
:10DD48000E03B3FBF2F300FB013118E7184621F08C
:10DD58001BFB3EE710E000E0207300202473002046
:10DD68002873002000ED00E0204B5B68C3F3080334
:10DD780030B4BBB9EFF31183A3B91D4B1D4C186820
:10DD8800A16800BF1A689042F9D11B4B1C684FF478
:10DD98007A7202FB04F3591AB1FBF4F130BC02FBAE
:10DDA80000107047EFF31182102383F31288114992
:10DDB8008C680B6813F4803F104B02D00120186068
:10DDC8008C680B49D2B20D68186882F311880A4B27
:10DDD80019684FF47A72284402FB01F31B1B30BC0C
:10DDE800B3FBF1F302FB0030704700BF00ED00E029
:10DDF8002473002010E000E0287300202073002026
:10DE08002DE9F84F8046FFF7AFFF254E2549DFF88B
:10DE1800A0E0254A254D844610274FF47A74012046
:10DE2800DEF80430C3F30803D3B9EFF31183BBB9A9
:10DE38000B68D2F808A000BFD1F800904B45F7D185
:10DE4800D6F800B004FB0BF9A9EB0A09B9FBFBF9FA
:10DE580004FB0393A3EB0C034345E1D3BDE8F88F20
:10DE6800EFF3118A87F31288D2F808B01368DB033E
:10DE780044BF2860D2F808B00B68D5F800905FFA64
:10DE88008AFA8AF31188D6F800A0994404FB0AF3A9
:10DE9800A3EB0B03B3FBFAF304FB0933DAE700BF88
:10DEA800287300202473002010E000E02073002075
:10DEB80000ED00E02DE9F04FDFF830C1474A48494E
:10DEC800484E494D8046102718F1FF38C0F084802D
:10DED800DCF80430C3F30803002B5CD1EFF31183A3
:10DEE800002B58D10B68946800BF08688342F9D1A9
:10DEF800D6F800904FF47A7000FB09FEAEEB040EE2
:10DF0800BEFBF9FE00FB03EEDCF80430C3F30803A4
:10DF18004FF47A740120FBB9EFF31183E3B90B686E
:10DF2800D2F808A000BFD1F800904B45F7D1D6F839
:10DF380000B004FB0BF9A9EB0A09B9FBFBF904FBD8
:10DF48000393A3EB0E03B3F57A7FBDD2DCF804305C
:10DF5800C3F30803002BDFD0EFF3118A87F312888D
:10DF6800D2F808B01368DB0344BF2860D2F808B0C1
:10DF78000B68D5F800905FFA8AFA8AF31188D6F808
:10DF880000A0994404FB0AF3A3EB0B03B3FBFAF3D9
:10DF980004FB0933D5E7EFF3118487F31288D2F82D
:10DFA80008901368D80303D501232B60D2F8089092
:10DFB8000B682868E4B284F31188D6F800A04FF4FF
:10DFC8007A7400EB030E04FB0AF3A3EB0903B3FB1B
:10DFD800FAF304FB0E3E97E7BDE8F08F10E000E08F
:10DFE80024730020287300202073002000ED00E037
:10DFF80030B4EFF31183102282F312880649074CDC
:10E008000A680748013200250A602560DBB2026809
:10E0180083F3118830BC70472473002020730020DC
:10E0280010E000E00F4B1B88014643B90E4B0F4A26
:10E038001B7810680BB981F0010117F02DBF0C4B4C
:10E048005A691AB118B91A68106058747047094AA1
:10E0580018681188084A92FBF1F20121026059748C
:10E06800704700BFFC720020FE7200200073002081
:10E07800047300201C73002020A107001D4B70B5FD
:10E088009C68236D626BDD69C2B1A36B2BB12B0752
:10E0980002D5236D08221A6270BD2A06F7D5A26A36
:10E0A800616A8A4220D0511CA069A162825C206901
:10E0B800266D81423285EAD3A362E8E7A906E4D552
:10E0C800E26A22B1988C216B80B29047DDE7E16962
:10E0D8009B8C6069DBB24E1CE6614354E169E368DE
:10E0E800994228BFE261D0E7226D136823F08003CC
:10E0F8001360CCE7FC3100201D4B70B55C68236DC4
:10E10800626BDD69C2B1A36B2BB12B0702D5236DFE
:10E1180008221A6270BD2A06F7D5A26A616A8A4285
:10E1280020D0511CA069A162825C2069266D8142C1
:10E138003285EAD3A362E8E7A906E4D5E26A22B108
:10E14800988C216B80B29047DDE7E1699B8C606910
:10E15800DBB24E1CE6614354E169E368994228BF8B
:10E16800E261D0E7226D136823F080031360CCE7E7
:10E17800FC3100202DE9F04FC04B1E788BB0002EEB
:10E1880040F0BC80BE4BBF4C1D78DFF818A3DFF809
:10E198001893DFF8188305F00105A4F10A0B54F869
:10E1A8000A3CBBB1CC2707FB06B7184617F032F874
:10E1B80080B154F80A0C17F025F814F8023C8BB912
:10E1C800242831D0F5B154F80A3C184617F022F843
:10E1D8000028EED10136032E04F1CC04DFD10BB0B8
:10E1E800BDE8F08F012B23D0022B2BD0032B37D087
:10E1F800042B67D0052B40D0062B4FD054F80A2C9F
:10E208001346D2E754F80A3C23281A4600F08981BD
:10E218009D4991F832108142C7D19C4BCAF80090B1
:10E22800C3F80C801346C0E7012304F8023CCAE790
:10E238004D2854F80A2C0CBF0223002304F8023C92
:10E248001346B2E700233C2804F8023C45D03E2898
:10E25800D4D10122032304F8012C04F8023CB2E7CC
:10E26800C02814D80022042304F8050C04F8040C70
:10E2780004F8062C04F8023CA5E714F8063C14F848
:10E28800052C9A422FD814F8043C834203D000236B
:10E2980004F8023C97E7062304F8023C14F801EC62
:10E2A800BEF1000F00F08281BEF1010F00F0C681BF
:10E2B80001360023032E04F8023C04F1CC047FF459
:10E2C8006EAF8CE714F8043C04F8030C584005239F
:10E2D80004F8040C04F8023C75E7032204F8013C36
:10E2E80004F8022C6FE714F8042CF91842400133A3
:10E2F80004F8042C04F8063C887264E7644B186838
:10E3080000283FF46CAF17F057FFDFF8A4A1614D68
:10E31800DFF8A091DAF8000016F07CFF00283FF43F
:10E328005EAFDAF8000016F06DFF09281BD03F2811
:10E3380019D02B68002B67D1042800F0A9810C287C
:10E3480000F0E8807F28E5D0A0F12002D2B25E2A52
:10E35800E0D80BB92028DDD05A1C09F803002A6040
:10E3680012F020FBD6E72C68002C5BD14A4FA3465D
:10E3780007F59878BBF1000F08BFBB46083747453B
:10E38800F8D1BBF1000F00F07881083FDBF80000FE
:10E398003A68065D135D9E42204402EB040140F09A
:10E3A8006A81661E4E4422460BB9FD2A5DD906F8DD
:10E3B800013F01322A6010F8013F11F801EF9E4534
:10E3C800F2D00AB15F4512D0344812F0F3FA5F4533
:10E3D80008D35BF8080B12F0EDFA092012F0E2FA04
:10E3E800BB45F6D92E4812F0E5FA2A680024944273
:10E3F80090D2661E4E4416F8010F12F0D3FA2B681D
:10E4080001349C42F7D385E70C2800F083800A2862
:10E4180052D00D2850D07F2800F0FD80FF2B3FF60A
:10E4280079AF91E71C4E002706F59878BB4602E0C5
:10E43800083646450DD0224631684846F3F7EAFAD1
:10E448000028F5D1B346002FF2D1374608364645A5
:10E45800F1D13B465F469B46002B97D1002F3FF4F6
:10E4680059AF0E4812F0A6FAB3E7511C202009F85C
:10E478000200296009F801300A46A3E7BC480020D9
:10E48800AB5A0020267C0020E871002000ED00E057
:10E49800D4350020D8360020BC430308B0690308EF
:10E4A800B8690308FC9F0020EFBEADDE0400FA0542
:10E4B8008C350020D835002012F0FDFA23217C4845
:10E4C80025F052FA002800F0E180A0EB090028604E
:10E4D80088B1431E19F80310202940F0E78009EBA2
:10E4E800030204E012F8011D202948D10346581EF2
:10E4F800002BF7D12B604FF480720021484625F09D
:10E508001CFA6C4B1B78002B3FF469AE6A4812F07A
:10E5180051FAFFE6694812F04DFA674812F04AFAD4
:10E52800F8E667496748C978674ADFF8CCE193623B
:10E53800003118BF012101706449D1624021136381
:10E5480082F8341082F83550614962480B602C32E9
:10E55800CEF80020574A0123137012F067FC564882
:10E5680012F028FA4FF4006003F048F85A4B93F879
:10E578003230232B00F0928014F8023C3CE62B60EA
:10E58800564C002204F5987809F8032002E0083474
:10E59800444577D02168484606F018FF0028F6D091
:10E5A80044456FD2636898470023A3E74C4BADF806
:10E5B80022E00FCB0DF1280C02AF87E80F004CF8D2
:10E5C80024ED14F8051C14F8033C069404EB010E22
:10E5D800624639464FF0010C06A8CDF81CE0ADF8AC
:10E5E80020308DF824C0F4F78DFEE8B9019F002390
:10E5F80004F8023C002F3FF4EDAD54F80A0C09F082
:10E60800E9F9013654F80A0CB847032E04F1CC0492
:10E618007FF4C5ADE3E5013B002232482B6009F8E1
:10E62800032012F0C7F975E6029A2F4B0392394678
:10E63800A4F10A00029309F047F9D7E714F8053C5A
:10E6480014F8032C0694234407936E2A4FF0000312
:10E6580008930993ADF820207FF42AAE06A8F3F7B3
:10E668005BFA06A8F3F74CFA06A8F3F749FA06A8E6
:10E67800F3F746FA1CE62246A3E61C48083F12F0C8
:10E6880099F9A6E61A4812F095F98DE728681FE768
:10E69800074806F0F9F80BB0BDE8F08F154A14F8F2
:10E6A800023CC2F80C80CAF80090A5E5034667E76B
:10E6B800D8350020BC480020B8690308C0690308A1
:10E6C800B8720020C02A00205C260020E54E02080F
:10E6D8008C350020EC690308E8710020BC4303086E
:10E6E800D8410308E869030824800020B0690308BA
:10E6F800CC69030800ED00E0D43500202DE9F04F87
:10E708002DED028B93B005461DF0AAFDB34B1E7884
:10E7180026B113B0BDEC028BBDE8F08FB04B1B687F
:10E728005805F6D5DFF81C83D8F80020002A00F039
:10E738001C81AC4CD4F8283103F5F43348339D429E
:10E74800C0F01381A84994F82C310968C4F82851FD
:10E758000133DBB2890784F82C3101F1108113F001
:10E76800070701F05D80282BA04B029301F09081F0
:10E778005E2090479E4B1B78002B6BD0994C9D4A8E
:10E78800D4F83031EB1A934200F2CE87DFF8B8A202
:10E798009AF80080B8F1000F33D1DFF86892D9F801
:10E7A800000016F037FDC0B201280ED90228924F9A
:10E7B80041F06E823B78002B41F09C83D4F83831CD
:10E7C800EB1AB3F57A6F81F048848C480768002FFC
:10E7D80040D09AF80030BBB9894BD9F800001B68C3
:10E7E8009B781E3B012B4FF0020141F28E830430CF
:10E7F80010F06EFB012200238AF8002084F84431CF
:10E8080026E07E4807682FB3D4F8403140F6B73287
:10E81800EB1A93421ED994F83C31002B01F02F8259
:10E82800013BDBB284F83C31002B01F0168117F86C
:10E83800011B94F84421076094F8453171480A4453
:10E848000133006884F8442184F8453116F0E6FC69
:10E85800C4F840516C4A029B12781B68012A03F1E4
:10E8680001030A9300F0B186684B1B786BB1684FBF
:10E878003B6853B1029B5B4CD3F800B0D4F85831D5
:10E88800ABEB0303632B00F24086DFF8C08198F8F6
:10E8980000A0BAF1020F01F0BC80574F97F874300E
:10E8A800032B00F087875B4B1B7873B15A4E336894
:10E8B8005BB14C4CFFF758FAD4F8643144F61F6248
:10E8C800C31A9342834600F2D580544B1B78002B21
:10E8D8004ED1534B1B7843B1424CD4F8B43203F5B4
:10E8E8000043E8339D4280F0E6864E4B1B78002BB0
:10E8F8003FF40FAF3B4E4C4C4C4D06F2BD27206801
:10E9080016F088FC00283FF404AF206816F07AFC63
:10E918002B7880465A1E33B120682A7016F07AFC8C
:10E928000028F2D1F5E603223946781E24F0EBFFE1
:10E9380096F8BC3296F8BD2286F8BF8283F47F43EE
:10E9480083F0FF039B1A1FFA88F89BB2B8EB132FCA
:10E95800D5D196F8BE22DBB29A42D0D1781E0FF0FC
:10E96800CFFD2B7818442870C9E7204B029301E7A4
:10E978002F4C2278002A40F01F86DFF8D49099F8AF
:10E988000040002C66D12B4E3078002841F03D82A3
:10E99800144C294ED4F8AC223178284B93FBF1F370
:10E9A80013449D4295D3264A94F8B032C4F8AC5229
:10E9B800D75CF90701F16F83BA0701F1B8837B07C8
:10E9C80001F1FF8294F8B0323178013393FBF1F210
:10E9D80001FB123384F8B0327BE700BFBC4800204B
:10E9E800B0650020D4260020DC50002024730020CD
:10E9F800226E00203F0D030024000020886D0020B7
:10EA0800846D002040510020236E0020306E0020CD
:10EA1800B4730020386E00203C6E00207C6E00200D
:10EA28008D6E0020426E0020486E00204C6E002043
:10EA3800146E0020846E00208C6E0020A0860100D9
:10EA4800886E0020906D00208C6D002062430020AD
:10EA5800856E0020054E376E002F41F05480044B20
:10EA680089F80070C3F8AC5233E700BF946E0020F9
:10EA7800D426002094F86A31002B40F0FB87E04B45
:10EA88001B6803F00802002A48F603414AF60B40C7
:10EA98004BF60F4249F6074704BF02460F4613F0EC
:10EAA800040F4FF0190118BF17469A0684F86A1127
:10EAB80003D547F4804747F0200703F057FAC7F318
:10EAC8000909002841F05184CE4B9B79002B41F075
:10EAD800BA84984664204FF0FF3A4FF0000C0A972A
:10EAE8000B97ADF834C0CDF83AC0CDF83EC0CDF89C
:10EAF80042C0CDF83090ADF83680ADF838A08DF82A
:10EB080046000AAF0FCFDFF80CE384F805C0AEE883
:10EB18000F0097E80F00AEE807002EF8023B714699
:10EB28004FF0010C1B0CFE271F20C82201F81E39CC
:10EB3800A770A27184F807C0E07094F87A01207178
:10EB480080F0F10383EA0313DAB2130983F0E703D1
:10EB580043EA022383EAC2031BB283EA0312D2B256
:10EB6800C3F3072383EA121343EA022383EAC203A7
:10EB78001BB283F0C80282EA0212D2B2C3F307239F
:10EB880083EA121343EA022383EAC2031BB283EA2D
:10EB98000C0787EA0717FFB2C3F3072282EA1712A6
:10EBA80042EA072200EB0C0382EAC7070EEB0C00CF
:10EBB80084F87A31278011F8013B7B4083EA0313FC
:10EBC800DBB21A0982EA172242EA032282EAC30365
:10EBD8001BB29FB281422780EDD183F07C0383EA88
:10EBE8000313DBB24FEA131E8EEA172E8EEA032EAA
:10EBF8008EEAC30E0FFA8EFE1FFA8EF9DFF818C2DE
:10EC0800A4F800905FFA8EFE4FEA192984F828903C
:10EC180084F827E00CF5D17804F1220ADCF800002A
:10EC2800DCF80410DCF80820DCF80C3047460FC785
:10EC38000CF1100CD445B846F0D1DCF8000038606F
:10EC4800714F9CF8043088F8043007F1270884F8DD
:10EC5800C9E184F8CA9117F8011F306816F0DEFA86
:10EC6800B845F8D194F86B21002A40F0FE86674930
:10EC7800029B08781B680A2184F86B11002801F0B0
:10EC8800B380DFF898E10128BEF80010059141F241
:10EC9800C0830228BEF8028001F07E83BEF804100B
:10ECA8000491032801F0BD830428BEF806A001F0F2
:10ECB800C583BEF808100391052801F0BB83062818
:10ECC800BEF80AC001F0C6830728BEF80C1001D0B0
:10ECD800BEF80E2094F87A010A93074687F03003AD
:10ECE80083EA0313DBB24FEA131E494806978EF0F6
:10ECF8007A0E4EEA032E008827718EEAC303DFF8E6
:10ED080020E1C0EB00208EFB007E8644C017C0EBDC
:10ED18006E270797059F4FF0000967F30F09049FB7
:10ED280068F31F494FF0000867F30F08039FCDF8F9
:10ED38002C901BB24FF0000E83EA031067F30F0EFE
:10ED48000027C0B261F30F07C3F307236CF31F4E0C
:10ED580062F31F474FF0000C9DF81C20CDF834E0FB
:10ED680083EA10136AF31F48CDF830800E978DF8A8
:10ED78003CC08DF83D2043EA00230DF1280883EAC2
:10ED8800C007B8E80F003FB287F0C80989EA091937
:10ED9800DFF880E084F805C05FFA89F9C7F3072730
:10EDA800AEE80F0087EA191747EA092398E8030035
:10EDB80083EAC9031BB283F023074EF8040B87EAE2
:10EDC8000717FFB2C3F3072282EA1712069B7046A1
:10EDD80042EA072203F1010882EAC70720F814195A
:10EDE8004FF0230CFE211622C82384F87A8127804D
:10EDF8000EF1020E84F807C0A170E270A37111E051
:10EE0800DC500020C0500020772800203442002029
:10EE1800446D0020DC260020D6260020506D0020FE
:10EE28000308208010F8013B7B4083EA0313DBB220
:10EE38001A0982EA172242EA032282EAC3031BB2B2
:10EE48009FB270452780EDD183F0F40383EA031362
:10EE5800DBB21A0982EA172282EA032282EAC30392
:10EE68001BB21FFA83FEE74FA4F800E05FFA83FCA9
:10EE78004FEA1E2984F81EC084F81F907968BA6882
:10EE88003868FB6807F5D17EAEE80F003869796904
:10EE9800BA6904F2C118AEE8070004F2A31784F8AF
:10EEA800C19184F8C0C117F8011F306816F0B6F98F
:10EEB800B845F8D194F87271002F40F0E485D24B30
:10EEC80094F87AC1B3F90010B3F90220B3F9043009
:10EED8009FEDCE6A677107EE103A029B1B680A9392
:10EEE8008CF06A0383EA031306EE901AD9B20B0971
:10EEF80083F0D50343EA012383EAC1031BB283EA03
:10EF080003115242C9B207EE902AC3F3072383EADA
:10EF1800111343EA0123F8EEE77AF8EEE66AB8EE51
:10EF2800C77A83EAC1031BB267EE867A66EE866A01
:10EF380027EE067A002083F0C80ECDED0C7ACDEDD1
:10EF48000B6A8DED0D7A0E900F9010908EEA0E18C8
:10EF58000DF128095FFA88F8C3F3072EB9E80F0006
:10EF68008EEA181E4EEA082E8EEAC80EDFF8B08226
:10EF78000FFA8EFEA8E80F008EF01E0799E807002A
:10EF880087EA071A5FFA8AFACEF3072787EA1A1779
:10EF980047EA0A2788E8070087EACA071C214FF0D2
:10EFA800050A4FF01E094FF0FE0EC8220CF10103AE
:10EFB800E17084F872A184F8079084F802E0A8F15F
:10EFC8001001A27108F10C0084F804C0278084F8AD
:10EFD8007A3111F8013B7B4083EA0313DBB21A094B
:10EFE80082EA172242EA032282EAC3031BB29FB2D3
:10EFF80081422780EDD183F0270383EA0313DBB234
:10F008001A0982EA172282EA032282EAC3031BB2A0
:10F018001FFA83FCDFF8EC81A4F800C05FFA83FED6
:10F028004FEA1C2C84F825C084F824E008F5D1792F
:10F0380004F1220AD8F80000D8F80410D8F80820FB
:10F04800D8F80C304F460FC708F11008D045B9461C
:10F05800F0D16F4FB8F80030A9F8003007F1240854
:10F0680084F8C6E184F8C7C117F8011F306816F0A4
:10F07800D5F8B845F8D194F873310293002B40F0D5
:10F08800FE8494F87AA1604B624AB3F90410B2F98D
:10F098000620614F6148DFF888E184F804A08AF00F
:10F0A800220383EA03135FFA83FC4FEA1C1383F0FD
:10F0B800590343EA0C2383EACC031BB2B2F5FA6F77
:10F0C80083EA031C5FFA8CFCA8BF4FF4FA62C3F30F
:10F0D8000723B2F57A7F83EA1C1343EA0C23B8BFEF
:10F0E8004FF47A7283EACC03A2F57A724FF0640C7B
:10F0F8000CFB02F287FB027C80FB0170D217C91758
:10F108004FF000091FB2C2EBAC12C1EBA0030DF126
:10F118002808CDF82890CDF82C90CDF83090CDF86F
:10F12800349087F0C80CADF83A20ADF83830C146B5
:10F13800B9E80F008CEA0C1C5FFA8CFCC7F30727B0
:10F1480087EA1C1747EA0C2787EACC07AEE80F00C6
:10F158003FB287F04A0383EA0311C9B2C7F3072312
:10F1680083EA111343EA0123724683EAC103D9F8FB
:10F1780000C09DF8081061710AF1010705204A21B5
:10F188004FF0FE0984F87A7142F810C914274FF03D
:10F19800C80C84F8730123800EF1040EE17184F821
:10F1A8000290E77084F806C0184612F8011B414027
:10F1B80081EA0111C9B20B0983EA102343EA01234A
:10F1C80083EAC10109B288B272452080EDD181F08D
:10F1D800140181EA0111C9B24FEA111E8EEA102EFC
:10F1E8008EEA012E8EEAC10E0FFA8EFE1FFA8EF9F4
:10F1F8004FEA192C034B034884F81DC05FFA8EFEB2
:10F2080010E000BFD6260020E050002088C3E43A72
:10F2180077280020506D0020D34D6210676666661F
:10F22800DC26002084F81CE0D94F59689A680068E9
:10F23800DB68A4F8009007F5D179A9E80F003869D0
:10F248007969B7F818A0A9E8030004F2A317A9F888
:10F2580000A0BA4684F8BFC184F8BEE104F2BF1921
:10F268001AF8011F306815F0D9FFD145F8D1C94BFC
:10F27800C94A1B781278013B12F00100DBB214BFB7
:10F28800C0214021172B03D8C44A13441B7B029387
:10F29800C34B1A8893071ABF002341F010010123BA
:10F2A80012F4027F18BF022312F0100F18BF0623B2
:10F2B80012F0200F18BF1023002840F0BF864FF02F
:10F2C800030994F87AC10A938CF0460383EA03137E
:10F2D800DAB2130983F0920343EA022383EAC203F2
:10F2E8001BB283EA0310C0B2C3F3072282EA1012EA
:10F2F80042EA002282EAC00212B282F0C80E8EEA06
:10F308000E1E00235FFA8EFE9DF808A08DF82CA033
:10F318000320C2F307228DF82F9082EA1E128DF87F
:10F328002D308DF82E108DF8300042EA0E2998E81D
:10F33800070089EACE0E0FFA8EF8DFF86CE2E37167
:10F3480088EA0819AEE803005FFA89F9C8F30728C4
:10F3580088EA191848EA092181EAC90994F8088055
:10F368008EF800200FFA89F988EA090282EA021861
:10F378005FFA88F8C9F3072282EA181242EA0822DB
:10F38800607AA17A94F80B90637182EAC80212B28B
:10F39800504080EA0010C0B2C2F3072282EA10127D
:10F3A80042EA002282EAC00212B2514081EA011107
:10F3B800C9B2C2F3072282EA111242EA012282EAA2
:10F3C800C10212B289EA020989EA09195FFA89F9C0
:10F3D800C2F3072282EA191242EA092294F80C8041
:10F3E800607BA17B84F804C082EAC90212B288EA71
:10F3F800020888EA08185FFA88F8C2F3072282EA46
:10F40800181242EA082282EAC80212B2504080EA80
:10F418000010C0B2C2F3072282EA101242EA0022A8
:10F4280082EAC00212B2514081EA0111C9B2C2F3A4
:10F43800072282EA111242EA012282EAC102E17B32
:10F4480094F8109013B281EA030282EA0212D2B24F
:10F45800C3F3072383EA121343EA022383EAC203AE
:10F468001BB289EA030282EA0212D2B2C3F307236B
:10F4780083EA121343EA022383EAC2031BB283F02E
:10F48800320282EA0212D2B2C3F3072383EA1213CA
:10F4980043EA022383EAC2031BB29AB24FF0FE0882
:10F4A800DBB222800920C8210CF1010C84F802800B
:10F4B8004FEA1228AEF10E02E070A17184F87AC109
:10F4C80084F812800293637451685EF80E0C926897
:10F4D8003EF8023C0EF5CA7CACE80700ACF80030F8
:10F4E8009DF808308CF802900EF5D27A84F8B48131
:10F4F80084F8B33117F8011F306815F08FFEBA454C
:10F50800F8D1C4F864B1FFF7E0B9DFF8A0A0DFF8DC
:10F51800A080DFF8A09041200FF038FABAF9023045
:10F5280088FB0320DB17C3EBA00080B20FF014FAAE
:10F53800BAF9003088FB0320DB17C3EBA00080B2C8
:10F548000FF00AFABAF9043088FB0320DB17C3EB83
:10F55800A00080B20FF000FA99F80010386815F092
:10F568005DFE94F85C3113F0010800F097830D4AB2
:10F57800C4F858B10133DBB2A2FB0312D20802EB84
:10F588008202A3EB420384F85C31FFF77EB900BF27
:10F59800D6260020A45D0020AB5A0020E8410308CD
:10F5A80030510020CDCCCCCCDC260020E05000200F
:10F5B8006766666618800020894B8A49186815F0C6
:10F5C800F9FD00232370FFF7D8B9874F3868002862
:10F5D8003FF44AA94FF0000ADFF83C82834CAB465F
:10F5E800554615F017FEF8B1F5B94FF00109AA46CE
:10F5F800386815F007FE83B27E2B00F01F8298F85A
:10F608000120002A49D194F84811B1B11B2B84F884
:10F61800482100F0ED810D2B45D0386888F801901D
:10F6280015F0F8FD0028E3D1AA4650460AAA704909
:10F638005D460FF0C3F9FFF717B97D2B00F0CB83B8
:10F6480094F84C2122B180F02003DBB284F84C11ED
:10F6580094F84721062A10D8B4F84A113868194492
:10F66800A4F84A11A118013281F8503184F84721D1
:10F6780015F0D0FD0028BBD1D6E7B4F84A2188F8A8
:10F68800019013449BB21A0A52FA83F3FF2BA4F891
:10F698004A31386802D1574DA3E7386815F0BAFDEA
:10F6A8000028A5D1C0E73868A4F84A2115F0B2FDB2
:10F6B80000289DD1B8E794F8B832C4F8B452012BA9
:10F6C80040F2E18294F8B9224B49981801EB800185
:10F6D800013202F001024E6A84F8B922BEB1474FE6
:10F6E8000B970DF14808123FA52348F8207D80228A
:10F6F80084F8103115232946404684F8112184F8EE
:10F708001231B047002840F0438294F8B8323C4A9E
:10F71800013382FB0312A2EBE37202EB42029B1A53
:10F7280084F8B832FFF7E1B8364A374B92F80BE065
:10F73800029A1B881068D4F834213449801A4FF48F
:10F748007A72DFB202FB0EF21B0A8F770F759042B6
:10F758004FF00007CB774B758F700F7180F0808268
:10F768002B4B2C481A689B68C4F8305180FB02E781
:10F77800D21780FB03E0C2EBA702DB17C3EBA003A1
:10F7880010124FEA232C4FF0F40E0A77012748771E
:10F7980081F8203030207522782381F821C081F843
:10F7A8001AE0CF7681F8220081F8232081F82430EE
:10F7B800FEF7ECBFDFF86490D9F8000015F01EFDE5
:10F7C80000283FF470A8D9F80000012115F012FDB7
:10F7D8000222002387F8742088F80030FFF763B806
:10F7E800806E0020D46D00203C510020D4260020DB
:10F7F8001A28002024280020E8410308F9270020BF
:10F8080056555555F44E0020EC4E0020506E002001
:10F81800D0500020676666662400002074440020EB
:10F828005E209047D8F8003002209847FF200EF05D
:10F83800EDFD0378FF2B00F0668390F90130DF17A8
:10F84800FFB2D8B21CF090FC38461CF08DFCD8F8FA
:10F8580000305E209847D8F8003003209847FF20F2
:10F868000EF0D4FD0378FF2B00F04A83B0F908307E
:10F87800D8B2C3F307271CF077FC38461CF074FC99
:10F88800B34B1B78042B74D0DFF8F0A2B4F82E2108
:10F898009AF80010DFF8E89292FBF1F301FB1323CA
:10F8A8009BB2B9F80020A4F82E311F01BFB264231F
:10F8B80003FB02134900B3FBF1F347EA0327C3F341
:10F8C80003225E20D8F80030BFB217439847D8F813
:10F8D800003006209847F8B21CF046FC380A1CF0A5
:10F8E80043FC9C4AB4F82E31517AB9F800900133A0
:10F8F8000129A4F82E3100F06985537B09EB8909A9
:10F908001FFA89F9002B40F0A383D8F80030924FF2
:10F918005E209847D8F800303A209847A7FB093767
:10F928007F091FFA87FA5FFA8AF01CF01DFC4FEA7C
:10F938001A201CF019FCD8F800305E209847D8F837
:10F9480000303B209847642303FB17939BB28348FE
:10F95800053380FB0320DB17C3EBA000C0B21CF00B
:10F9680003FC00201CF000FC7D4FBB79002B40F00D
:10F97800F58294F82C31D8F80020FEF7F4BEDFF8B1
:10F9880004929FED788AA9F1300A4FF0240B5E208B
:10F9980090475846D8F800309847BAF81430F9EC30
:10F9A800016A07EE103AF8EEE66AB8EEC77A0BF18C
:10F9B800010BC6EE877A5FFA8BFB67EE887AFDEE5D
:10F9C800E77ACDED027ABDF90870F8B21CF0CCFBED
:10F9D800C7F307201CF0C8FBBBF1270F02D0D8F8EB
:10F9E8000020D4E794F82C31D8F80020FEF7B7BEF1
:10F9F800386815F00FFC00287FF40FAE386884F8DB
:10FA0800469188F8019015F005FC00287FF4F0ADC8
:10FA18000AE6FEF7A9F9544B1B68A0EB030B40F666
:10FA2800B8339B4500F2CC81504B1A793A2A00F042
:10FA3800E183002388F80030FEF735BF386884F882
:10FA480046A184F847A184F8489188F801A015F0E8
:10FA5800E1FB00287FF4CCADE6E594F8441194F876
:10FA6800453143484A1CFEF7EBBE013A84F86B2146
:10FA7800FFF720BA013B84F86A31FFF7F3B8013B7E
:10FA880084F873313DE5013F84F87271FFF7F3BAEA
:10FA98004FF0000A5E201F6884F82CA19047D8F820
:10FAA8000030DFF8E4901720984750461CF05CFBC4
:10FAB800304BA3FB07239B0BA9FB03125209C2EB94
:10FAC8000212A3EB8203D8B21CF04EFBD8F8003028
:10FAD8005E209847D8F8003018209847264BA3FB9B
:10FAE80007239B09A9FB03125209C2EB0212A3EBDD
:10FAF8008203D8B21CF038FB50461CF035FBD8F80E
:10FB08000020FEF735BE0024DFF8808027464FF03E
:10FB1800500A02E0DBB283F3118816F804B0601CC7
:10FB2800594630440EF016FE002840F067810BF16C
:10FB380001031C44EFF311838AF31288326E944256
:10FB4800E8DB0022DBB2326683F31188FEF787BF59
:10FB5800806D0020F44E00201F85EB5167666666B5
:10FB6800C050002000007A44684300205043002021
:10FB78004051002073B2E745D34D6210024F002078
:10FB8800EC4E00201851002089888888E9C10208B5
:10FB98000A9EBE4240F232843D46002141F22100D5
:10FBA80015F8013B81EA0323590013F4004F80EA5A
:10FBB800010289B292B208BF0A46530012F4004FFC
:10FBC80080EA03019BB289B208BF19464B0011F4C1
:10FBD800004F80EA03029BB292B208BF1A46530054
:10FBE80012F4004F80EA03019BB289B208BF19469C
:10FBF8004B0011F4004F80EA03029BB292B208BF97
:10FC08001A46530012F4004F80EA03019BB289B2EE
:10FC180008BF19464B0011F4004F80EA03029BB25B
:10FC280092B208BF1A46510080EA010312F4004F4D
:10FC38009BB289B218BF1946B542B1D14046F1F717
:10FC4800A1FFB4490A9DB4486D1A152DA8BF152502
:10FC58002A4622F0DFFCB14A94F8B832157056E50E
:10FC6800AF4B029A1B781268C4F83421013B012B70
:10FC78003FF676AD102202238A700B7170E51CF0F6
:10FC880053FAFEF7E5BDA74A02EB8302566A25E55B
:10FC98001CF03CFA01233B70FEF797BDA24B1B8872
:10FCA800D90515D4DA0600F17E83980600F1A08301
:10FCB800590600F1A5831A0700F1A583D80700F1BA
:10FCC800A58313F0020F0CBF4FF004084FF00C0887
:10FCD800964B974A1B78D27803F001030AB143F098
:10FCE8000203532003930EF051FE924A128802EB4E
:10FCF800820202EB8202900080B20EF02DFE0020FC
:10FD08000EF02AFE8C4A8D4912883868C2EBC2125E
:10FD1800520081FB023111444FEAE27ACAEB612AB0
:10FD28005FFA8AFA514615F079FA99F80020039B90
:10FD3800386848EA03088AEA020A002189F800A01C
:10FD480015F06CFA4146386815F068FA99F80030F1
:10FD5800386888EA0303DBB2194689F8003015F0E1
:10FD68005DFA94F85C31002B7FF401AC4F200EF063
:10FD78000DFE21F013F821F011F821F00FF8012100
:10FD8800386815F04BFA6E4A99F8003092F80080FE
:10FD9800386808F00108414683F0010389F800300B
:10FDA80015F03CFA99F80030386888EA03084146AB
:10FDB80089F8008015F032FA94F85C31FFF7D7BB68
:10FDC800604AB2F85E3100210133A2F85E3188F84A
:10FDD8000010FEF768BD386884F84C9115F01AFADF
:10FDE80000287FF405AC1FE4014684460390824650
:10FDF8000490804605900246FEF76CBF41463A20C3
:10FE08000EF004FC0743FFB291E64F494F4B0093B5
:10FE1800A1F13F074E4B4F4A099101F8404C0AA8FF
:10FE28004D490897F1F786FF089F7B1C08933C70A3
:10FE3800089B2922591C08911A70089BEA22591C10
:10FE480008911A70089BC822591C08910AA81A70B0
:10FE580021F058FC00F101080AA94246089822F04E
:10FE6800D9FB089A02EB08030133089302F808400B
:10FE7800089B5A1C08921C70089B5A1C08921C70FC
:10FE8800089B5A1C08921C70089B5A1C08921C70EC
:10FE9800089B5A1C08921C70089B5A1C08921C70DC
:10FEA800089B5A1C08921C70089B5A1C08921C70CC
:10FEB800089B5A1C08921C70089B5A1C08921C70BC
:10FEC800089B5A1C08921C70089B5A1C08921C70AC
:10FED800089B0122991812A808911A7050F8283D19
:10FEE800DB1B3B701CF062F9164B3470C3F8AC5244
:10FEF800FEF7EFBCC4F8385187F80080FEF765BC00
:10FF080000273846B7E438469CE415F073F9FEF745
:10FF180071BC00BFE427002030380020453800209D
:10FF2800806D0020E841030830510020AB5A0020C2
:10FF38001C530020EC4E0020446D00200308208054
:10FF48003C6D0020D4260020D46D0020BE72002015
:10FF5800106A0308186A0308246A0308D8F80030EE
:10FF6800DFF888A2DFF880925E209847D8F8003042
:10FF780028209847DAF8003089FB0329DB17C3EB00
:10FF8800A9095FFA89F01CF0EFF8C9F307201CF003
:10FF9800EBF8D8F800305E209847D8F800300420F5
:10FFA80098473B89002B40F00182DAF8087087F304
:10FFB8001007F8B21CF0D8F8C7F307201CF0D4F8E3
:10FFC800D7E47D4B0B93A3F1400800222121A3F134
:10FFD8003D0903F8402C88F8021088F80120CDF874
:10FFE80028900CF093F8754B754A1B8875490028C2
:08FFF8000ABF1146032704278C
:020000040801F1
:10000000580500F1E481DA0700F1F98103F00203F9
:100010006F4A002B1CBF032711463A466D4822F059
:10002000FDFA09EB070312A86B4A013340F8203DA3
:100030009B1A002209F8072088F801301CF0BAF852
:10004000FEF7C4BC654AD278002A0CBF4FF0040901
:100050004FF00509FFF739B99AF8003099FBF3F929
:1000600057E40123D9F800003B7015F0CFF807469C
:10007000D9F8000015F0CAF87F067EF4AAAB8E28E6
:100080007EF4A7AB9AF80030002B7EF4BEAB544B45
:10009000544A1A602D2384F83C31FEF7A1BBDFF8E7
:1000A00058919FED518AB9F90230454A0B9207EEFB
:1000B000903AF8EEE77A0DF1480867EE887AA2F1F7
:1000C0004003FDEEE77AA2F13D0148F8201D02F859
:1000D000400C0822CDED027A5A701E229A70BDF8AB
:1000E00008104046F1F72CFDB9F9003007EE903AC0
:1000F000F8EEE77A404667EE887AFDEEE77ACDEDD6
:10010000027ABDF80810F1F71BFDB9F9043007EECB
:10011000903AF8EEE77A404667EE887AFDEEE77AA5
:10012000CDED027ABDF80810F1F70AFD40461CF04B
:1001300041F8FEF745BC224A2C4B0B920DF14808C2
:10014000A2F13D0048F8200D1988DFF8A890A2F12F
:10015000400300204FF00A0E02F8400C082283F8FA
:1001600001E040469A70F1F7EBFCD9F800302049E5
:10017000DA1781FB0313C2EBA30399B24046F1F7F0
:10018000DFFC01F005FFD9F808900A9B4FEA1942FD
:10019000591C0A911A700A9B4FEA1922591C0A919C
:1001A0001A700A9B5A1C0A9283F800900A9B5A1CE8
:1001B0000A92187040461BF0FDFFFEF704BC00BF1A
:1001C000D46D002030510020F4690308FC69030855
:1001D0000C6A0308976D0020956D00201C530020C9
:1001E000886D0020506E002058A08B41EC4E0020FE
:1001F00067666666D0500020E0500020997803932F
:1002000018460AF09BFB00287FF417AC9549964FDF
:10021000964A974C0988DFF86C929368F9611168E7
:10022000B4F85E21F863C7F86CB0FB64F962D9F8E2
:100230000000FA6514F02AFE834600287EF432ABF3
:100240005146D9F8000014F0D9FF039B94F86021BF
:10025000DB780493642A4FF0040387F8743040F08D
:10026000178194F86131DFF820A2072B08BF84F8CA
:1002700061B194F86121069207EB021BDBF80410D0
:100280000591084621F042FADBF8083003935FFA43
:1002900080FB184621F03AFAC3B20BEB0300069A32
:1002A0000599059308308AF8070022F00F008AF8B4
:1002B0000A0002F00F0203EBCB008AF80D208AF847
:1002C0000E005A460AF10F0022F0A8F9059B039987
:1002D0000BF109001A460AF10603184422F09EF9B0
:1002E0009AF8073003F1010BD3B1013B5FFA83FCAD
:1002F0000CF1080CDFF894E1D4440AF10700002364
:1003000010F8011B59408B00CA0883EA410302F030
:1003100018024B404EFA02F253408445DBB2EFD153
:10032000544A04980BF8023022F05AF994F86131DB
:100330000022013384F8613184F860219AF8023098
:100340005BB11AF80610D9F8000014F06BFF013603
:100350009AF80230F6B2B342F3D894F8603103222F
:10036000013384F8603187F8742088F80020FFF7A3
:1003700027BA3C4B404A1B88927903EB830303EB7B
:1003800083034FEA83081FFA88F8002A53D0374BBB
:100390001B680FFA83FA01F0FBFD40B2FEF7A1BB28
:1003A00011469446039292460492FEF797BC4FF092
:1003B000340891E401F0ECFD1BF0DAFE00201BF0A4
:1003C000D7FE94F82C31D8F80020FEF7D0B90327D7
:1003D0002A4922E6D8F800305E209847D8F8003045
:1003E000392098475FFA89F01BF0C2FE4FEA1920C6
:1003F0001BF0BEFEFFF7BCBA4FF024086CE42049A6
:1004000004270AE600211DE44FF0100864E44FF0D1
:10041000200861E44FF008085EE411469446039218
:10042000924604929046FEF759BC114694460392B8
:100430009246FEF753BC4FF0FF33AAE711469446AD
:10044000FEF74CBC114694460392FEF747BC074B9F
:100450008046B3F900A06420FEF743BB1146FEF7C7
:100460003DBC00BFEC4E002024000020D0500020F6
:10047000D426002092730020C0500020006A030898
:10048000046A0308744400208C7300200007090EDE
:1004900097F87530DFF81CA10596190704BF0133E2
:1004A000DBB2072B28BF01234FEA031B07EB0B022C
:1004B0003D49107C00228AF80A2011F800C05FFA3A
:1004C0008BF203920AF10D02039E07EB0B013043FE
:1004D000BCF1010F1070C96802F101000ED9ACF136
:1004E0000206F6B206F1020E9644024602F8011B1D
:1004F00072454FEA1121F9D101363044BB4421F055
:10050000600201339BF81110DBB20A43082B027022
:1005100000F1010244D04FEA031B07EB0B00224E0F
:10052000007C224916F800C0039E511A06F1100EF5
:1005300001EB0C0606965FFA8EF60396069E132EC6
:10054000C2DD059EDFF870E0C9B28A1DD2B242F06A
:1005500040008AF8070002F1010BCAB14A1DD2B26D
:100560000832524403920EF1010C00221CF8010BD8
:100570005040820082EA4002C10842400C4801F02B
:10058000180140FA01F14A4003996145D2B2EDD118
:1005900004980BF80E2087F8753022F021F8CDE68C
:1005A0000249059E511ACDE7E841030899730020DE
:1005B0000007090E8C7300209273002008B50BF021
:1005C0003DF8024B024ADA60FEE700BF00ED00E0B2
:1005D0000400FA05024A034B127819780DF050B85E
:1005E00038230020392300202DE9F04F2DED028B18
:1005F000A0F10A0389B00C46ED2B00F27286DFE809
:1006000013F0220170067006700670067006700600
:10061000700670067006700670067006700670062A
:10062000700670067006700670067006700670061A
:1006300070062F0270067006700636067006700689
:10064000700699017006560170063E01700633016E
:1006500070062802700603027006EF01700670062D
:100660007006EA01E4017006D20170067006CC0142
:100670007006A5017006700670068A047006700682
:10068000700670066C04700602017006450632059D
:100690007006700670067006700670067006060515
:1006A0007006D8047006A50470066F0570065C0617
:1006B00070067006700670060503FB05F405C30599
:1006C000EE00700670062803A60270066F02E902AB
:1006D0007006700670067006DE0270067006BD02B7
:1006E000700670067006AF02F303BB037A03700650
:1006F000700670066C03700670064C037006700678
:100700007006700670067006700670067006700639
:100710007006700670067006700605037006700697
:100720007006700670067006700670067006700619
:100730007006700670067006700670067006700609
:1007400070067006700670067006700670067006F9
:1007500070067006700670067006700670067006E9
:10076000700670063E03700670067006700670060E
:1007700070067006700670067006700670067006C9
:1007800070067006700670067006700670067006B9
:1007900070067006700670067006700670067006A9
:1007A0007006700670067006700670067006700699
:1007B0007006700670067006700670067006700689
:1007C0007006700670067006700670067006620489
:1007D0003804700670067006700670060904AF4E85
:1007E000337853B1AE4F002537F8021F2046F1F79A
:1007F000CDF933780135AB42F6DC012009B0BDEC10
:10080000028BBDE8F08FA54E3378002BF5D0A54FB5
:100810000025B846236817F81520591C21601A7066
:1008200098F8011001EB810101EB810101F2EE2149
:1008300089B22046F1F7AAF933780135AB4208F1C5
:100840000208E7DCD9E7984D284620F05FFF002832
:10085000D3DD2B460544226813F8011B501C9D4232
:1008600020601170F7D1C8E7904D05F1800655F86A
:10087000041F2046F1F772F9AE42F8D1BDE78C4D66
:1008800005F14006B5F880102046F1F77FF923689E
:1008900095F88220591C21601A70236895F88320EE
:1008A0000435591CAE4221601A70EBD1A5E7814D89
:1008B0000B682A7A591C21601A70A98B2046F1F71F
:1008C00065F9298B2046F1F761F9698B2046F1F72C
:1008D0005DF92368EA7C591C21601A70A98C2046B6
:1008E000F1F754F9E98C2046F1F750F92368AA7F13
:1008F000591C21601A70236895F82020591C21602A
:100900001A70698C2046F1F741F92368EA7A591C7C
:1009100021601A70E9682046F1F720F923682A7CE3
:10092000591C21601A70236895F82120591C2160F8
:100930001A7062E70B68604A581C117820601970C1
:1009400023685278591C21601A7056E70B685A4A7E
:100950005A4D11785A4A581C206019701168204667
:10096000F1F7FCF82368534A591C127A21601A7077
:1009700029882046F1F70AF9A9882046F1F706F9F7
:1009800029892046F1F702F920460021F1F7FEF807
:1009900020460021F1F7FAF82FE7084608224549DA
:1009A000F1F7C4F829E70B68464A474990785D1C7F
:1009B0002560187023685278581C20601A702368CC
:1009C0000A79591C21601A7017E70B6801229918DF
:1009D00021601A7011E708460021F1F7BFF80CE713
:1009E0003A4D3B4E05F1300795F90210394B93F91A
:1009F00006208A4203F1080300F076849E42F6D175
:100A00000835BD42F0D1F8E6334B03F15A052268B0
:100A10005979501C2060117022681978501C206090
:100A2000117022685978501C2060117022689978E2
:100A3000501C206011702268D978501C2060117001
:100A4000226819790633501C9D4220601170DED156
:100A5000D3E60B68174A591C527D21601A70CCE608
:100A60001E4D05F15006287807F03AFF2368027AF8
:100A7000591C21601A7023686A78591C21601A7009
:100A80002368AA78591C21601A702368EA78043513
:100A9000591CAE4221601A70E5D1AEE63442002006
:100AA0004E6D0020E4440020765600206C5100205A
:100AB00070510020BC710020A45D00202032002075
:100AC000B85F0020805D00203C230020E8710020FA
:100AD000306B0020006B002050340020D8430020F1
:100AE000AF4D0B682A68591C127821601A702B6868
:100AF00022689978531C2360002311702A682168AA
:100B00001A4401335279481C032B20600A70F5D136
:100B100023682A68591C127A21601A7023682A688F
:100B2000591CD27821601A7023682A68591C1279DE
:100B300021601A702B6820465989F1F727F82A6836
:100B40002368527A591C21601A702A68F8E62046F8
:100B50000021F1F703F820460021F1F717F84CE6E1
:100B6000904D08462988F1F711F869882046F1F779
:100B70000DF8A9882046F1F709F83EE68A4D05F1FF
:100B80006006A9882046F1F701F8E9882046F0F7C9
:100B9000FDFF29892046F0F7F9FF2368AA7A591C3E
:100BA00021601A702368EA7A591C21601A7055F87E
:100BB0000C1B2046F0F7D2FFB542E2D11DE67B497F
:100BC00052232268501C2060137011F8013F002B43
:100BD000F7D112E6764800232268056803EB43014B
:100BE000561C6D5C26601570026825680A446E1CF0
:100BF000527826602A70026825680A440133927888
:100C0000691C0A2B21602A70E6D1F6E50025814691
:100C1000DFF8C881DFF8C8B10495039505950695FE
:100C200001214FF6FF7A05E001350B2D00F07A83A4
:100C300018F9011F4F1C4AFA05F3F5D0DE07F3D56A
:100C4000BBF800302B41D807EED505A8F1F712FB11
:100C5000EAE7584D08462988F0F798FF698820464A
:100C6000F0F794FFB5F90430534AD91782FB0323F8
:100C7000C1EBA301204689B2F0F788FFBDE50B6800
:100C80004E4A591C1278216005A81A70F0F770FEC0
:100C900023685A1C22601870AFE50B68484F591C36
:100CA0003A7821601A703B78002B3FF4A6AD0025FE
:100CB000EEB230460DF0AEFB23684278591C21603D
:100CC00030461A700DF0A6FB01892046F0F75EFF52
:100CD0003B780135AB42EBDC8FE53A4D0846298A7B
:100CE000F0F754FF698A2046F0F750FFA98A2046A2
:100CF000F0F74CFF81E5DFF8ECE00027FEB271462B
:100D000000232268501C206016702268501C20604E
:100D10001370226811F8010F0133551C062B256052
:100D20001070EED10137062F0EF1060EE6D12649DE
:100D300000232268501C206017702268501C20601D
:100D40001370226811F8010F0133551C0B2B25601D
:100D50001070EED123681D4A581C072120601970BD
:100D600023680021581C20601970236892F8F02035
:100D7000591C21601A7040E50B68154A1549107816
:100D8000154A5D1C2560187023688978581C2060FE
:100D9000197023689278591C21601A702DE500BFE4
:100DA0003851002048460020983200201C42030899
:100DB00034510020E0500020676666664C38002001
:100DC000C94D0020B0670020535200207051002010
:100DD00014630020605D0020705D00204C42030819
:100DE000305100202F5200200A68B04BB0491878CB
:100DF000551C2560107022685878551C25601070AD
:100E000022689B78501C206013702046C988F0F738
:100E1000BDFEF2E405A8F0F7ABFD00283FF4EDAC11
:100E2000BDF814102046F0F7B1FE23689DF8162097
:100E3000591C21601A7023689DF81720591C2160E5
:100E40001A7023689DF81820591C21601A702368B5
:100E50009DF81920591C21601A7023689DF81A20EA
:100E6000591C21601A702046BDF81C10F0F78EFE48
:100E7000C3E4904B03F1700522681978501C206080
:100E8000117022685978501C20601170226899787E
:100E9000501C206011702268D978501C206011709D
:100EA00022681979501C2060117022685979501CF1
:100EB00020601170226899790733501C9D42206090
:100EC0001170D9D199E47C4D0846E989F0F75EFEAE
:100ED000A9892046F0F75AFE8FE40B68774D591C1C
:100EE0002A7921601A7023686A79591C21601A7066
:100EF00029882046F0F74AFE2368AA79591C216008
:100F00001A7069882046F0F741FE2368EA79591C77
:100F100021601A7071E4F1F723FA2368684D002804
:100F200003F101010CBF0222032221601A702988FB
:100F30002046F0F713FEA9682046F0F70FFEF1F700
:100F4000B7F901462046F0F709FE56E45D4E0B68FE
:100F500072795D4D591C21601A702B682046198CDE
:100F6000F0F714FE2B682046D98BF0F70FFE71893D
:100F70002046F0F70BFEB1892046F0F707FE2B68FC
:100F80002046598CF0F702FE2B682046998CF0F72A
:100F9000FDFDF1892046F0F7F9FD318A2046F0F792
:100FA000F5FD2A68236892F82620591C21601A70E2
:100FB00023E4444EF378002B00F087820B6808226C
:100FC000591C21601A7023680122991821601A7037
:100FD00023683E4D591C2A7921601A702368AA782B
:100FE000591C21601A7029882046F0F7CFFDE98945
:100FF0002046F0F7CBFD2368F279591C21601A7066
:101000002368EA78591C21601A70FFF7F6BB0CF0D0
:101010001BFBFF28054600F0748208A8002300F897
:101020000C3D0CF0E3FA2268294B511C216015702D
:1010300022681978501C2060117022685978501C61
:101040002060117022689978501C2060117022680D
:101050009DF81410501C2060117020469988F0F7FC
:1010600095FDFFF7CABB0B681A4D591C0122216080
:101070001A702368AA78591C21601A7015F048FB71
:101080002368154A15495E1C26601870B1F90010D6
:10109000B2F90000F0F79CFF23685A1C2260187018
:1010A00029882046F0F772FDFFF7A7BB585D0020A6
:1010B0004846002058330020605D00206046002034
:1010C000C81F00201463002034510020B0670020A6
:1010D000B45A00203E6D0020DE5B0020E05B002063
:1010E00020460021F0F752FD20460021F0F74EFD8A
:1010F00020460021F0F74AFD2368AA4D00265A1C1D
:1011000022601E7023682A68591C92F82C202160E6
:101110001A7023682A68591C92F8362021601A70C8
:1011200023682A68591C92F8372021601A702368B6
:101130005A1C22601E7023685A1C22601E7023688D
:101140005A1C22601E702B682046598FF0F71EFD36
:101150002B682046198FF0F719FD23682A68591C5F
:1011600092F82E2021601A7023685A1C22601E708B
:101170002B682046598EF0F709FD2B682046998E82
:10118000F0F704FDFFF739BB874D884E9FED888A45
:10119000DFF85C82DFED878A05F120070EE0FCEEC8
:1011A000E77ACDED017ABDF8041020460435F0F75A
:1011B000EDFCAF4206F118063FF41FAB717C00292D
:1011C000F3D07D4BD5ED007A1B78012BE7D17B4B1B
:1011D0001B68DB0440F16F81F5EE407AF1EE10FA06
:1011E00040F0978140F2DC51DFE708461022744955
:1011F000F0F79CFCFFF701BB724B9B8AB3F5006FC5
:1012000000F26181B3F5806F00F28181B3F5007F58
:1012100034BF012702276C4D05F10C0655F8041B5D
:1012200091FBF7F1204689B2F0F7B0FCAE42F5D160
:10123000664D674F05F10C06B5EC010AD7ED077A4C
:1012400080EE270A21F0C0FB81B22046F0F79EFC19
:10125000B542F1D15F4D05F10C0655F8041B20464F
:1012600089B2F0F793FCB542F7D1FFF7C6BA5A4DF1
:1012700008462988F0F78AFCA9882046F0F786FC02
:1012800029892046F0F782FCFFF7B7BA0B680025E2
:101290005A1C0A601D700B685A1C0A601D700B688E
:1012A0005A1C0A60204629461D70F0F757FC294653
:1012B0002046F0F753FCFFF7A0BA0B68474A4849AD
:1012C000D078484A5D1C2560187023684979581CFD
:1012D000206019702368D278591C21601A70FFF7BA
:1012E0008CBA0020FFF78ABA23685A1C2260197052
:1012F00029882046F0F74AFC2368EA78591C2160C7
:101300001A7023682A79591C21601A702368AA79F7
:10131000591C21601A7023686A79591C21601A705F
:10132000FFF76EBBDFF8CCA000254FF0A808013511
:10133000C5F1200208FA02F2A5F120032AFA05F607
:10134000164328FA03F31E43282D06F001024FF03E
:1013500000030BD01343EAD0E8B20AF0E9FE0028FC
:10136000E5D0294605A8F0F785FFE0E71E4B1B787E
:10137000DA0700F1B68000251C4E2F4602E0013549
:10138000282D39D029463046F0F784FF0028F6D0C2
:10139000294605A8F0F77EFF002840F08780013736
:1013A000EDE700BF34510020985B0020F06600207C
:1013B0000000404200E08244D4670020B065002075
:1013C000885B0020E850002018510020A465002010
:1013D000286300209C46002020320020605D002011
:1013E0007C6F0020705D0020AB5A00204C41002033
:1013F000DB9B914190E33FF4644B654DB3F8501093
:101400002046F0F7C3FB00212046F0F7BFFB614BFD
:1014100019684B0103F02002C1F340031343C1F3E9
:10142000800243EA4203C1F3C00243EA8203C1F3EC
:10143000401243EAC20301F0100119432046F0F7BD
:10144000A5FB03A904222046F0F770FB2368297846
:10145000514A581C2060197011886429A8BF642162
:101460002046F0F793FBB9F1960F3FD000212046BC
:10147000F0F78CFB2168B7F1190348BFA7F11203FD
:10148000A3F3C4034A1C226020461A460B7004A929
:10149000F0F74CFB2368414A581C11212060197059
:1014A00020461168F0F75AFBFFF7A7B9394603A8A1
:1014B000F0F7E0FE73E7F4EEC87AF1EE10FA44DAE2
:1014C0004FF47A7171E60827A5E60B68B178344AC3
:1014D000581C2060197023681278591C21601A70FA
:1014E00076E5059B43F00103059344E72368032257
:1014F000591C21601A7023686A78591C21601A707F
:10150000B8E723685A1C22601870FFF776B90427E1
:1015100081E6F4EEC87AF1EE10FA3FF563AEF4EE30
:10152000E87AFDEEE77AF1EE10FA17EE901A1ED87F
:101530006FF4F973303903FB01F140F2E73391FBAB
:10154000F3F101F2DB5189B22FE6FDEEE77A40F2CA
:10155000E73217EE903A303B02FB03F388FB0312AD
:10156000D917C1EB622101F2E93189B21DE640F2DF
:10157000F313A1F5836103FB01F140F2E73391FB23
:10158000F3F101F2DD5189B20FE600BF64080020DB
:10159000B8720020DC500020963200202C51002030
:1015A000545D002038B5094D2B8823EA00008342A2
:1015B00028800AD0064B1421FF220E2002241C7022
:1015C00059709A7006F0A4FF288838BD3051002069
:1015D0009035002038B5094D2B8818438342288068
:1015E0000AD0074B1421FF220E2002241C705970D0
:1015F0009A7006F08DFF288838BD00BF305100205A
:1016000090350020024A136818431060704700BFED
:101610002C510020704700BF30B4034600F1240570
:10162000064C07CC0C3343F80C0C43F8081C43F869
:10163000042CAB42F4D130BC704700BF58420308C1
:10164000034B33F80C2F02809B788370704700BFE8
:10165000584203086E4B1B78002B39D02DE9F0411E
:101660006C4B6D4D9B792C682860013B82B0041B4C
:10167000032B00F29B80DFE803F0490230280AF0D8
:101680005DFD002800F09A80644B65491B786A8FE5
:10169000D1ED037A6A64DB0700F1A98002FB04F054
:1016A00007EE900ADFED5F6A5F4BB8EEE77AD5EDA3
:1016B000107A5A60E7EE267A1A60BDEEE77AC5ED39
:1016C000107A85ED0F7A83ED027A02B0BDE8F081E1
:1016D000554A1360536093607047544B1B68180160
:1016E000F3D5FF200CF096FE03780A2B88BF00216B
:1016F0004D4B9CBFB0F90420B0F90610A96488BF17
:101700000A46EA645A601A609960DEE7484A494B23
:10171000D279DFF8308133F81220B8F90230464828
:10172000B8F9001092B207EE902A40F6E44707FBA2
:1017300002F6C3EB1633B8EE670A4FF47A7606FB6F
:1017400003F393FBF1F32B61EEF7AEFED5F810E057
:10175000D5ED027ADFED336AB8F90220324BB8F9E1
:1017600000C0C3F804E00EFB04F007EE100AB8EE68
:10177000C77ABCEEC06AE7EE267A8DED016ABDF845
:101780000410C5ED027ABDEEE77A07FB01F7C2EB64
:10179000173706FB07F683ED027A96FBFCF685ED1C
:1017A000017AEE601E6002B0BDE8F0811E4B00229F
:1017B0001A605A609A6002B0BDE8F0811B4B1B684A
:1017C000DE067FF561AF154B6A8F1B786A64D90717
:1017D0007FF564AFB5F93810184B00FB01F083FBBF
:1017E0000013C017C0EBA31002446A6456E7FDEE75
:1017F000E77A134E17EE900AA0F57A7101FB01F318
:1018000086FB0306D817C0EB26100844E2E700BFAA
:10181000024F0020C050002094290020AB5A002025
:10182000044F00202FE33E31D0500020B06500204F
:10183000C4720020E4720020A8290020D34D621059
:101840001F85EB51505D0020F0B53E4B5B79012BBD
:1018500083B03DD0022B0FD03B4B00221A805A8020
:101860003A4B1B78022B05D1374A394B51881288E5
:1018700019805A8003B0F0BD364B1B681B01EFD5B1
:10188000FF200CF0C7FD03780A2B56D8B0F90220D0
:101890003149D31781FB0212C3EBA2039BB207EEBF
:1018A000903AB8EE670A2D4C04F15400A4F8523077
:1018B000EEF7FAFDFCEEC07A234AB4F85230CDEDD3
:1018C000017A5380BDF80430A4F850301380C7E784
:1018D000234A244B9278214D33F81240A4B207EEEC
:1018E000904A05F17C00B8EE670AEEF7DDFD1E4A6E
:1018F0001549107896785378FCEEC07A00EB4010CA
:10190000CDED017ABDF8042044F6FB77C3EB033339
:1019100000FB027200FB0474B2FBF3F2B4FBF3F3BE
:10192000B2FBF6F2B3FBF6F392B29BB2A5F87820C5
:10193000A5F87A300A804B8092E79FED0C0A0023CD
:10194000B1E700BFC0500020EC4E0020E84D002061
:10195000EC4D0020B0650020676666669429002083
:10196000C4720020E47200204B5E002000000000E2
:10197000F8B52D4D2D4968792D4C2E4B2E4E042255
:1019800064270A7001284FF0000184F8A02084F831
:10199000A970A4F8A210A4F8A41084F8A810C4F8A0
:1019A000AC1031701980598021D0022810D0A9794B
:1019B000224A00230129136084F8B03053609360F9
:1019C00023D0022912D11E4AE36353609360F8BD0D
:1019D000282204F1500021F0B4FF4CF250319FED69
:1019E000190A04F15400F0F701FBE0E7F8BD2822E2
:1019F00004F1780021F0A5FF4CF250319FED110A5F
:101A000004F17C00F0F7F2FAD1E70F4A636053600B
:101A10009360D3609FED0D0A02F110004CF250313B
:101A2000BDE8F840F0F7E2BAC0500020806D002019
:101A300094290020EC4E0020024F0020D0500020BE
:101A4000D0290020CDCCCC3D98290020CDCCCC3E57
:101A50002DE9F04F0C68B94F2588B94EB6FBF2F26C
:101A600085B0013B013ABC429BB2ADB292B2BDF827
:101A700038609DF83CE063D007F50067BC425FD05A
:101A8000B4F1804F5CD0A7F59837BC4258D007F529
:101A90008067BC4254D0AB4FBC4257D007F580673B
:101AA000BC4253D025F4407507F58C37ADB2BC422B
:101AB0002580E36222850ED0A34B9C420BD003F518
:101AC00040639C4207D003F580639C4203D003F53A
:101AD00080639C4201D100232386012363614B79FB
:101AE000CA79BEF1000F01D082F0010212F00201AA
:101AF00030D012F0010F4FF040054FF000020CBF44
:101B000090464FF008089446039291469646174631
:101B100001924FF4806102954FF0040A0C2B00F201
:101B2000E080DFE813F0AE00DE00DE00DE008A00B9
:101B3000DE00DE00DE006500DE00DE00DE002E00DE
:101B4000804F25F07005BC42ADB2A7D12580E3627D
:101B50002285C2E74FF4806512F0010F03954FF024
:101B600001050CBF0027022702918A4688464FF4E0
:101B700080424FF4805C4FF010094FF4807E019555
:101B8000CCE7216ADFF8B4E121F480512162216AB7
:101B90006568D4F81C8021F4005141EA0C0C7445AE
:101BA00028F4E6414CEA073741F4C04100F0E780F1
:101BB0000EF5006E744500F0E2806560E161266418
:101BC0002762E26942F40062E261626C42F4004220
:101BD00062642288214692B242F0010221F8342B3D
:101BE0000022CD1844600560CA5005B0BDE8F08FF2
:101BF000226ADFF8489122F480722262226A6568C4
